:020000040000FA
:200000000208540200800402003F00020008B522FFFFFF02008014FFFFFFFF0200801CFFAE
:20002000FFFFFF02008024504F452D47535737323234542D32344C56312E30EB7002E722CE
:2000400089828A831410E704F593E022F593E49322BB0002F722BB8000500989828A838BC1
:20006000931593F022BC000BBE0029EF8DF084FFADF022E4CCF875F008EF2FFFEE33FEEC9A
:2000800033FCEE9DEC984005FCEE9DFE0FD5F0E9E4CEFD22EDF8F5F0EE008420D21CFEADD5
:2000A000F075F008EF2FFFED33FD4007985006D5F0F222C398FD0FD5F0EA22A3F8E0C5F033
:2000C00025F0F0E582158270021583E0C838F0E822BB0006F709A7F01922BB8000500D8985
:2000E000828A838B931593F0E5F0A3F022E88FF0A4CC8BF0A42CFCE98EF0A42CFC8AF0ED79
:20010000A42CFCEA8EF0A4CDA8F08BF0A42DCC3825F0FDE98FF0A42CCD35F0FCEB8EF0A40D
:20012000FEA9F0EB8FF0A4CFC5F02ECD39FEE43CFCEAA42DCE35F0FDE43CFC22EB9FF5F0F0
:20014000EA9E42F0E99D42F0E89C45F022E8600FEFC333FFEE33FEED33FDEC33FCD8F122D5
:20016000BB0006E9F802000332BB8000500C89828A838B9315930200017B22ECF0A3EDF035
:20018000A3EEF0A3EFF022EB700C87F009E608B5F019DFF6801589828A831410E70FF59383
:2001A000E0F5F0A3E608B5F002DFF5806AF593E493F5F0A3E608B5F05EDFF4805ACB701311
:2001C00088828C838B9387F009E493A3B5F048DFF580441410E71F88848C858B9589828ACD
:2001E00083F593758620E0F5F0E493A3A3B5F024DFF4DEF2801E88848C858B9589828A83F8
:20020000F593758620E493F5F0E493A3A3B5F004DFF3DEF17586007FFFB5F0020F22400245
:200220007F012202000187809488F0EF60010E4E60F0ED60EE1410E7EECB701288828C8370
:20024000F59387F009E0A3B5F0CDDFF680C91410E71E88848C858B9589828A83F593758682
:2002600020E0F5F0E0A3A3B5F0AADFF5DEF380A488848C858B9589828A83F593758620E47F
:2002800093F5F0E0A3A3B5F08BDFF4DEF28085EB7008E709F608DFFA801B89828A831410E7
:2002A000E70AF593E0A3F608DFFA8009F593E493A3F608DFF9ECFAA9F0EDFB2288F0EF601A
:2002C000010E4E60F088F0ED60C51410E7E7CB700E88828C838B93E709F0A3DFFA80D614AF
:2002E00010E71C88848C858B9589828A83F593758620E0F0A3A3DFFADEF875860080B68875
:20030000848C858B9589828A83F593758620E493F0A3A3DFF9DEF77586008099C5F0F8A3AF
:20032000E028F0C5F0F8E582158270021583E038F022ECF608EDF608EEF608EFF62290008E
:200340007004E0F54090007005E0F541854082854183E020E7077E007F00C2D72289428A6E
:20036000435407F54512000539E02402F54450020545120003E0053AE53A7002053BE54050
:200380002544F540E541354530E604C2E6242DF5411200040090007004E540F090007005A2
:2003A000E541F0AE45AF44D2D72290007010E020E61EA3EDF0A3E9F0A3EAF0EC5407D2E6EA
:2003C00090007010F00538E53870020539D2D7227C007D00C2D72290007010E0A2E6B32247
:2003E00075F001800375F0041200040078407F06900070921200052190007090E5F0F02217
:2004000090007090E0540770F7221200046D90007008742DF0900070107508101200045861
:20042000E490007004F090007006F0742D90007005F090007007F0751D10751C10751E008B
:20044000751F2D75832D758200E4F0753800753900753A00753B0022E4A808F0A3D8FC22F2
:20046000120005171200040A120004AB22900004A175080A79707860120005287518C075CD
:2004800019A8751A00751B647510C07511A87512007513017514FF7515FF7516FF7517006E
:2004A00022000B78667788C0A800649000706AE0440CF0229000706AE054F3F02290007017
:2004C0006AE04401F0229000706AE054FEF0229000706AE04402F0229000706AE054FDF0A0
:2004E000229000706AE04440F0229000706AE054BFF02290007000E04410F0229000700045
:20050000E054EFF02290007000E04420F02290007000E05420F0229000700AF000000000F0
:2005200022E6F008A3DFFA2289A0E493A3F208B800030989A0D508F222A3E58330E6037569
:20054000832D22754300754200754100754000754508754400120003E5754308754200758E
:200560004108754000754508754400120003E51200040090000000750910750800750B00D7
:20058000750A0012000638400B9000706CE04408F0D2D722C2D7227543007542007541000E
:2005A000754000754508754400120003E5754308754200754108754000754508754400129A
:2005C0000003E51200040090000000750910750800750B00750A00120006384051754310DA
:2005E000754200754110754000754508754400120003E575431875420075411875400075D5
:200600004508754400120003E51200040090001000750910750800750B10750A00120006F2
:2006200038400B9000706CE04418F0D2D722C2D722E6F008A3DFFA22A90B89A0A80AE49397
:20064000F5F0A3E265F0701008B800030989A01200067D50E9C2D722D2D722A90B89A0A88D
:200660000AE0F5F0A3E265F0701008B800030989A01200067D50EAC2D722D2D722E50860BA
:200680000A14F50845097007D2D72215091508C2D7229000700B7418F09000700C7420F0A2
:2006A00075A06022120006927824E2E2B408157400F21200072912000721120007071200B4
:2006C000070E802E22120006927816E2E2703708E2E2B4013178281200079C5029120007F9
:2006E0003912000779120007411200078178177402F27800E2E2FC4480F208E2E2FD7918FC
:200700007A20120003AA22781AE4F208F222782680F7E2E2F5F0E3E3F2E5F0F30809DAF2BF
:20072000227A04781C792080E9790878027A0680E1E2E2F30809DAF922780879027A0680EF
:20074000F0780879227A0680E8E4F309F3227A08E480037A04E4F309DAFC22E0F3A309E013
:20076000F3227A04E0F3A309DAFA227A0280027A04E2E2F0A308DAF922900070607A068041
:20078000E3781879227A0A8089E0F5F0E2E265F0700708A3DAF3D2D722C2D7229000706605
:2007A0007A0480E59000200AE0FEA3E08E8375820075814F73220D0A205446333331465556
:2007C0003A333956463038302031364B2D626173656420426C616E6B20436865636B696E64
:2007E00067002E2E2E5B6661696C5D0A002E2E2E5B6F6B5D0A000D0A205446333331465581
:200800003A6465766963655B53535420333956463038305D000D0A20544633333146553A7F
:20082000536563746F722D62617365642832353620736563746F72732920466C61736820DD
:2008400045726173652028314D29002E2E2E5B6F6B5D2E0075C7AA75C755759D02787FE409
:20086000F6D8FD900000007F007E607D01E4F0A3DFFCDEFADDF875814F12000517D20D12DF
:200880000004B41200040A12001DE312001DFF12000FB8EF7004020008A5020008AF12008A
:2008A0001D22EF700AC20D120004AB02000C57D20D02008000300D040200800CC0E0C0D03B
:2008C00075D00012001D98D0D0D0E0320D0A436865636B20436865636B53756D3D0030787D
:2008E00025782E2E2E4F4B21210D0A00307825782E2E2E4661696C21210D0A001B5B324A48
:20090000000D0A436865636B204D6167696320436F64652E2E2E004F4B2121004661696C64
:200920002121000D0A2849503D200025752E00257529000D0A284D41433D200025782E007D
:20094000257829000D0A54463333313A205446545020646F6E652E204A756D7020746F201E
:20096000307825782E0A00496C6C6567616C206669726D77617265002E000D0A20496E7631
:20098000616C6964206669726D776172652021000D0A20466C617368206572726F7220214F
:2009A000004387049000555574AAF090002AAA7455F09000555574A0F08F828E838D93E59F
:2009C0002EF05387FB229000262FEEF0A3EFF0E4784EF608F6D390002630E094009000263C
:2009E0002FE094005003010C5690002620E0FF94094003010B12EF705E9000262FE0FEA3C8
:200A0000E0FFD39400EE94004031784EE6FC08E67B012448F974203CFA1200003B643A6011
:200A20001A90002630E024FFF09000262FE034FFF0784F06E61870C10680BEEF4E700301EA
:200A40000C56784B7601900026207401F0784F06E618704F06804C90002620E0784BF6787C
:200A60004BE6C39409504E90002630E094009000262FE09400403E784E0806E61886067048
:200A80000106147B012448F974203EFA1200003BFF784BE6062423F582E43426F583759317
:200AA00000EFF090002630E024FFF09000262FE034FFF080AA784BE690002620F0C394099D
:200AC0005003010C569000261A7426F0A37423F0120018BDEF64014E700690002620F022F5
:200AE000120018BDEF64044E7003010C077D027F01120018C19000261CEFF07D067C007FCA
:200B0000037E00120018C590002614EEF0A3EFF0807E9000261DE0FFA3E090002614CFF07F
:200B2000A3EFF090002621E06066D390002630E094009000262FE0940040559000261A7457
:200B400026F0A37421F0784E0806E6188606700106147B012448F974203EFA1200003B90E4
:200B6000002622F090002630E024FFF09000262FE034FFF07D017C00E4FFFE120018C512A0
:200B800000152CE490002621F09000261CE014F09000261A7420F0A37448F0A3E0FF784CCA
:200BA000760008A607D3784DE6940018E694004049D390002630E094019000262FE0940056
:200BC0004038784EE6FE08E6FF2401FDE43EFC120018C51200152C784F740226F618E436F9
:200BE000F618E6161870011690002630E024FEF09000262FE034FFF080AB784DE690002600
:200C00001CF0E61846700890002620F00109D59000262FE07004A3E064017026784E0806DC
:200C2000E6188606700106147B012448F974203EFA1200003B90002621F0E49000262FF025
:200C4000A3F090002614E0FFA3E09000261DCFF0A3EFF00109D5227F0A7E0012001A69EF35
:200C6000784AF612001DC0900070FFE0784AF61200127D7E097F23E4FDFC12000E50E478C3
:200C80004AF6784AE6FDC39403501E7E097F2B74042DF582E43420F583759300E0FD7C0049
:200CA00012000E50784A0680D97E097F2F90002007E0FD7C0012000E507E097F33E4FDFCD8
:200CC00012000E50E4784AF6784AE6FDC39405501E7E097F3C74122DF582E43420F5837508
:200CE0009300E0FD7C0012000E50784A0680D97E097F4090002017E0FD7C0012000E507B26
:200D0000017A2079181200033E90002608EEF0A3EFF0D39424EE940040E590002026E0B49A
:200D2000081FA3E0B4061A90002609E024F0F090002608E034FFF0120006C5784AA6078005
:200D4000BE90002026E0B408B6A3E0B400B19000202AE0FFA3E090002608CFF0A3EFF090FA
:200D6000002034E0FCA3E0FDA3E0FEA3E0FF900020001200017BE4784AF6784AE6FF7C00C3
:200D80007B012420F9EC3420FA1200003BFE740C2FF582E43420F583759300EEF006E6B4B9
:200DA00006D890002028E064456003010CFF9000202EE0543F6003010CFF90002031E0B450
:200DC000010E120006A4E490002608F0A3F0805190002031E0B411499000203EE07004A39E
:200DE000E06445701690002609E024E4F090002608E034FFF01200111B80269000203EE0DA
:200E000064FC7004A3E064036003010CFF90002609E024E4F090002608E034FFF012001625
:200E2000389000264DE07003010CFF12001E259000200A741FF0A374FCF07E097F44FD7CC0
:200E40001F12000E50C2A9C2AF120007A4010CFF90002638EEF0A3EFF0A3ECF0A3EDF09081
:200E6000002638E475F001120000BB85F082F583759300E4939000263DF07003010FB7E012
:200E800064256003010F989000263C740AF090002638E475F001120000BB85F082F5837575
:200EA0009300E49324DB7003010F98800090002639E024FFF090002638E034FFF090002605
:200EC00038E475F001120000BB85F082F583759300E4939000263DF0E0249D601424EE606B
:200EE0001924FD6003010F989000263C7410F080099000263BE0FF010FB09000263E740ABC
:200F0000F09000263AE07002A3E0605A9000263CE0FBFD7C009000263AE0FEA3E0FF1200BA
:200F20000065AA059000263AE0FEA3E0FFEBFD7C00120000659000263AEEF0A3EFF0D3EA65
:200F400064809489EA40052457FF80032430FF9000263EE014F0244EF582E43426F5837525
:200F60009300EFF0809B9000263EE0B40A047F30803E9000263EE0C3940A4003010E5FE01B
:200F8000FF04F0744E2FF582E43426F583759300E0FF12001E3780DA9000263DE0FF1200B4
:200FA0001E379000263DE0640A6003010E5F7F0D12001E37010E5F22E4FFFEFDFC900026B7
:200FC0002F1200017BE490002633F07F0AFE12001A69EF12001DC07E087FFCE4FDFC1200AD
:200FE0000E507E097F01E4FDFC12000E507FFC7EFF7D0F7C00900026341200017B90002611
:201000002FE0F8A3E0F9A3E0FAA3E0FBC000C001C002C003A3E0FFE4FDFEA3A3E0F9A3E049
:20102000FAA3E02FFFEE3AFEED39FDE42FFFE43EFEED3481FDA907AA06AB051200003BFF8F
:20104000D003D002D001D000EB4FFFEAFEE9FDE8FC9000262F1200017B9000262FE0FCA388
:20106000E0FDA3E0FEA3E0FF78081200014D9000262F1200017B90002633E004F0E0C39449
:20108000035003010FFD9000262FE0F8A3E0F9A3E0FAA3E0FBC000C001C002C003A3E0FF31
:2010A000E4FDFEA3A3E0F9A3E0FAA3E02FFFEE3AFEED39FDE42FFFE43EFEED3481FDA9073A
:2010C000AA06AB051200003BFFD003D002D001D000EB4FFFEAFEE9FDE8FC9000262F12003C
:2010E000017B7F557EAA7D557CAA9000262FE0F8A3E0F9A3E0FAA3E0FBC31200013C700DBD
:201100007E097F17FDFC12000E507F01227E097F1CE4FDFC12000E507F002290002044E0C3
:20112000FEA3E0FFEE600301127CEF24FD606404600301127C12001C3C9000203CE0FFA3AD
:20114000E090002643CFF0A3EFF09000203EE0FEA3E0FF90002641EEF0A3EFF090002044DC
:20116000E4F0A37404F0E4A3F0A3F09000203CEEF0A3EFF090002643E0FFA3E09000203EF1
:20118000CFF0A3EFF090002608E4F0A37404F0020013D59000203EE0FEA3E0FF9000264142
:2011A000E06E7003A3E06F60030112749000263FE0FEA3E0FF90002046E0B50608A3E0B56C
:2011C000070301127090002640E02401FF9000263FE03400FE90002046E06E7003A3E06FD8
:2011E00060030112749000203CE0FFA3E090002643CFF0A3EFF07E097F78E4FDFC12000E02
:2012000050C390002609E09404FF90002608E09400FE120009C69000262EE0702B9000265F
:2012200017E0C3941450067E097F7A80047E097F90E4FDFC12000E507F047E0012001BD011
:201240009000264D7401F02290002640E004F070079000263FE004F0C390002609E0940400
:2012600090002608E0940250079000264D7401F002001D5EE490002608F0A3F022D2A9D26A
:20128000AFE49000262FF0A3F09000262FE0FEA3E0FFC39402EE9400505BEF2404FFE43E50
:2012A000FE12001A6990002631EEF0A3EFF0E0FD90002630E025E0FB9000262FE033FA744B
:2012C000042BF58274203AF583759300EDF090002631E0FF74052BF58274203AF58375930E
:2012E00000EFF090002630E004F0709D9000262FE004F08094E49000262FF0A3F090002679
:201300002FE0FEA3E0FFC39403EE9400505412001A6990002631EEF0A3EFF0E0FD9000264F
:2013200030E025E0FB9000262FE033FA74122BF58274203AF583759300EDF090002631E091
:20134000FF74132BF58274203AF583759300EFF090002630E004F070A49000262FE004F0B1
:20136000809BE4784BF6784BE6FF2404F582E43420F583759300E0FEEF2466FDE434708D4D
:2013800082F583759300EEF006E6B404D9E4784BF6784BE6FF2412F582E43420F583759346
:2013A00000E0FEEF2460FDE434708D82F583759300EEF006E6B406D99000706CE054FDF0DE
:2013C00090007001743FF0900070007410F0900070DAE4F02290002609E02408FE900026A6
:2013E00008E0340090002040F0A3CEF0E4A3F0A3F090002000E0FCA3E0FDA3E0FEA3E0FF77
:20140000900020381200017B90002004E0FCA3E0FDA3E0FEA3E0FF900020341200017B9041
:20142000002609E0241CF090002608E03400F0900020287445F0E4A3F09000202E7440F031
:20144000E4A3F0A37410F0A304F090002608E0FFA3E09000202ACFF0A3EFF090002009E093
:2014600004F0700790002008E004F090002008E09000202CF090002009E09000202DF0E4C7
:2014800090002032F0A3F0900020187490F090002609E02412F090002608E03400F0C3A33E
:2014A000E0944090002608E094005006E4F0A37440F090002018E054F8FE90002608E04EF7
:2014C000FFA3E090002018CFF0A3EFF0E4FF740C2FF582E43420F583759300E0FEEF7C0077
:2014E0007B01241AF9EC3420FAEE120000510FEFB406DBE4FF74122FF582E43420F58375E7
:201500009300E0FE74202FF582E43420F583759300EEF00FEFB406DD900020267408F0A310
:20152000E4F07B017A207918020003AA90002618EEF0A3EFF090002614E475F0011200002D
:20154000BBAFF090002631F0A3EFF090002619E0FF9000262CF090002046E07004A3E06427
:201560000160030115E790002631E0FCA3E0FDC39427EC9400403CD3ED943AEC94005033BC
:2015800090002617E004F08D828C83759300E4936F6006E49000262DF090002617E0B4140C
:2015A000129000262DE07004A3F080079000262E7401F090002616E0702DA3E064147027A4
:2015C0009000262EE06020E4F52F1200059712001725120017FCEF70069000262EF02290B3
:2015E0000026167401F02290002631E0FEA3E04E7002052F9000262EE06401703A90002663
:2016000016E0640170319000262CE0FDF46028E52F7011C3EE9440401E90002631E0FEA3B3
:20162000E0FF800F90002631E0FEA3E0FF9000262CE0FD12001B62227FD87E5A7D947C01C8
:2016400090002054E0F8A3E0F9A3E0FAA3E0FBC31200013C600301172490002046E0FEA30F
:20166000E0FF64014E6007EF4E6003011724E490002052F0A3F090002050E0FEA3E0FFEEDE
:201680006003011724EF24FB600B24FB600924096003011724802D78127C207D017B017A97
:2016A0002079487E007F0612000229EF707690002608E4F0A37428F090002050E4F0A37488
:2016C0000BF0800E12001C8F90002050E4F0A3740CF078487C207D017B017A2079127E00E4
:2016E0007F06120002BC90002044E4F0A37402F0A3E4F0A304F09000204EE4F0A37402F0DB
:201700009000203EE0FEA3E0FF9000203CE0FDA3E0A3CDF0A3EDF09000203CEEF0A3EFF003
:20172000120013D5227E077FF6E4FDFC12000E507E087F15E4FDFC12000E50E4F52FF523BF
:20174000752408AE23AF24E4FCFDFB7A10F9F8120000ED8F288E278D268C25A2AFE433F5C5
:2017600022C2AF4387049000555574AAF090002AAA7455F0900055557480F074AAF09000E7
:201780002AAA7455F0E47FFF7EFFFDFCAB28AA27A926A825D31200013C401BE42528FFE413
:2017A0003527FEE5263401FDA907AA06AB05743012000051800C8528828527837593007415
:2017C00030F05387FBE52224FF92AFAE23AF24E4FCFDFB7A10F9F8120000ED120019E7059C
:2017E00024E52470020523C3E523940150030117437E087F4BE4FDFC02000E507E077FB6CD
:20180000E4FDFC12000E50E4752502F524F523F522E47F3FFEFDFCAB25AA24A923A822D313
:201820001200013C40030118AFE4F526F527E4FF7E40FDFCAB25AA24A923A822120000ED66
:201840008F2B8E2A8D298C28E4FCFDE52B2527F52BE52A3526F52AED3529F529EC3528F523
:2018600028E4252BFFE4352AFEE5293481FDA907AA06AB051200003BF4600D7E077FE2E484
:20188000FD12000E507F00220527E52770020526C3E52694404097E5252401F525E4352466
:2018A000F524E43523F523E43522F5220118117E077FEDE4FDFC12000E507F01227D087F5B
:2018C000077C007E0090002631ECF0A3EDF0E4A3F0A3F0AD07AC06C390002632E09D90009C
:2018E0002631E09C40629000261AE0FEA3E08E837593002DF582E5833CF583759300E0F988
:2019000090002634E0C4F8540FC868F090002633E0C454F048F0E9D39439500BE9C3943061
:20192000FFE49400FE8013C3E99441FFE49400CF240ACF3400FE90002633E04EF0A3E04FD0
:20194000F00DBD00010C808F90002633E0FEA3E0FF229000263AEEF0A3EFF09000265C7470
:2019600008F0F5C84402F0F5C87F327E0012001E249000265CE04404F0F5C87F647E0012E2
:20198000001E2412001E169000265A7408F0A3E4F09000265AE0FCA3E0FD4C6043A3E0549A
:2019A000FAF09000263AE0FEA3E0FFEC5EFEED5F4E60089000265CE04404F09000265CE087
:2019C00012001E1E12001E209000265CE04401F0F5C89000265AE0C313F0A3E013F080B118
:2019E0009000265CE0FF22900026361200017B752901E4F52CF52D90002636A3E0FDA3E0A5
:201A0000FEA3E02400FFE43EFEED3481FDA907AA06AB051200003BF52A532A40E52960407C
:201A200090002636A3E0FDA3E0FEA3E02400FFE43EFEED3481FDA907AA06AB051200003BF7
:201A4000F52B532B40E52AB52B03E4F529852B2A052DE52D7002052CB4FFC1E52CB4FFBCFF
:201A6000E5297F0060027F0122C2AFEE4408FE120019529000265CEFF0E490002638F0A359
:201A8000F09000265A7480F0A3E4F09000265AE07002A3E060379000265CE054FA12001EFF
:201AA0001D12001E16AFC8EF30E3149000265AE0FEA3E0FF90002638E04EF0A3E04FF09068
:201AC00000265AE0C313F0A3E013F080BE9000265CE054F8F0F5C87F907E0112001E24D27D
:201AE000AF90002638E0FEA3E0FF229000262FEBF0A3EAF0A3E9F0E490002637F0A3F0902A
:201B000000263574FFF5F0120000BB45F0604690002632E0FBA3E0FAA3E0F91200003BFF62
:201B20009000262FE0FBA3E0FAA3E0F990002637E475F001120000BBFCE925F0F9EA3CFAD5
:201B4000EF1200005160B890002633E475F0011200031C80AA9000262FE0FBA3E0FAA3E0CD
:201B6000F92290002633EEF0A3EFF0A3EDF0AF2FE4FCFDFEFBFA7901F8120000ED8F268E1F
:201B8000258D248C2390002633E0FEA3E0FFE4FCFDE5262FF526E5253EF525ED3524F52484
:201BA000EC3523F523A3E0F52EA2AFE433F522C2AFAF26AE25AD24AC23120009A1AF26AEAC
:201BC00025AD24AC23120019E7E52224FF92AF22900070007429F090002044E4F0A3740530
:201BE000F0A3EEF0A3EFF064044E7020900026327481F0A37409F0A37467F0A3E4F0A374D3
:201C000011F07B017A20794812001AEB90002641E0FFA3E09000203CCFF0A3EFF090002699
:201C200043E0FFA3E09000203ECFF0A3EFF090002608E4F0A37415F0020013D5E49000269E
:201C40003FF0A3F090002000E0FCA3E0FDA3E0FEA3E0FF900026451200017BE4900026414F
:201C6000F0A3F0A3F0A3F09000264DF09000262EF090002617F090002616F09000262D0494
:201C8000F0900070007421F0900070DAE4F0227B017A20796CE475F004120000D174022935
:201CA000F9E43AFAE475F008120000D1740229F9E43AFA90002004E0FCA3E0FDA3E0FEA3FB
:201CC000E0FF12000160740429F9E43AFEC3E99444FFEE942090002608F0A3EFF0229000F5
:201CE000262FEEF0A3EFF0E4F523D3ED9400EC9400402C9000262FE0FEA3E0AA06F97B8108
:201D00001200003B2523F523ED1D70011C90002630E004F070D49000262FE004F080CBAFCE
:201D200023227E087FCCE4FDFC12000E50E4F522FD7C80FF7E8012001CDE8F22E522B4FFD8
:201D40000E7E087FDEFD7C0012000E507F01227E087FECAD227C0012000E507F002290002A
:201D60002044E4F0A37404F090002641E0FFA3E09000203CCFF0A3EFF090002643E0FFA31F
:201D8000E09000203ECFF0A3EFF090002608E4F0A37404F0020013D5C0D0C2A9C2AFE54913
:201DA0002401F549E43548F548E43547F547E43546F546758C5D758A3DD2AFD2A9D0D02294
:201DC0007598504387805389CF438920EFB40108758DF3758CF38006758DE5758CE5D28E7D
:201DE000D29922E58954F04401F589758C5D758A3DE4F549F548F547F546D2B9D28C2275F1
:201E000098504387805389CF438920758DE5758CE5D28ED299229000265CE04401F0F5C85B
:201E20007FF47E01229000706CE054E7F022AF49AE48AD47AC46223099FDC2998F9922FF95
:201E4000FFFFFFFFFFFFFFFFFFFFFFFFFFFFFFFFFFFFFFFFFFFFFFFFFFFFFFFFFFFFFFFFA2
:201E6000FFFFFFFFFFFFFFFFFFFFFFFFFFFFFFFFFFFFFFFFFFFFFFFFFFFFFFFFFFFFFFFF82
:201E8000FFFFFFFFFFFFFFFFFFFFFFFFFFFFFFFFFFFFFFFFFFFFFFFFFFFFFFFFFFFFFFFF62
:201EA000FFFFFFFFFFFFFFFFFFFFFFFFFFFFFFFFFFFFFFFFFFFFFFFFFFFFFFFFFFFFFFFF42
:201EC000FFFFFFFFFFFFFFFFFFFFFFFFFFFFFFFFFFFFFFFFFFFFFFFFFFFFFFFFFFFFFFFF22
:201EE000FFFFFFFFFFFFFFFFFFFFFFFFFFFFFFFFFFFFFFFFFFFFFFFFFFFFFFFFFFFFFFFF02
:201F0000FFFFFFFFFFFFFFFFFFFFFFFFFFFFFFFFFFFFFFFFFFFFFFFFFFFFFFFFFFFFFFFFE1
:201F2000FFFFFFFFFFFFFFFFFFFFFFFFFFFFFFFFFFFFFFFFFFFFFFFFFFFFFFFFFFFFFFFFC1
:201F4000FFFFFFFFFFFFFFFFFFFFFFFFFFFFFFFFFFFFFFFFFFFFFFFFFFFFFFFFFFFFFFFFA1
:201F6000FFFFFFFFFFFFFFFFFFFFFFFFFFFFFFFFFFFFFFFFFFFFFFFFFFFFFFFFFFFFFFFF81
:201F8000FFFFFFFFFFFFFFFFFFFFFFFFFFFFFFFFFFFFFFFFFFFFFFFFFFFFFFFFFFFFFFFF61
:201FA00075C7AA75C755759D02787FE4F6D8FD900000007F007E607D01E4F0A3DFFCDEFA5B
:201FC000DDF875814F12000517C20D120004B41200040A12001DE312001DFFC20D120004DB
:201FE000AB02000C57FFFFFFFFFFFFFFFFFFFFFFFFFFFFFFFFFFFFFFFFFFFFFF020008548A
:20200000FFFFFFFFFFFFFFFFFFFFFFFFFFFFFFFFFFFFFFFFFFFFFFFFFFFFFFFFFFFFFFFFE0
:20202000FFFFFFFFFFFFFFFFFFFFFFFFFFFFFFFFFFFFFFFFFFFFFFFFFFFFFFFFFFFFFFFFC0
:20204000FFFFFFFFFFFFFFFFFFFFFFFFFFFFFFFFFFFFFFFFFFFFFFFFFFFFFFFFFFFFFFFFA0
:20206000FFFFFFFFFFFFFFFFFFFFFFFFFFFFFFFFFFFFFFFFFFFFFFFFFFFFFFFFFFFFFFFF80
:208000000200B811257300740074002202022930740074000202DD403098FDAF99C2987EA8
:208020000022740002008FFF020083BDE86480F8E933E83360110460EFED33EC337009E879
:20804000FCE9FDEAFEEBFF220460DDD3EB9FEA9EE99DE8C2E78CF0C2F795F0400CE8CCF85B
:20806000E9CDF9EACEFAEBCFFB1200838885D0F05804700320D5B1E80470085002B2D502D4
:208080000083C792D5EC0460F6E4CCC0E0C398F8603C94186009400ED0E0FB0200839FE494
:2080A000FBFAC9FC8028E830E406E4C9FBE4CAFCE830E305E4C9CACBFCE854076010F8C35E
:2080C000E913F9EA13FAEB13FBEC13FCD8F130F531C3E49CFCEF9BFFEE9AFEED99FDD0E020
:2080E000FBEF4E4D4C701322DB04020083C4EC2CFCEF33FFEE33FEED33FDED30E7EA020081
:20810000839FEF2BFFEE3AFEED39FDD0E0FB50140BBB0004020083C7ED13FDEE13FEEF13B8
:20812000FFEC13FC0200839FEC4D6011E8497018ED33EC3304600DE4FCFFFEFD22E933E80E
:20814000330470F8020083BD1200838858046009E4CC2481500728500B020083C728400475
:20816000020083C4C0E0EB4A7046B98007D0E0FB020083B3EF4E701DBD8008EBFFEAFEE93E
:20818000FD80EAE98DF0A4FEE5F002008217E9CDF9EAFEEBFFEF89F0A4FCE5F0CE89F0A4B7
:2081A0002EFFE435F0CD89F0A42DFEE435F08067EF4E7005BD80D780C2EF8BF0A4ACF0EEE4
:2081C0008BF0A42CFCE435F0F8EF8AF0A42CE5F038FCE433CB8DF0A42CFCE5F03BF8EE8A6A
:2081E000F0A42CFCE5F038F8E433CF89F0A42CFCE5F038CF3400CE89F0A42FFFE5F03EFE59
:20820000E433C98DF0A42EFEE5F039CD8AF0A42FFFE5F03EFEE43DFD33D0E0FB50080BBBDF
:208220000010020083C7EC2CFCEF33FFEE33FEED33FD0200839F020083C7EC5D046005E867
:2082400059047004020083BD12008388580460F4EC4860F0EC7004FDFEFF22C860D8248199
:20826000C8500AC39860025007020083C49850C6F582E9294B4A7006AB82020083B375F073
:20828000007C1A7880C3EF9BEE9AED99400DC3EF9BFFEE9AFEED99FDE842F0DC24ACF0D0CD
:2082A000E0FFD0E0FED0E0FDAB8220E7101BEB60B8EC2CFCEF33FFEE33FEED33FD0200832C
:2082C0009FE803F830E705C0F075F000EF2FFFEE33FEED33FD40B730E7C180A974F8CC64FE
:2082E00080CCC86480C8F582046043C3EB9FF5F0EA9E42F0E99D42F0E89C45F0603050184B
:20830000E5825FFFE582F42B5582FB50210ABA001D09B90019088016E5825BFBE582F42F2E
:208320005582FF50090EBE00050DBD00010CC3EB9FF5F0EA9E42F0E99D42F0E89C45F060A9
:2083400007CC4820E701B3EC2275F020800E75F010800575F0087D007E007F003392D5307B
:20836000D50412008932EC334010EF33FFEE33FEED33FDEC33FCD5F0ED22E5F0247EA2D5AE
:2083800013CC92E7CDCEFF22E9D2E7C933E833F892D5EDD2E7CD33EC33FC5002B2D522EC09
:2083A00030E7100FBF000C0EBE00080DBD00040BEB6014A2D5EB13FCED92E7FD2274FFFC4B
:2083C000FDFEFF22E480F8A2D574FF13FC7D80E480EFF920E73624F950037907E4F42402B8
:2083E000FBE582158270021583DBF6E024FB501BE96014E4F0E582158270021583E004F032
:20840000B40A08E4F0D9EE7401F00A22C2D522ED33EC3392D5FA602AB4FF33EDC2E77BFF91
:2084200060067A847934E4227A84793D20D5047A847938224E614E002B494E46002D494EDE
:208440004600E47A08F0A3DAFC7B00740722C093C083C082ECC0E0EDC0E0EEC0E0EFC0E0E1
:20846000EA75F010A4CAABF075F04DA42BFBE435F0FCEA2410FAEB34C5FBEC34D9FCEDC278
:20848000E7FF75F056A4F42411C5F0F434C58FF0A42AE5F03BE43CF020E7161200855DD07E
:2084A000E0FFD0E0FED0E0FDD0E0FC1200823A8016F4041200855DD0E0FFD0E0FED0E0FD7C
:2084C000D0E0FC12008128D082D083D093E0FAEDD2E7CD33EC332482FBE4C3CF33CFCE3374
:2084E000CECD33CD33DBF37B0775F00A846004F0A31B0AE5F0F0A38FF0740AA4FFACF08E1D
:20850000F0740AA42CFEACF050010C8DF0740AA42CFDE435F0F0A3DBDE740722ED33EC332D
:20852000600A047003BD8004ECB2E7FC223F8000004120000042C80000447A0000461C40EC
:208540000047C35000497424004B1896804CBEBC205A0E1BCA6753C21C749DC5AEFB6006B7
:2085600054076020232312008590EB5438600C1200857B1200858B12008128ECF8EDF9EE29
:20858000FAEFCB22EB1200858B80F0543803241C9000852DFE93FC0EEE93FD0EEE930ECEF3
:2085A00093FF22EB7008E709F608DFFA801B89828A831410E70AF593E0A3F608DFFA8009AA
:2085C000F593E493A3F608DFF9ECFAA9F0EDFB2288F0EF60010E4E60F088F0ED60C5141078
:2085E000E7E7CB700E88828C838B93E709F0A3DFFA80D61410E72A89828A83F593ECFAE0E0
:20860000A3C8C582C8CCC583CCCBC593CBF0A3C8C582C8CCC583CCCBC593CBDFE2DEE080DB
:20862000AA89828A83F593ECFAE493A3C8C582C8CCC583CCCBC593CBF0A3C8C582C8CCC550
:2086400083CCCBC593CBDFE1DEDF020085CBEB7002E72289828A831410E704F593E022F502
:2086600093E49322F8EB7006E7C828F3E82289828A831410E708F593E0C828F0E822F5939C
:20868000E49322BB000327F722F8EB89828A831410E706F593E028F022F593E4932822BB91
:2086A0000002F722BB8000500989828A838B931593F022EF8DF0A4A8F0CF8CF0A428CE8D01
:2086C000F0A42EFE22BC000BBE0029EF8DF084FFADF022E4CCF875F008EF2FFFEE33FEEC1F
:2086E00033FCEE9DEC984005FCEE9DFE0FD5F0E9E4CEFD22EDF8F5F0EE008420D21CFEADEF
:20870000F075F008EF2FFFED33FD4007985006D5F0F222C398FD0FD5F0EA22C2D5EC30E7E2
:2087200009B2D5E4C39DFDE49CFCEE30E716B2D5E4C39FFFE49EFE120086C5C3E49DFDE403
:208740009CFC8004120086C530D507C3E49FFFE49EFE22C5F0F8A3E028F0C5F0F8E582153C
:208760008270021583E038F022A3F8E0C5F025F0F0E582158270021583E0C838F0E822EB41
:208780007007E7F5F009E7192289828A831410E708F593E0F5F0A3E022F593E493F5F074F6
:2087A000019322F8EB700C09E5F027C7F5F019E837C72289828A831410E707F593E8020036
:2087C0008769F593E4740193F5F0E49322BB000B09C5F027F7C5F01937F722F8EB89828A7F
:2087E000831410E707F593E802008753F59374019325F0F5F0E4933822BB0006F709A7F0E5
:208800001922BB8000500D89828A838B931593F0E5F0A3F022E88FF0A4CC8BF0A42CFCE926
:208820008EF0A42CFC8AF0EDA42CFCEA8EF0A4CDA8F08BF0A42DCC3825F0FDE98FF0A42CB0
:20884000CD35F0FCEB8EF0A4FEA9F0EB8FF0A4CFC5F02ECD39FEE43CFCEAA42DCE35F0FDFB
:20886000E43CFC2275F008758200EF2FFFEE33FECD33CDCC33CCC58233C5829BED9AEC991A
:20888000E58298400CF582EE9BFEED9AFDEC99FC0FD5F0D6E4CEFBE4CDFAE4CCF9A8822293
:2088A000B800C1B90059BA002DEC8BF084CFCECDFCE5F0CBF97818EF2FFFEE33FEED33FD73
:2088C000EC33FCEB33FB10D703994004EB99FB0FD8E5E4F9FA227818EF2FFFEE33FEED336D
:2088E000FDEC33FCC933C910D7059BE99A4007EC9BFCE99AF90FD8E0E4C9FAE4CCFB22759B
:20890000F010EF2FFFEE33FEED33FDCC33CCC833C810D7079BEC9AE899400AED9BFDEC9A8B
:20892000FCE899F80FD5F0DAE4CDFBE4CCFAE4C8F922C3E49FFFE49EFEE49DFDE49CFC2216
:20894000EB9FF5F0EA9E42F0E99D42F0EC6480C864809845F022EB9FF5F0EA9E42F0E99D1C
:2089600042F0E89C45F022E8600FECC313FCED13FDEE13FEEF13FFD8F122E8600FEFC333B1
:20898000FFEE33FEED33FDEC33FCD8F122EB7006E9F802008F3A89828A831410E706F593D8
:2089A00002008F46F59302008F52BB0006E9F802008FABBB8000500C89828A838B93159322
:2089C00002008A6922EB7006E9F802008F9489828A831410E706F59302008A3DF593020015
:2089E0008F52EB7006E9F802008F6289828A831410E706F59302008F6FF59302008F7B74A8
:208A000001FF3395E0FEFDFCA3A3A3E0CF2FF0E582158270021583E0CE3EF0E582158270AE
:208A2000021583E0CD3DF0E582158270021583E0CC3CF0227401FF3395E0FEFDFCA3A3A3C4
:208A4000E02FFFF0E582158270021583E03EFEF0E582158270021583E03DFDF0E5821582F4
:208A600070021583E03CFCF022ECF0A3EDF0A3EEF0A3EFF022F5F0C582A4C582C5F0C5832D
:208A8000A42583F58322A42582F582E5F03583F58322E0FBA3E0FAA3E0F922F8E0FBA3A3F8
:208AA000E0F925F0F0E582158270021583E0FA38F022F8E0FBA3A3E025F0F9F0E5821582B7
:208AC00070021583E038FAF022EBF0A3EAF0A3E9F022EB7006E9F802008FB789828A8314BC
:208AE00010E706F59302008A92F59302008FC9BB001CD093D0F0D0E0F8D0E0C9FBD0E0FA31
:208B0000D0E0CBC8C0E0C0F0C09302008FC0BB80005022D093D0F0D0E0F8D0E0C9F582D0E6
:208B2000E0CAF583D0E0CB14C8C0E0C0F0C093889302008AC9D093D083D082D0E0D0E0D071
:208B4000E0E473D093D083D082F8E4937012740193700DA3A393F8740193F5828883E473AE
:208B60007402936860EFA3A3A380DFD093D083D082F8E4937012740193700DA3A393F8742A
:208B80000193F5828883E473740293B5F0067403936860E9A3A3A3A380D88B938A838982DF
:208BA000159353937FE473759308E5582582F582E5573583F583B557048582582210AF0624
:208BC000858258F55722858258F557D2AF22759308E5582582F582E5573583F58322EB7026
:208BE0000C87F009E608B5F041603F80F489828A831410E70FF593E0F5F0A3E608B5F02A23
:208C0000602880F3F593E493F5F0A3E608B5F01A601880F2CB701588828C838B9387F00934
:208C2000E493A3B5F004600280F380611410E72E89828A83F593ECFAE0F5F0A3C8C582C8BD
:208C4000CCC583CCCBC593CBE493A3C8C582C8CCC583CCCBC593CBB5F033603180DA8982B9
:208C60008A83F593ECFAE493F5F0A3C8C582C8CCC583CCCBC593CBE493A3C8C582C8CCC553
:208C800083CCCBC593CBB5F004600280D97F00F845F0600EE863F0806480D395F01F4002C1
:208CA0007F012202008BDE02008C14ED60F51410E7F5CB701488828C83F59387F009E0A3D0
:208CC000B5F0CA60C880F480C41410E72D89828A83F593ECFAE0F5F0A3C8C582C8CCC58334
:208CE000CCCBC593CBE0A3C8C582C8CCC583CCCBC593CBB5F097609580DB89828A83F59366
:208D0000ECFAE493F5F0A3C8C582C8CCC583CCCBC593CBE0A3C8C582C8CCC583CCCBC5936C
:208D2000CBB5F0A360A180DAEB7008E709F60870FA801B89828A831410E70AF593E0A3F641
:208D40000870FA8009F593E493A3F60870F9ECFAA9F0EDFB2288F0ED60CE1410E7F0CB70BD
:208D60000E88828C83F593E709F0A370FA80DF1410E72889828A83F593ECFAE0A3C8C582AD
:208D8000C8CCC583CCCBC593CBF0A3C8C582C8CCC583CCCBC593CB70E280B589828A83F571
:208DA00093ECFAE493A3C8C582C8CCC583CCCBC593CBF0A3C8C582C8CCC583CCCBC593CB43
:208DC00070E1808CEB700C87F009E608B5F019DFF6801589828A831410E711F593E0F5F0B8
:208DE000A3E608B5F002DFF502008E75F593E493F5F0A3E608B5F07DDFF48079CB70138829
:208E0000828C838B9387F009E493A3B5F067DFF580631410E73089828A83F593ECFAE0F5B0
:208E2000F0A3C8C582C8CCC583CCCBC593CBE493A3C8C582C8CCC583CCCBC593CBB5F03561
:208E4000DFDCDEDA802F89828A83F593ECFAE493F5F0A3C8C582C8CCC583CCCBC593CBE4E2
:208E600093A3C8C582C8CCC583CCCBC593CBB5F004DFDBDED97FFFB5F0020F2240027F01E5
:208E80002202008DC402008DFC88F0EF60010E4E60EEED60EC1410E7ECCB701288828C83CA
:208EA000F59387F009E0A3B5F0CBDFF680C71410E72F89828A83F593ECFAE0F5F0A3C8C5E6
:208EC00082C8CCC583CCCBC593CBE0A3C8C582C8CCC583CCCBC593CBB5F09ADFDDDEDB801E
:208EE0009489828A83F593ECFAE493F5F0A3C8C582C8CCC583CCCBC593CBE0A3C8C582C85A
:208F0000CCC583CCCBC593CBB5F004DFDCDEDA02008E75EF4E6022EF60010EEDBB0007F79F
:208F200009DFFCA9F022BB8000500E89828A838B931593F0A3DFFCDEFA22E6FC08E6FD08DE
:208F4000E6FE08E6FF22E0FCA3E0FDA3E0FEA3E0FF22E493FC740193FD740293FE74039314
:208F6000FF22E6FB08E6F908E6FA08E6CBF822E0F8A3E0F9A3E0FAA3E0FB22E493F87401F8
:208F800093F9740293FA740393FB227401FF3395E0FEFDFC080808E62FFFF618E63EFEF6B6
:208FA00018E63DFDF618E63CFCF622ECF608EDF608EEF608EFF622E6FB08E6FA08E6F9229B
:208FC000EBF608EAF608E9F622E493FB740193FA740293F922EFB40A08740D12008FE174FB
:208FE0000A309811A899B8130CC2983098FDA899C298B811F63099FDC299F5992274003286
:2090000032342D506F72742031302F31303020506F45202B20322D506F72742047696761AC
:2090200062697420536D617274205377697463680000000000000000000000000000000038
:209040000000000000000000000000000000000000555352393937363234000000000000D1
:209060000000000000000000000000000000000000000000000000000000312E30302E30D3
:209080003300740074000012233445660180C200000F00000000000084382484382C8438CB
:2090A0002F84383261000A3C7472206865696768743D33303E0A203C746420616C69676E26
:2090C0003D63656E7465723E3C623E25730A203C74643E3C623E0A00844CB8844CC6844CD0
:2090E000D4844CE7844CFB844D12844D2A844D3E844D12844D55844D64844D78844D8A84C7
:209100004D9D20203C696E70757420747970653D636865636B626F78206E616D653D2573BD
:209120002076616C75653D25642025733E2025733C62723E0A00203C74643E0A203C736576
:209140006C656374206E616D653D25733E0A203C6F7074696F6E2076616C75653D25643E53
:2091600025730A003C74723E3C746820636F6C7370616E3D343E25730A3C74723E0A203CAE
:2091800074643E3C623E42797465730A203C746420636F6C7370616E3D333E256C750A0AC0
:2091A000003C74723E0A203C74643E3C623E25730A203C74643E256C750A203C74643E3C25
:2091C000623E25730A203C74643E256C750A0A007400740074007400740074003C74723EA9
:2091E0003C746820636F6C7370616E3D27382720616C69676E3D6C6566743E504F452050DF
:209200006F7274205374617475730A3C74723E0A203C74642077696474683D27333027205F
:20922000616C69676E3D2763656E746572273E3C623E49440A203C74642077696474683DB5
:209240002738302720616C69676E3D2763656E746572273E3C623E506F6520456E61626CE1
:20926000650A203C74642077696474683D273130302720616C69676E3D2763656E746572DF
:20928000273E3C623E706F776572206C696D69740A203C74642077696474683D27353527AE
:2092A00020616C69676E3D2763656E746572273E3C623E506F7765722857290A203C74646A
:2092C0002077696474683D2736302720616C69676E3D2763656E746572273E3C623E566F47
:2092E0006C746167652856290A203C74642077696474683D2737302720616C69676E3D27BB
:2093000063656E746572273E3C623E43757272656E74286D41290A203C7464207769647493
:20932000683D273130302720616C69676E3D2763656E746572273E3C623E436C61737369F9
:209340006669636174696F6E0A203C74642077696474683D273230302720616C69676E3DBD
:209360002763656E746572273E3C623E5374617475730A3C2F74723E0A003C74723E0A2053
:209380003C74642077696474683D343020616C69676E3D63656E7465723E3C623E49440A3E
:2093A000203C74642077696474683D393020616C69676E3D63656E7465723E3C623E506FD1
:2093C0006520456E61626C650A203C74642077696474683D31303020616C69676E3D636545
:2093E0006E7465723E3C623E706F776572206C696D69740A00485454502F312E30203230A4
:2094000030204F4B0D0A507261676D613A206E6F2D63616368650D0A436F6E74656E742D7C
:20942000547970653A20746578742F68746D6C0D0A436F6E6E656374696F6E3A20636C6FC8
:2094400073650D0A0D0A3C68746D6C3E0A3C6C696E6B2072656C3D7374796C65736865656D
:209460007420687265663D666F726D2E6373733E0A3C736372697074206C616E6775616733
:20948000653D6A6176617363726970743E0A66756E6374696F6E2068656C7028290A7B0A9C
:2094A0002077696E646F772E6F70656E282768656C702E68746D2361636C272C20276865EB
:2094C0006C70272C2027746F703D3231302C6C6566743D3232302C77696474683D37393022
:2094E0002C6865696768743D3435302C7363726F6C6C626172733D79657327293B0A7D0AE4
:209500003C2F7363726970743E0A3C68313E495020416363657373204C69737420536574DD
:2095200074696E673C2F68313E0A3C7461626C6520626F726465723D312077696474683D60
:209540003235303E0A3C747220616C69676E3D63656E7465723E0A203C74642077696474CD
:20956000683D34303E3C623E49440A203C74643E3C623E495020616464726573730A000A30
:209580003C74723E0A203C746420616C69676E3D63656E7465723E3C623E253032640A2015
:2095A0003C74643E25642E25642E25642E25640A000A3C747220616C69676E3D63656E7463
:2095C00065723E0A203C74643E266E6273703B0A203C74643E416C6C20686F7374204950BA
:2095E000206164647265737320616C6C6F7765640A003C2F7461626C653E0A0A3C666F720B
:209600006D206E616D653D6164645F61636C20616374696F6E3D6367695F61646461636C61
:20962000206D6574686F643D4745543E0A203C696E70757420747970653D68696464656E0D
:20964000206E616D653D6E756D2076616C75653D25643E0A3C2F666F726D3E0A3C666F7287
:209660006D206E616D653D64656C5F61636C20616374696F6E3D6367695F64656C61636CE9
:20968000206D6574686F643D4745543E0A3C2F666F726D3E0A3C7461626C65207769647441
:2096A000683D3235303E0A3C74723E0A203C74643E0A203C74642077696474683D35303EEC
:2096C0003C696E70757420747970653D627574746F6E2076616C75653D2741646427206F03
:2096E0006E636C69636B3D6164645F636865636B28293E0A203C74642077696474683D35B4
:20970000303E3C696E70757420747970653D627574746F6E2076616C75653D2744656C6599
:20972000746527206F6E636C69636B3D64656C5F636865636B28293E0A203C74642077698A
:209740006474683D353020616C69676E3D72696768743E3C696E70757420747970653D6276
:209760007574746F6E2076616C75653D2748656C7027206F6E636C69636B3D68656C70284D
:20978000293E0A3C2F7461626C653E0A0A3C736372697074206C616E67756167653D4A6176
:2097A00076615363726970743E0A66756E6374696F6E2064656C5F636865636B28290A7B27
:2097C0000A2069662028646F63756D656E742E6164645F61636C2E6E756D2E76616C75653A
:2097E000203D3D2030290A207B0A2020616C65727428274E6F2049502041636365737320F8
:209800004C69737427293B0A202072657475726E3B0A207D0A20646F63756D656E742E643A
:20982000656C5F61636C2E7375626D697428293B0A7D0A66756E6374696F6E206164645FDB
:20984000636865636B28290A7B0A2069662028646F63756D656E742E6164645F61636C2E80
:209860006E756D2E76616C7565203D3D202564290A207B0A2020616C65727428274578636B
:20988000656564206D6178696D756D20495020416363657373204C697374206E756D62655E
:2098A0007227293B0A202072657475726E3B0A207D0A20646F63756D656E742E6164645FA0
:2098C00061636C2E7375626D697428293B0A7D0A3C2F7363726970743E0A3C2F68746D6C11
:2098E0003E006E756D3D006E756D3D256400485454502F312E3020323030204F4B0D0A50B6
:209900007261676D613A206E6F2D63616368650D0A436F6E74656E742D547970653A207458
:209920006578742F68746D6C0D0A436F6E6E656374696F6E3A20636C6F73650D0A0D0A3CF1
:2099400068746D6C3E0A3C6C696E6B2072656C3D7374796C65736865657420687265663D34
:20996000666F726D2E6373733E0A3C666F726D206D6574686F643D504F53543E0A3C683143
:209980003E495020416363657373204C6973742053657474696E673C2F68313E0A3C696E65
:2099A00070757420747970653D68696464656E2076616C75653D2564206E616D653D6163FE
:2099C0006C5F69643E0A3C7461626C6520626F726465723D312077696474683D3335303E04
:2099E0000A3C747220616C69676E3D63656E7465723E0A203C74642077696474683D3830F1
:209A00003E3C623E49440A203C74643E3C623E253032640A0A3C747220616C69676E3D635B
:209A2000656E7465723E0A203C74643E3C623E495020616464726573730A203C74643E3C1B
:209A4000623E3C62723E0A00203C696E70757420747970653D74657874206E616D653D6937
:209A6000702073697A653D34206D61786C656E6774683D333E2E0A003C62723E3C62723EC0
:209A80000A3C2F7461626C653E0A0A3C7461626C652077696474683D3335303E0A203C7486
:209AA0006420616C69676E3D72696768743E3C62723E3C696E70757420747970653D7375BD
:209AC000626D69742076616C75653D274170706C79273E0A3C2F7461626C653E0A0A3C695A
:209AE0006E70757420747970653D68696464656E206E616D653D706F73745F75726C207608
:209B0000616C75653D6367695F61636C2E3E0A3C2F666F726D3E0A3C2F68746D6C3E00481C
:209B20005454502F312E3020323030204F4B0D0A507261676D613A206E6F2D63616368653C
:209B40000D0A436F6E74656E742D547970653A20746578742F68746D6C0D0A436F6E6E6537
:209B60006374696F6E3A20636C6F73650D0A0D0A3C68746D6C3E0A3C6C696E6B2072656CA4
:209B80003D7374796C65736865657420687265663D666F726D2E6373733E0A3C68313E496D
:209BA0005020416363657373204C6973742044656C6574653C68313E0A3C666F726D206D1A
:209BC0006574686F643D504F53543E0A3C7461626C6520626F726465723D3120776964747E
:209BE000683D3235303E0A3C747220616C69676E3D63656E7465723E0A203C74642077695A
:209C00006474683D33303E266E6273703B0A203C74642077696474683D33303E3C623E4991
:209C2000440A203C74643E3C623E495020416464726573730A000A3C74723E0A203C746457
:209C400020616C69676E3D63656E7465723E3C696E70757420747970653D636865636B62F2
:209C60006F78206E616D653D7663622076616C75653D25643E0A203C746420616C69676E1A
:209C80003D63656E7465723E3C623E253032640A203C74643E25642E25642E25642E2564D7
:209CA0000A000A3C2F7461626C653E0A3C62723E0A3C7461626C652077696474683D323555
:209CC000303E0A203C746420616C69676E3D72696768743E3C696E70757420747970653D89
:209CE0007375626D69742076616C75653D27204170706C7920273E0A3C2F7461626C653EC9
:209D00000A3C696E70757420747970653D68696464656E206E616D653D6E756D2076616C91
:209D200075653D25643E0A3C696E70757420747970653D68696464656E206E616D653D70D6
:209D40006F73745F75726C2076616C75653D6367695F64656C61636C2E3E0A3C2F666F7262
:209D60006D3E0A3C2F68746D6C3E00706F72743D00706F72743D25303264007370656564D0
:209D80003D0073706565643D2564007365745F716F733D007365745F716F733D256400733D
:209DA00065745F666C6F773D007365745F666C6F773D2564006367695F736574706F7274AA
:209DC0003D256400506F72742053657474696E67004D6564696120747970652069732063D9
:209DE00068616E6765642E3C62723E43757272656E742073706565642073657474696E674E
:209E0000206973206E6F74207375697461626C652E00766C616E5F69643D00766C616E5F04
:209E200069643D256400646573633D0026006367695F766C616E00564C414E205365747459
:209E4000696E6700564C414E206465736372697074696F6E206D75737420626520756E6993
:209E6000717565007663623D007663623D25303264006367695F736574766C616E3D256467
:209E800000496620616E7920706F727420696E206120564C414E2047726F75702062656C7D
:209EA0006F6E677320746F2061207472756E6B2C2074686520564C414E2047726F757020E8
:209EC0006D75737420696E636C75646520616C6C20706F72747320696E20746861742074A8
:209EE00072756E6B2E006E756D3D006E756D3D2564007663623D2564006367695F64656C09
:209F0000766C616E0076747970653D0076747970653D25640044656661756C7400737276FD
:209F20003D007379733D006C6F633D006C6F67696E3D0053797374656D2053657474696E5B
:209F40006700496E76616C696420485454502073657276657220706F7274006367695F73D2
:209F6000797300496E76616C6964206C6F67696E2074696D656F75742076616C7565006928
:209F8000703D00496E76616C69642049502061646472657373006D6B3D00496E76616C6916
:209FA00064207375626E6574206D61736B0067773D00496E76616C69642067617465776145
:209FC00079204950004950207375626E6574206D75737420657175616C20746F2067617485
:209FE00065776179207375626E65740061636C5F69643D0061636C5F69643D2564004950A6
:20A0000020416363657373204C6973742053657474696E67006367695F61636C006F6C6413
:20A020005F706173733D006E65775F706173733D0072656E65775F706173733D00436861B0
:20A040006E67652050617373776F72640070617373776F7264206C656E6774682063616EEC
:20A060006E2774206265207A65726F006367695F70617373006F6C642070617373776F7259
:20A08000642069732077726F6E67006E65772070617373776F726420697320696E636F6E03
:20A0A00073697374656E7400547261702053657474696E6700496E76616C696420547261F3
:20A0C00070204950006367695F74726170006669623D00636F703D00706F653D00257325E3
:20A0E000256400656E61626C65253032643D00746B70253032643D002530326426005472FA
:20A10000756E6B2053657474696E6700416C6C20706F72747320696E2074686520747275AF
:20A120006E6B206D7573742062656C6F6E6720746F207468652073616D6520564C414E2823
:20A1400073292E006367695F7472756E6B006D6F64653D006D6F64653D2530326400736EDF
:20A1600069666665723D00736E69666665723D25303264006D63623D006D63623D2530321C
:20A180006400647669643D00647669643D256400647072693D00647072693D25640056490A
:20A1A000442025303264206973206E6F742065786973742C6F7220506F72742025303264B9
:20A1C000206973206E6F7420746865206D656D626572206F662056494420253032642E00E8
:20A1E000276367695F707669642700505649442053657474696E67007669643D0056494438
:20A200002053657474696E6700564944206D757374206265206265747765656E20322061B0
:20A220006E642034303934006367695F616464766964005468652056494420697320657840
:20A2400069737420696E20564944207461626C65007025643D002564007461675F69643D28
:20A26000007461675F69643D2564005468652064656661756C7420766964206F6620706F33
:20A28000727420253032642069732025642C20736F2069742063616E6E2774206265207526
:20A2A0006E73656C65637465642E00276367695F7365747669643D256427005468652076CD
:20A2C0006964206973207468652064656661756C7420766964206F6620706F72742025309D
:20A2E00032642C20736F2069742063616E6E27742062652064656C657465642E0063676903
:20A300005F7365747669643D25640052656D6F766520564C414E007061737377643D00708B
:20A320006F72745F69643D00706F72745F69643D2564006D676D6E743D006D676D6E743DE8
:20A340002564007077725F6C696D007077725F6C696D3D2564007468726573686F6C645F8E
:20A3600076616C75653D00504F452053797374656D2053657474696E6700496E76616C6999
:20A380006420506F776572205468726573686F6C642053657474696E67006367695F7370EC
:20A3A0006F6573797300E5502456F582E43430F583759308E0055022900830533027049017
:20A3C000083056E475F00112008A9B0200864E2020E57F2ED2208018EF540F2490D43440EE
:20A3E000D4FF30240BEF24BFB41A0050032461FFE551600215510554E55470020553302703
:20A400001190083053E475F00112008A9BEF0200869F02008FD57403D2278003E4C227F55E
:20A42000509008305312008AC9E4F551F553F554E55160087F201200A3F080F47552FFC2B3
:20A4400021C220C222C223C225C226C2281200A3B8FF700E3027067F001200A401AF54AE49
:20A460005322B42563C2D5C2241200A3B8FF24D0B40A00501A75F00A785130D50508B6FF27
:20A480000106C6A426F620D5047002D22380D824CFB41A00EF5004C2E5D2240200A73ED21D
:20A4A0002180C4D22080BED22280BAD2D580B8D22580B27F201200A3F02022077401B551C9
:20A4C0000040F01200A3A6FF1200A3F00200A430D228D226808F1200A3A6FB1200A3A6FACB
:20A4E0001200A3A6F94A4B7006794B7AA87B8120223DE55160397E00E9C0E02EF9EAC0E015
:20A500003400FA1200864EF9D0E0FAD0E0C960060EEE655270E2C2D5EBC0E0EAC0E0E9C04B
:20A52000E0EE1200A7A6D0E0F9D0E0FAD0E0FB1200864EFF6096EBC0E0EAC0E0E9C0E01265
:20A5400000A3F0D0E02401F9D0E03400FAD0E0FBE5520460DAD552D70200A4CCD222808F29
:20A560001200A78260F6E552700104120083D2A952600EE552600A14F5521200A835EF6094
:20A58000F2EA30E702F404C39940040200A615EAF425520430E701E404F552800F1200A789
:20A5A0008260B9EA05522552120083D2EA90083082F030E701E4255204D5520420250114C1
:20A5C0001200A7A6E4C0E01200A83590083082E0601420E70814F01200A3D8802604F0D001
:20A5E000E014C0E07F001200A3D8E55260081200A3CF1552800D3025041200A3CFD0E00215
:20A6000000A430D0E00480BD1200A7826093E55204120083D290083082EAF0E55220250203
:20A6200060010424041200A7A674FF04C0E01200A8351200A3D8E55220250260041200A304
:20A64000CFD0E0B552E57F451200A3E290083082E07F2B30E7047F2DF404C0E01200A3F05C
:20A66000D0E075F00A84C0F01200A3D9D0E01200A3D90200A430791080027908C226C22887
:20A680008008D2D5790A8004790AC2D5E552047002F552E4FAFDFEFF1200A3A6FC7B0820A4
:20A6A00021161200A3A6FD7B1030200C1200A3A6FE1200A3A6FF7B20EC3382D592D5501396
:20A6C000C3E43020069FFFE49EFEE42021039DFDE49CFCE4CBF8C221EC700CCFCECDCCE811
:20A6E00024F8F870F38017C3EF33FFEE33FEED33FDEC33FCEB33FB994002FB0FD8E9EB3037
:20A700002105F8D0E0C448B221C0E00AEC4D4E4F78207B0070C2EAB5520040BCC0E0120028
:20A72000A7A8D0F0D0E0202104C4C0E0C4B221C0F01200A3D9D0F0D5F0EA0200A430120085
:20A740008B43A4D653A67658A4A34CA49F42A67A4FA68244A68249A4B943A68855A59D46DB
:20A76000A60845A56047A86850A4A72DA4AB2EA4D22BA4AF23A4D020A8542AA46548000023
:20A78000A4C8E552B4FF037552061200A3A6FC1200A3A6FD1200A3A6FE1200A3A6FF900899
:20A7A000307B0200840F790AA2D5202314302509B910020404B9080104A2D5202602500101
:20A7C0000420226D9222B551005036C0E07F2030231A7F30A2227226722550101200A8011D
:20A7E000C222C226C225C2287F308010302503E9C0E01200A3F0302503D0E0F9D0E0B55140
:20A80000CA3025197F30B9100D1200A3F07F583024077F788003B908041200A3F030220668
:20A820007F2D0200A3F07F202028F77F2B2026F222922280CC7F00B40700500E247BF58247
:20A84000E43430F583759308E0FF22286E756C6C2900D2211200A3A63021F7C221785130A9
:20A86000D50108F60200A4651200A3A67F4960087F4310E7027F5814C0E0EF1200A3E1742F
:20A880003A1200A3E1D0E0600DC0E0C41200A3D9D0E01200A3D9D2237551040200A676417D
:20A8A0002D4F00442D6000000000422D660000412D7803412D7700442D9300000000422D35
:20A8C0009E0000422D91000043321BFFFFFF4A387B00000000000000000000413A24FF4171
:20A8E0003CE80142329D000A4232A50000423299000042329B000042329500004232A700BF
:20A900000042329FFFFF42329780004432910000000042328B000042328D000042328F0091
:20A92000004120F0004231DB00004F367D84335084335C84336D84337F84336D4C37478490
:20A940003EFC843F04843F07843F0A462F40841CA6841CAD582F28841CB2841CBA841CC25A
:20A96000841CCB841CD4841CDD841CE4841CEB582F52841CF3841CFB841D05841D0F841D6E
:20A9800018841D21841CB2841D26462F46841CB2841D2B462F4C841D32841D3648324A00BC
:20A9A00001000900110019483262000800100018001A432E4E000000623F041083E72963D3
:20A9C00067695F64756D790000000000000000000000008315336367695F6C6F67696E0013
:20A9E00000000000000000000000838D336367695F706F72740000000000000000000000BD
:20AA00000082101D6367695F736574706F727400000000000000000082CAC26367695F76CE
:20AA20006C616E0000000000000000000000008300076367695F736574766C616E000000C2
:20AA400000000000000082AE846367695F64656C766C616E00000000000000000082BE7812
:20AA60006367695F707669640000000000000000000000008225A16367695F766964000074
:20AA800000000000000000000000008299E36367695F6164647669640000000000000000BA
:20AAA000000081DCAA6367695F6465766963650000000000000000000081EB246367695F6B
:20AAC00064657461696C000000000000000000008254B66367695F737461746973740000D9
:20AAE00000000000000000830BEF6367695F7472756E6B0000000000000000000000822C65
:20AB0000366367695F6D6972726F72000000000000000000008309916367695F706173736C
:20AB20000000000000000000000000008249926367695F73797300000000000000000000C7
:20AB400000000081F4F76367695F7472617000000000000000000000000083CCA26367691C
:20AB60005F6261636B7570000000000000000000008342FF6367695F62616B5F6461746183
:20AB8000000000000000000083CCEF6367695F72657365740000000000000000000000833F
:20ABA00047A76367695F706F65000000000000000000000000008232756367695F736574CA
:20ABC000706F65000000000000000000008387026367695F73706F6573797300000000007D
:20ABE000000000000000000000000000000000000000000000000000000000423BCF000009
:20AC0000422E4A0000422E4C0000421D4A0000421C110000411B2300411BEC00491BEF810B
:20AC2000B0EF81B0FD81B125521D1381B13981B15181B16881B17F81B19881B1B54C1D25F6
:20AC400081B1D381B1F081B20E81B225551B0E81B23E81B24D81B25E81B27081B28481B2A7
:20AC60009981B2B6421AF200004A38E9FC06FC03FC0400A120004217870001433C5683FF9F
:20AC8000F1433C5983FFF3433C5C83FFF5433C5F818007423BE30000423BE500005235589D
:20ACA00084641C84642484642A84643184643A846442433C68819084433C6B83FFF7433CAF
:20ACC0006E8191D6443525000000004435290000001444352100000001433C7A81800943E9
:20ACE0003C7D818010433C80818012433C83818022433C86818FFD433C8981BA62442FC762
:20AD0000000000004F2FCB84000784000E84002A8400378400454C2FDA84004E8400538419
:20AD2000005984005F492FAC84006484006D840072522FB584007684007E84008684008E96
:20AD400084009684009E00E527302C0104F823282412F582E43431F583759308229008319E
:20AD60000F302C0490083112E475F00112008A9B0200864E60E6C52B7002152A14C52B2027
:20AD80002C05FF0200BA599008310F74FFF5F002008AB2FF0202E124E5286006D528037F06
:20ADA0000022202C101200BA2CEF6008052BE52B7002052A229008310F12008A9212008625
:20ADC0004EFF60E59008310FE475F00112008A9B80D71200ADA2EFC0E01200AD93D0E040FF
:20ADE000F18091D22C8002C22C9008310F12008AC9E4F529F527F52AF52B752800C22BC2FD
:20AE000029C22AC22D1200AD5DFF7005AF297E0022B425321200AD5DFF24D0B40A00500CF2
:20AE200075F00AC528A42528F52880E824CFB41A00EF5002C2E50200B0BAD22A80D6D229DE
:20AE400080D2D22D80CEEF1200AD9350091200ADD2EF600F80A4EFC0E01200ADA2D0E06F97
:20AE60006098EF70040200AEED1200AD74809D1200ADA2EF6077E52870080528800412001B
:20AE8000ADA2EF6017202D111200AD47E475F00112008A9BEF1200869FD528E2202D0405BD
:20AEA00027052980AF1200AD98EFC0E01200AD93D0E050051200AD74E4FF202D111200AD9E
:20AEC00047E475F00112008A9BEF1200869FEF70D4202D04052705290200AE54E528600233
:20AEE00005281200ADD21200AD98EF70BD302C05E41200AD74E52960030200AE0C7EFF7F80
:20AF0000FF22E528600205281200ADD2D22FD22E1200AD98EF302F0260D3C0E01200AD7435
:20AF2000D0E0AC2CAD2DAE2EAF2F1200B7368C2C8D2D8E2E8F2F50081200ADA2C22E80D011
:20AF4000202D13202E0205291200AD4712008A920527120089AA0200ADFAD0E0808F79008D
:20AF6000800A7910800679088002790AD22EE52860020528E9C0E01200ADD2EF60DC1200BF
:20AF8000ADA2BF2D04D22B8003BF2B0B1200ADD2EF60C71200AD98D0E0B40A028034B4081F
:20AFA00002802FBF302870027408C22EC0E01200AD98D0E0BF78028003BF58160528D52831
:20AFC000028007D52804D22E800B7410801B7002740ABF000BEFF8E4FCFDFEFF0200B062AE
:20AFE000C0E0EF1200AD74D0E0F9E4FCFDFEFFE9C0E0ECC0E0EDC0E0EEC0E0EFC0E012003B
:20B00000AD98EFF8D0E0FFD0E0FED0E0FDD0E0FCD0F0E8604DB461004007B47B005002C25A
:20B02000E524D0503DFA24F6500724F95034240AFAEAB5F000502BCFA9F0A42FFF92D5E9E2
:20B04000C5F0CEA4A2D53EFE92D5E9C5F0CDA4A2D53DFD92D5E9C5F0CCA4A2D53CFCC22EDB
:20B06000808DE8C0E0202D30202E090529302B04120089321200AD4712008A920527202964
:20B080000C202A0FEE8FF0120087F9800B120089AA8005EF1200869FD0E01200AD740200EC
:20B0A000ADFA202D131200AD4712008A920527E52A852BF0120087F980E412008B43AEDC1A
:20B0C00053AF6258AE3E4CAE3A42AE1448AF664FAF6A44AE6F43AF5E49AF6A55AF0246AFBD
:20B0E0000245AF0247AE422AB0A24E0000AE4653797374656D20626F6F747570004C6F6703
:20B10000696E20696E76616C69642070617373776F72642066726F6D2025642E25642E2537
:20B12000642E25640041757468656E7469636174696F6E206661696C00506F72742025642A
:20B140004620666962657220696E73657274656400506F7274202564462066696265722027
:20B1600072656D6F76656400506F727420256446206669626572206C696E6B2075700050FE
:20B180006F727420256446206669626572206C696E6B20646F776E00506F72742025644609
:20B1A0002066696265722072656365697665206572726F7200506F72742025644620666997
:20B1C000626572207472616E736D6974206572726F7200506F727420256420636F707065D5
:20B1E000722072656365697665206572726F7200506F727420256420636F70706572207405
:20B2000072616E736D6974206572726F7200506F727420256420636F70706572206C696E8C
:20B220006B20757000506F727420256420636F70706572206C696E6B20646F776E00504F62
:20B240004520706F776572206661696C00506F727420256420706F776572206F6E00506F49
:20B26000727420256420506F776572206F666600506F7274202564206F76657263757272D1
:20B28000656E7400506F72742025642073686F72746369726375697400506F776572206940
:20B2A000732061626F766520746865207468726573686F6C6400506F776572206973206215
:20B2C000656C6F7720746865207468726573686F6C640032342D506F72742031302F313020
:20B2E0003020506F45202B20322D506F7274204769676162697420536D617274205377693A
:20B300007463680028256429004745542000696E6465782E68746D00706F73745F75726C0D
:20B320003D002E006367695F6C6F676F757400636F6E6669672E62696E006367695F626144
:20B340006B5F64617461006367695F006367695F6C6F67696E004C6F67696E004F6E6C79B1
:20B36000206F6E6520757365722063616E206C6F67696E006367695F646576696365007788
:20B38000726F6E672070617373776F7264006C6F67696E2074696D656F7574006367695F92
:20B3A000706F7274006367695F64656C766C616E006367695F766C616E006367695F747295
:20B3C000756E6B006367695F6D6972726F72006367695F737973006367695F7061737300B8
:20B3E0006367695F74726170006367695F7365747674797065006367695F70766964006346
:20B4000067695F736574766964006367695F766964006367695F6164647669640063676968
:20B420005F64656C766964006367695F7265736574006367695F736574706F65006367692B
:20B440005F706F65006367695F73706F65737973006367695F636C727374617400636769DF
:20B460005F73746174697374006367695F616464766C616E006367695F736574766C616E66
:20B48000006367695F7365747669643D2564006367695F736E6D705F636D757479616464BB
:20B4A000006367695F736E6D705F636D757479736574006367695F736E6D705F636D7574F7
:20B4C0007964656C006367695F736E6D705F636D757479006367695F736E6D70006367695A
:20B4E0005F736E6D705F74726170616464006367695F736E6D705F747261707365740063DB
:20B5000067695F736E6D705F7472617064656C006367695F736E6D705F74726170009000FD
:20B520007004E0F54090007005E0F541854082854183E020E7077E007F00C2D72289428ADC
:20B54000435407F5451200B719E02402F544500205451200B5C0053AE53A7002053BE5409A
:20B560002544F540E541354530E604C2E6242FF5411200B5E090007004E540F0900070057D
:20B58000E541F0AE45AF44D2D72290007010E020E61EA3EDF0A3E9F0A3EAF0EC5407D2E658
:20B5A00090007010F00538E53870020539D2D7227C007D00C2D72290007010E0A2E6B322B5
:20B5C00075F001800375F0041200B5E078407F06900070921200B70190007090E5F0F02262
:20B5E00090007090E0540770F7221200B64D90007008742FF0900070107508101200B638AA
:20B60000E490007004F090007006F0742F90007005F090007007F0751D10751C10751E00F7
:20B62000751F2F75832F758200E4F0753800753900753A00753B0022E4A808F0A3D8FC225C
:20B640001200B6F71200B5EA1200B68B229000B68175080A797078601200B7087518C07563
:20B6600019A8751A00751B647510C07511A87512007513017514FF7515FF7516FF751700DC
:20B6800022000B78667788C0A800649000706AE0440CF0229000706AE054F3F02290007085
:20B6A0006AE04401F0229000706AE054FEF0229000706AE04402F0229000706AE054FDF00E
:20B6C000229000706AE04440F0229000706AE054BFF02290007000E04410F02290007000B3
:20B6E000E054EFF02290007000E04420F02290007000E05420F0229000700AF0000000005F
:20B7000022E6F008A3DFFA2289A0E493A3F208B800030989A0D508F222A3E58330E60375D7
:20B72000832F22C230C231C232C233F9E4F555F556FCFDFEFFE9102FEA20320CB42D04D2D8
:20B7400032D322B42B02D32224D0504A94095044240A303315F88556F0740AA42872E740E1
:20B7600054C5F0705085F056D322D231C0E0E4FBFA7920784112008128ECF8EDF9EEFAEF16
:20B78000FBD0E0FCE412008353120080303030B11555D322240A203321B4FE0720301BD26C
:20B7A00030D32224EB600424E0700FA2329230D233C232D322C3020083BDE430330BE55658
:20B7C000303202F404A23092323031E9255520D2E4A2E792335002F404B4260050D7CCC0B8
:20B7E000E0EDC0E0EEC0E0EFC0E0EC1200855DD0E0FFD0E0FED0E0FDD0E0FC2033061200BE
:20B80000812880041200823A3032041200851CC32275C7AA75C755759D0275C7AA75C7552D
:20B8200075C600787FE4F6D8FD755704755800758158D20D0200B86202017254E493A3F866
:20B840005407240CC8C333C4540F4420C8834004F456800146F6DFE4800C010204081020F0
:20B8600040809000A89FE47E019360CCA3FF543F30E509541FFEE493A360010ECF54E0B40B
:20B88000E02AE493FBA3E493FAA3E493F9A3E493C083C082C0931200869FD093D082D083D4
:20B8A000A309E970010ADFE6DEE480BA54C025E0602B4088E493A3FAE493A3F8E493A3C843
:20B8C000C582C8CAC583CA759308F0759300A3C8C582C8CAC583CADFE3DEE18089E493A37B
:20B8E000F8E493A34003F68001F208DFF40200B86668656C6C6F3F3F3F00686968692323D6
:20B9000023006D616320777269746500676F206C6F6164657200636C6F7365746D006D6156
:20B92000632072656164002573006D6163006D6F64656C2072656164006D6F64656C3A0007
:20B94000667776657220726561640066777665723A00726263686B004661696C004F6B005D
:20B9600044656661756C740061646D696E004D444C3A5553523939373632342D56312E3091
:20B98000302E303220202020202020202020202020202020202000000000000000000000A7
:20B9A000000000000000000000000000696E6465782E68746D006C6566742E68746D007462
:20B9C0006F702E68746D0062756C6C65742E67696600666F726D2E637373006C6F676F2E1B
:20B9E000676966006D6F64656C2E676966000A0A776562207365727665722072756E6E6947
:20BA00006E672E2E2E205B25645D0A00496E69742066696E69736865642E0A000A706F65D8
:20BA20005F696E69745F72657472790010350D12008018BF0D027F0A02008FD590083CF9D8
:20BA4000E0FF22E4FFFE1200864E600C0FEF70010E09E970F10A80EE2290083CF9EFF0D2CA
:20BA600035227400EF6402600301BC1590081AF0F0A3F090081AEDE0FBA3E0FAA3E0241599
:20BA8000F9E43AFA1200864EFFB4073090081AEDA3E0FAA3E02416F9E43AFA7401120086CE
:20BAA00083D39405500301CBCA90081AEDA3E0FAA3E02415F9E43AFAE401CBC6EFB4052285
:20BAC00090081AEDE0FBA3E0FAA3E02416F9E43AFA740112008683D39405500301CBCA01BB
:20BAE000BC0E90081AEDE0FBA3E0FAA3E02415F9E43AFA1200864EFF700301CBCA20E403C3
:20BB000001BBBA90081AEDA3E0FAA3E02416F9E43AFA74FF12008683600301CBCA12028AA0
:20BB20009490081AEDE0FBA3E0FAA3E02417F9E43AFA740112008664B4052090081AEDE0E2
:20BB4000FBA3E0FAA3E02415F9E43AFAE41200869F900819E37480F001C74E90081AEDE078
:20BB6000FBA3E0FAA3E02415F9E43AFA1200864E540F14700301C2AE24FE60301470030105
:20BB8000C6BF24FE700301C6BF24FE700301C6BF2406600301CBCA9008177EE0FBA3E0FA42
:20BBA000A3E0240DF9E43AFAE401C2C1900819E37404F01202D3B601C86190081AEDE0FB1B
:20BBC000A3E0FAA3E02415F9E43AFA1200864E540F6403600301CBCA90081AEDA3E0FAA3B3
:20BBE000E02416F9E43AFA74FF12008683600301CBCA90081AEDA3E0FAA3E02417F9E43AA2
:20BC0000FA7401120086646405600301CBCA12028A9401BB3B90082D97E0FBA3E0FAA3E0F7
:20BC2000F990081AF0E0FEA3E0FFE92FF9EA3EFAE41200869F90081AED7409F0A37419F08F
:20BC4000A374EEF090082D97E0FBA3E0FAA3E0F990081778EBF0A3EAF0A3E9F0240EF9E4B5
:20BC60003AFA90081784EBF0A3EAF0A3E9F090081778E0FBA3E0FAA3E0240CF9E43AFA1234
:20BC800000877FFFAEF0BE0807BF060402023C8690081778E0FBA3E0FAA3E0240CF9E43A5C
:20BCA000FA1200877F7004E5F06408600301C41E90081784E0FBA3E0FAA3E02402F9E43A2C
:20BCC000FA1200877FFFAEF090081AF0EEF0A3EFF0D394DCEE9405400301C41E9008178490
:20BCE000E0FBA3E0FAA3E0F91200864E6445600301C41EE92406F9E43AFA1200877FE5F08A
:20BD0000543F600301C41E1202E30F90081784E0FBA3E0FAA3E02410F9E43AFA120089E274
:20BD2000C312008956602590081784E0FBA3E0FAA3E02410F9E43AFA1200898D74FFFBFAE7
:20BD4000F9F8C312008956600301C41E120253AEEFF47002EEF4600301C41E90081784E053
:20BD6000FBA3E0FAA3E0240CF9E43AFA1200898D90081778E0FBA3E0FAA3E02406F9E43A1C
:20BD8000FA120233F390081784E0FBA3E0FAA3E02409F9E43AFA1200864EB40149120086A7
:20BDA0004EFF90081AEDE0FBA3E0FAA3E02414F9E43AFAEF1200869F90081784E0FBA3E0BC
:20BDC000FAA3E0240CF9E43AFA1200898D90081AEDE0FBA3E0FAA3E02404F9E43AFA1200B8
:20BDE00089AA0202C13890081784E0FBA3E0FAA3E02409F9E43AFA1200864E641160030108
:20BE0000BEEE90081784A3E0FAA3E02414F9E43AFA90081781EBF0A3EAF0A3E9F090082D31
:20BE200097E0FBA3E0FAA3E0F91202BAAF90081784E0FBA3E0FAA3E02409F9E43AFA1200BC
:20BE4000864EFF90081AEDE0FBA3E0FAA3E02414F9E43AFAEF1200869F90081781E0FBA378
:20BE6000E0FAA3E02402F9E43AFA1200877FFF90081AEDE0FBA3E0FAA3E0F9E5F08FF0123E
:20BE80000087F990081781E0FBA3E0FAA3E0F91200877FFF90081AEDE0FBA3E0FAA3E02469
:20BEA00002F9E43AFAE5F08FF0120087F990081784E0FBA3E0FAA3E0240CF9E43AFA120028
:20BEC000898D90081AEDE0FBA3E0FAA3E02404F9E43AFA120089AA90081AEDE0FBA3E0FA5D
:20BEE000A3E0F91200877FFFAEF00202CD3C90081784E0FBA3E0FAA3E02409F9E43AFA12A6
:20BF000000864E6406600301C41E90081784E0FBA3E0FAA3E02414F9E43AFA9008177EEB2E
:20BF2000F0A3EAF0A3E9F01202E5CC9008177EE0FBA3E0FAA3E02402F9E43AFA1200877FFC
:20BF40006F7003EE65F0600301C41E90083B65E4F0A304F090083B65E0FEA3E0FFC39405DF
:20BF6000EE9400400301C0327C007D33120086B374EE2FF974193EFA7B0990081AEDEBF045
:20BF8000A3EAF0A3E9F02415F9E43AFA1200864E700301C01F9008177EE0FBA3E0FAA3E01D
:20BFA0002402F9E43AFA1200877FFFAEF090081AEDE0FBA3E0FAA3E0F91200877F6F700328
:20BFC000EE65F0705AE92402F9E43AFA1200877FFFAEF09008177EE0FBA3E0FAA3E0F9126C
:20BFE00000877FB50739E5F0B5063490081AEDE0FBA3E0FAA3E02404F9E43AFA1200898DA7
:20C0000090081784E0FBA3E0FAA3E0240CF9E43AFA120089E2C312008956700301C3C49015
:20C02000083B66E004F0700790083B65E004F001BF549008177EE0FBA3E0FAA3E0240DF9BA
:20C04000E43AFA1200864E6402600301C41E90083B65E4F0A304F090083B65E0FEA3E0FFFB
:20C06000C39405EE9400502D90081A0375F033EF12008A86EE75F033A42583F583759308AD
:20C08000E0605E90083B66E004F070CB90083B65E004F080C290083B65E4F0A304F0900831
:20C0A0003B65E0FEA3E0FFC39405EE9400502F90081A0375F033EF12008A86EE75F033A49B
:20C0C0002583F583759308E06407601590083B66E004F070C990083B65E004F080C001C419
:20C0E0001E90083B65E0FEA3E0FF7C007D33120086B374EE2FF974193EFA90081AED7409A8
:20C10000F0A3EAF0A3E9F090081784E0FBA3E0FAA3E02409F9E43AFA1200864EFF90081A53
:20C12000EDE0FBA3E0FAA3E02414F9E43AFAEF1200869F90081AEDE0FBA3E0FAA3E0241614
:20C14000F9E43AFA74021200869F90081AEDE0FBA3E0FAA3E02417F9E43AFAE41200869F40
:20C160009008177EE0FBA3E0FAA3E02402F9E43AFA1200877FFF90081AEDE0FBA3E0FAA3CF
:20C18000E0F9E5F08FF0120087F99008177EE0FBA3E0FAA3E0F91200877FFF90081AEDE049
:20C1A000FBA3E0FAA3E02402F9E43AFAE5F08FF0120087F990081784E0FBA3E0FAA3E02435
:20C1C0000CF9E43AFA1200898D90081AEDE0FBA3E0FAA3E02404F9E43AFA120089AA90088A
:20C1E0001AEDE0FBA3E0FAA3E02415F9E43AFA74111200869F900819EAE0FCA3E0FDA3E0DD
:20C20000FEA3E0FF90081AEDE0FBA3E0FAA3E0240CF9E43AFA120089AAEF2401FFE43EFE6B
:20C22000E43DFDE43CFC90081AEDE0FBA3E0FAA3E02410F9E43AFA120089AA9008177EE0B3
:20C24000FBA3E0FAA3E02404F9E43AFA1200898DEF2401FFE43EFEE43DFDE43CFC90081A63
:20C26000EDE0FBA3E0FAA3E02408F9E43AFA120089AA90081AEDE0FBA3E0FAA3E0242AF9B3
:20C28000E43AFAC003C002C00190081AEDA3E0FAA3E02428F9E43AFA90083A90EBF0A3EA7A
:20C2A000F0A3E9F0D001D002D0031202C7B59008177EE0FBA3E0FAA3E0240DF9E43AFA744E
:20C2C000101200869F9008177EE0FBA3E0FAA3E0240DF9E43AFA1200864E44021200869F6A
:20C2E0009008177EE0FBA3E0FAA3E02414F9E43AFA90083B67EBF0A3EAF0A3E9F074021257
:20C3000000869F90083B67E0FBA3E0FAA3E02401F9E43AFA74041200869F90083B67E0FBE9
:20C32000A3E0FAA3E02402F9E43AFA74051200869F90083B67E0FBA3E0FAA3E02403F9E4FD
:20C340003AFA74781200869F90083B67E0FBA3E0FAA3E02404F9E43AFA74011200869F90FC
:20C36000083B67E0FBA3E0FAA3E02405F9E43AFA74011200869F90083B67E0FBA3E0FAA31D
:20C38000E02406F9E43AFA74041200869F90083B67E0FBA3E0FAA3E02407F9E43AFA74020C
:20C3A0001200869F90081AF0E4F0A37430F09008177EE0FBA3E0FAA3E0240CF9E43AFA74DC
:20C3C0007001CAE5E4900819E3F09008177EE0FBA3E0FAA3E0240DF9E43AFA1200864E3075
:20C3E000E22490081AEDE0FBA3E0FAA3E02415F9E43AFAE41200869F900819E37420F0122E
:20C4000002D3B601C9A79008177EE0FBA3E0FAA3E0240DF9E43AFA1200864E20E40301C91F
:20C42000A79008177EE0FBA3E0FAA3E0240CF9E43AFA1200864EC4540F25E025E0FF7E0078
:20C4400090083B65EEF0A3EFF02414FFEE33FEC390081AF1E09FFF90081AF0E09EFEF0A359
:20C46000EFF0D39400EE9400403490081AEDE0FBA3E0FAA3E02408F9E43AFA1200898D9011
:20C4800008177EE0FBA3E0FAA3E02404F9E43AFA120089E2C312008956600301CAB1900843
:20C4A0001AEDE0FBA3E0FAA3E02410F9E43AFA1200898D9008177EE0FBA3E0FAA3E02408F9
:20C4C000F9E43AFA120089E2C312008956706690081AEDE0FBA3E0FAA3E02410F9E43AFA85
:20C4E0001200898D90081AEDA3E0FAA3E0240CF9E43AFA120089AA90081AEDE0FBA3E0FAF8
:20C50000A3E02415F9E43AFA1200864EFF30E425900819E37401F0EF54EF1200869F900836
:20C520001AEDE0FBA3E0FAA3E02416F9E43AFA74021200869F90081AEDE0FBA3E0FAA3E0A7
:20C540002415F9E43AFA1200864E540F14B40800400301CAAD9000C56475F004A4C583258A
:20C56000F0C583730200C5840200C5A00200C6230200C8C20200C9AA0200CA780200CAB1B1
:20C580000200C8A7900819E3E030E01174031200869F900819E37440F01202D3B601C9A7A1
:20C5A000900819E3E030E0789008177EE0FBA3E0FAA3E0240DF9E43AFA1200864E64127069
:20C5C0005F90081AEDE0FBA3E0FAA3E02415F9E43AFA74031200869F9008177EE0FBA3E0FF
:20C5E000FAA3E02404F9E43AFA1200898D90081AEDE0FBA3E0FAA3E02408F9E43AFA120094
:20C6000089AA1200898DEF2401FFE43EFEE43DFDE43CFC120089AA74421202D3A901C72FD0
:20C6200001C9A79008177EE0FBA3E0FAA3E0240DF9E43AFA1200864E20E00301C6C2900835
:20C640001AF1E02401FF90081AF0E03400FEE4FCFD90081AEDE0FBA3E0FAA3E02408F9E4B7
:20C660003AFA120089AA74101202D3A990081AEDE0FBA3E0FAA3E02410F9E43AFA120089D3
:20C680008DEF2401FFE43EFEE43DFDE43CFC120089AA90081AEDE0FBA3E0FAA3E02415F9AF
:20C6A000E43AFA74181200869F90081AEDE0FBA3E0FAA3E02417F9E43AFAE41200869F01BD
:20C6C000C7BBD390081AF1E0940090081AF0E094004045900819E3E04402F090081AEDE02A
:20C6E000FBA3E0FAA3E02408F9E43AFAC003C002C001120089E290081AF0E0FEA3E0FFE459
:20C70000FCFDEB2FFFEA3EFEED39FDEC38FCD001D002D003120089AA900819E3E0540370A8
:20C720000301C8A41202D3B6EF4E700301CAB1900819E3E0FF30E52C90081AEDE0FBA3E00F
:20C74000FAA3E02415F9E43AFAE41200869F9008177EE0FBA3E0FAA3E0240DF9E43AFA7439
:20C760001401CAC4EF30E46990081AEDE0FBA3E0FAA3E02410F9E43AFA1200898DEF2401AF
:20C78000FFE43EFEE43DFDE43CFC120089AA90081AEDE0FBA3E0FAA3E02415F9E43AFA74C3
:20C7A000141200869F90081AEDE0FBA3E0FAA3E02417F9E43AFAE41200869F9008177EE040
:20C7C000FBA3E0FAA3E0240DF9E43AFA741101CAC4D390081AF1E0940090081AF0E0940008
:20C7E000407790081AEDE0FBA3E0FAA3E02415F9E43AFA1200864E20E45F1200864E44103B
:20C800001200869F90081AEDE0FBA3E0FAA3E02417F9E43AFAE41200869F90081AEDE0FB86
:20C82000A3E0FAA3E02410F9E43AFAC003C002C001120089E290081AF0E0FEA3E0FFE4FC0E
:20C84000FDEB2FFFEA3EFEED39FDEC38FCD001D002D003120089AA8008E490081AF0F0A3FD
:20C86000F0D390081AF1E0940090081AF0E094005008900819E3E030E12A90081AF1E0241A
:20C8800028F090081AF0E03400F09008177EE0FBA3E0FAA3E0240DF9E43AFA74181200866C
:20C8A0009F01CAD201C9A7900819E3E020E00301CAAD90081AEDE0FBA3E0FAA3E024150128
:20C8C000CAA4D390081AF1E0940090081AF0E09400403D90081AEDE0FBA3E0FAA3E02408C7
:20C8E000F9E43AFAC003C002C001120089E290081AF0E0FEA3E0FFE4FCFDEB2FFFEA3EFE46
:20C90000ED39FDEC38FCD001D002D003120089AA9008177EE0FBA3E0FAA3E0240DF9E43AC9
:20C92000FA1200864E30E049900819E3E090081AED30E027E0FBA3E0FAA3E02415F9E43A49
:20C94000FA74071200869F90081AEDE0FBA3E0FAA3E02416F9E43AFAE4800FE0FBA3E0FA9B
:20C96000A3E02415F9E43AFA74161200869F01CA3D900819E3E030E01A90081AEDE0FBA366
:20C98000E0FAA3E02415F9E43AFA74051200869F01CAADD390081AF1E0940090081AF0E05C
:20C9A0009400400301CAB101CAADD390081AF1E0940090081AF0E09400403D90081AEDE0B0
:20C9C000FBA3E0FAA3E02408F9E43AFAC003C002C001120089E290081AF0E0FEA3E0FFE476
:20C9E000FCFDEB2FFFEA3EFEED39FDEC38FCD001D002D003120089AA9008177EE0FBA3E076
:20CA0000FAA3E0240DF9E43AFA1200864E30E05590081AEDE0FBA3E0FAA3E02415F9E43A42
:20CA2000FA74071200869F90081AEDE0FBA3E0FAA3E02416F9E43AFAE41200869F90081AB8
:20CA4000EDE0FBA3E0FAA3E02408F9E43AFA1200898DEF2401FFE43EFEE43DFDE43CFC122A
:20CA60000089AA804CD390081AF1E0940090081AF0E09400503B8035900819E3E030E02DC6
:20CA800090081AEDE0FBA3E0FAA3E02415F9E43AFA74071200869F90081AEDE0FBA3E0FA29
:20CAA000A3E02416F9E43AFAE41200869F0202E74F9008177EE0FBA3E0FAA3E0240DF9E43D
:20CAC0003AFA74101200869F90081AF0E4F0A37428F09008177EE0FBA3E0FAA3E0240CF991
:20CAE000E43AFA74501200869F90081AEDE0FBA3E0FAA3E02408F9E43AFA1200898D9008AC
:20CB0000177EE0FBA3E0FAA3E02408F9E43AFA120089AA90081AEDE0FBA3E0FAA3E0240C79
:20CB2000F9E43AFA1200898D9008177EE0FBA3E0FAA3E02404F9E43AFA120089AA90081A84
:20CB4000EDE0FBA3E0FAA3E0F91200877FFF9008177EE0FBA3E0FAA3E0F9E5F08FF0120096
:20CB600087F990081AEDE0FBA3E0FAA3E02402F9E43AFA1200877FFF9008177EE0FBA3E0E2
:20CB8000FAA3E02402F9E43AFAE5F08FF0120087F99008177EE0FBA3E0FAA3E0240EF9E4E4
:20CBA0003AFA740575F078120087F97F027E001201690490081AEDE0FBA3E0FAA3E0241626
:20CBC000F9E43AFA74021200869F229008177EE0FBA3E0FAA3E02414F9E43AFA9008177BFA
:20CBE000EBF0A3EAF0A3E9F090081AEDE0FBA3E0FAA3E0242CF9E43AFA90080663EBF0A307
:20CC0000EAF0A3E9F090081AEDA3E0FAA3E0242BF9E43AFA90080403EBF0A3EAF0A3E9F04C
:20CC200090081AEDA3E0FAA3E02418F9E43AFA9008064FEBF0A3EAF0A3E9F090081AEDA305
:20CC4000E0FAA3E0241AF9E43AFA90080400EBF0A3EAF0A3E9F090081AEDA3E0FAA3E024F5
:20CC60001CF9E43AFA90080660EBF0A3EAF0A3E9F090081AEDA3E0FAA3E0241EF9E43AFAC3
:20CC800090080652EBF0A3EAF0A3E9F090081AEDA3E0FAA3E02420F9E43AFA90080655EBFE
:20CCA000F0A3EAF0A3E9F090081AEDA3E0FAA3E02422F9E43AFA9008040AEBF0A3EAF0A3F4
:20CCC000E9F090081AEDA3E0FAA3E02424F9E43AFA90080659EBF0A3EAF0A3E9F090081A06
:20CCE000EDA3E0FAA3E02426F9E43AFA9008040DEBF0A3EAF0A3E9F0900819E3E0FD30E6E8
:20CD00006790080663E0FBA3E0FAA3E0F9E41200869F90080663E0FBA3E0FAA3E02402F9C1
:20CD2000E43AFAE4F5F0120087F99008064FE0FBA3E0FAA3E0F9E475F001120087F990084B
:20CD40000660E0FBA3E0FAA3E0F9E475F001120087F990080655E0FBA3E0FAA3E0F9E4F51D
:20CD6000F0120087F901DCA5ED30E70301DCA5900819E3E020E10301D9FA90080663E0FBFE
:20CD8000A3E0FAA3E0F91200864E600301D9FA90083A127481F0A374B3F0A37409F0A3E463
:20CDA000F0A37404F09008177BE0FBA3E0FAA3E0F91202B7AEEF600301CE429008316CF079
:20CDC0009008177BE0FBA3E0FAA3E02405F9E43AFA9008316CE0FF7C0029F9EC3AFAA3EBB4
:20CDE000F0A3EAF0A3E9F01200864EFE64206004EEB43F1174702FF582E43431F583759339
:20CE000008E4F080199008316CE0FF04F074702FF582E43431F583759308EEF080A27B09B6
:20CE20007A3179701200BA43EF4E600301CF0478707C317D097B817AB3790E12008D55011B
:20CE4000CF04900837CE7481F0A374B3F0A37418F09008177BE0FBA3E0FAA3E0F912029002
:20CE60008C9008316DEBF0A3EAF0A3E9F09008316DE0FBA3E0FAA3E04A4B703F90080658D1
:20CE8000E06403700301D28190081AF0E0FEA3E0FF7D009008177BE0FBA3E0FAA3E0F912F5
:20CEA000008F13E490081AF0F0A3F09008177BE0FBA3E0FAA3E0F902018B09900834C3742F
:20CEC00081F0A374B3F0A37418F0A37481F0A374B3F0A37422F0A37409F0A37431F0A3743E
:20CEE00070F09008316DE0FBA3E0FAA3E0F91202596590080663E0FBA3E0FAA3E0F97401AC
:20CF00001200869F90083A127481F0A374B3F0A37424F0A3E4F0A3740AF07B097A3179708C
:20CF20001202B7AEEF704990081AEDE0FBA3E0FAA3E02404F9E43AFA1200898D9008065CFB
:20CF4000E0F8A3E0F9A3E0FAA3E0FBC312008956700301CFE6E4FFFEFDFC9008065CE0F8F9
:20CF6000A3A3A3E0C312008956600301D0E0807690083A127481F0A374B3F0A3742FF0A3CE
:20CF8000E4F0A3740AF07B097A3179701202B7AEEF701078707C317D097B817AB3793A12A3
:20CFA000008D5590083A127481F0A374B3F0A37447F0A3E4F0A37404F07B097A3179701212
:20CFC00002B7AEEF700301D09F900839637409F0A37431F0A37467F07B097A3179701202A5
:20CFE0008B77EF4E702378707C317D097B817AB3794C12008D55900806587401F0E4FFFE26
:20D00000FDFC9008065C01D22F90080663E0FBA3E0FAA3E0F974021200869F90083167E089
:20D02000FBA3E0FAA3E0F9C003C002C00190080663E0FBA3E0FAA3E02404F9E43AFA12008F
:20D040008AEF9008316AE0FEA3E0FF90080663E0FBA3E0FAA3E02402F9E43AFAEE8FF01232
:20D060000087F91202E2EFC004C005C006C0071202E61CE4FCFD7B587A02F9F81200881553
:20D08000D003D002D001D000EB2FFFEA3EFEE93DFDE83CFC9008040612008A6901DBB790FE
:20D0A000081AEDE0FBA3E0FAA3E02404F9E43AFA1200898D9008065CE0F8A3E0F9A3E0FA5A
:20D0C000A3E0FBC312008956603EE4FFFEFDFC9008065CE0F8A3A3A3E0C3120089566028CF
:20D0E0009008395A7481F0A374B3F0A3745CF0A37481F0A374B3F0A3744CF07B817AB379CC
:20D10000561202A5C001DCA590080663E0FBA3E0FAA3E0F91200864E6401600301D23690A2
:20D12000083A127481F0A374B3F0A37474F0A3E4F0A3740AF07B097A3179701202B7AEEF79
:20D14000600301D2369008177BE0FBA3E0FAA3E0F91202ABBEEF4E707D1202E33FE4FBFAAF
:20D16000F9F8C31200895660451202E34FEF5402FFE4FEFDFC7B02FAF9F8C3120089567074
:20D180002D90081AEDE0FBA3E0FAA3E02404F9E43AFA1200898D90083A0112008A69E4903B
:20D1A000083A05F0A3F07FEA7E03120278609008395A7481F0A374B3F0A3747FF0A37481E7
:20D1C000F0A374B3F0A3744CF07B817AB379561202A5C001DCA590081AEDE0FBA3E0FAA3C5
:20D1E000E02404F9E43AFA1200898D9008065C12008A69900806587402F01202E2EFC004EA
:20D20000C005C006C0071202E61CE4FCFD7B587A02F9F812008815D003D002D001D000EBA9
:20D220002FFFEA3EFEE93DFDE83CFC9008040612008A6901D6D690083A127481F0A374B370
:20D24000F0A3744CF0A3E4F0A37409F07B097A3179701202B7AEEF70099008065804F00120
:20D26000D6D690080658E0B4010F78707C317D097B817AB3794C01D69590080658E0B40366
:20D280003C9008395A7481F0A374B3F0A3748EF0A37481F0A374B3F0A3744CF07B817AB335
:20D2A00079561202A5C0900806587401F0E4FFFEFDFC9008065C12008A6901DCA5900806D2
:20D2C00063E0FBA3E0FAA3E0F91200864E6401600301D6D690083A127481F0A374B3F0A396
:20D2E000749CF0A3E4F0A37408F07B097A3179701202B7AEEF70139008177BE0FBA3E0FA23
:20D30000A3E0F91201F6B901D6D690083A127481F0A374B3F0A374A5F0A3E4F0A3740BF06A
:20D320007B097A3179701202B7AEEF70269008177BE0FBA3E0FAA3E0F912021FA8EF4E7051
:20D340000301D6D278707C317D097B817AB379B101D69590083A127481F0A374B3F0A374AD
:20D36000B1F0A3E4F0A37408F07B097A3179701202B7AEEF701A9008177BE0FBA3E0FAA357
:20D38000E0F91201E1CDEF4E600301D6D601D6D290083A127481F0A374B3F0A374BAF0A316
:20D3A000E4F0A37409F07B097A3179701202B7AEEF701A9008177BE0FBA3E0FAA3E0F9126F
:20D3C00001E490EF4E600301D6D601D6D290083A127481F0A374B3F0A374C4F0A3E4F0A37A
:20D3E000740AF07B097A3179701202B7AEEF701A9008177BE0FBA3E0FAA3E0F91201EF1B9A
:20D40000EF4E600301D6D601D6D290083A127481F0A374B3F0A374CFF0A3E4F0A37407F038
:20D420007B097A3179701202B7AEEF701A9008177BE0FBA3E0FAA3E0F912013E31EF4E60C5
:20D440000301D6D601D6D290083A127481F0A374B3F0A374D7F0A3E4F0A37408F07B097A8E
:20D460003179701202B7AEEF701A9008177BE0FBA3E0FAA3E0F912023AD6EF4E600301D607
:20D48000D601D6D290083A127481F0A374B3F0A374E0F0A3E4F0A37408F07B097A31797005
:20D4A0001202B7AEEF701A9008177BE0FBA3E0FAA3E0F912018EE3EF4E600301D6D601D6D4
:20D4C000D290083A127481F0A374B3F0A374E9F0A3E4F0A3740CF07B097A3179701202B79A
:20D4E000AEEF70269008177BE0FBA3E0FAA3E0F912026F89EF4E700301D6D278707C317D84
:20D50000097B817AB379B101D69590083A127481F0A374B3F0A374F6F0A3E4F0A37408F03D
:20D520007B097A3179701202B7AEEF701A9008177BE0FBA3E0FAA3E0F912022758EF4E60B3
:20D540000301D6D601D6D290083A127481F0A374B3F0A374FFF0A3E4F0A3740AF07B097A63
:20D560003179701202B7AEEF70269008177BE0FBA3E0FAA3E0F91201CDB2EF4E700301D67C
:20D58000D278707C317D097B817AB4790A01D69590083A127481F0A374B4F0A37412F0A345
:20D5A000E4F0A3740AF07B097A3179701202B7AEEF70269008177BE0FBA3E0FAA3E0F91260
:20D5C00001C7B8EF4E700301D6D278707C317D097B817AB4790A01D69590083A127481F075
:20D5E000A374B4F0A3741DF0A3E4F0A3740AF07B097A3179701202B7AEEF70259008177B85
:20D60000E0FBA3E0FAA3E0F912022CD2EF4E700301D6D278707C317D097B817AB4790A8083
:20D620007490083A127481F0A374B4F0A37428F0A3E4F0A37409F07B097A3179701202B759
:20D64000AEEF701290082D52F0A304F0900819E37410F001DCA590083A127481F0A374B4EF
:20D66000F0A37432F0A3E4F0A3740AF07B097A3179701202B7AEEF70229008177BE0FBA33F
:20D68000E0FAA3E0F91202664878707C317D097B817AB4793D12008D55803B90083A127470
:20D6A00081F0A374B4F0A37445F0A3E4F0A3740BF07B097A3179701202B7AEEF70189008C9
:20D6C000177BE0FBA3E0FAA3E0F912029C74EF4E7004FE7F0122E49008316CF090083A1282
:20D6E0007481F0A374B4F0A37451F0A3E4F0A3740BF07B097A3179701202B7AEEF70141293
:20D70000029E8678707C317D097B817AB4795D12008D5590083A127481F0A374B4F0A37439
:20D7200069F0A3E4F0A3740BF07B097A3179701202B7AEEF701A90083CD0F0A304F07870EA
:20D740007C317D097B817AB4797512008D558008E490083CD0F0A3F0E490083CCAF0A3F0F2
:20D7600090083A127481F0A374B3F0A374FFF0A3E4F0A3740AF07B097A3179701202B7AE07
:20D78000EF7045900831127481F0A374B4F0A37481F0A37409F0A3743CF0A374CAF07B093A
:20D7A0007A3179701200ADE378707C317D097B817AB4790A12008D5590083CCBE024FFF0E5
:20D7C00090083CCAE034FFF090083A127481F0A374B4F0A3748FF0A3E4F0A37411F07B097B
:20D7E0007A3179701202B7AEEF701790083BE5F0A304F078707C317D097B817AB479A10107
:20D80000D94990083A127481F0A374B4F0A374A1F0A3E4F0A37411F07B097A3179701202FF
:20D82000B7AEEF700301D90990083A127481F0A374B4F0A374B3F0A3E4F0A37411F07B09ED
:20D840007A3179701202B7AEEF700301D90990083A127481F0A374B4F0A374C5F0A3E4F0AF
:20D86000A3740EF07B097A3179701202B7AEEF701690083BE3F0A3F078707C317D097B813D
:20D880007AB479D401D94990083A127481F0A374B4F0A374DDF0A3E4F0A37410F07B097AF6
:20D8A0003179701202B7AEEF701790083BE5F0A304F078707C317D097B817AB479EE01D99A
:20D8C0004990083A127481F0A374B4F0A374EEF0A3E4F0A37410F07B097A3179701202B715
:20D8E000AEEF7002802390083A127481F0A374B4F0A374FFF0A3E4F0A37410F07B097A312F
:20D9000079701202B7AEEF700990083BE5F0A3F0803B90083A127481F0A374B5F0A374109B
:20D92000F0A3E4F0A3740DF07B097A3179701202B7AEEF701890083BE3F0A304F078707CC3
:20D94000317D097B817AB479D412008D559008316CE0FD75F017A42410F582E5F03404F5C6
:20D9600083759308E0FBA3E0FAA3E04A4B700A900819E37410F001DCA5ED75F017A424135C
:20D98000F9740435F0FA7B091200BA4390083A15EEF0A3EFF09008316CE075F017A42413B1
:20D9A000F9740435F0FA90083A127409F0A3EAF0A3E9F07B097A3179701202B7AEEF70306D
:20D9C00090080663E0FBA3E0FAA3E0F974031200869F9008316CE0FF90080663E0FBA3E051
:20D9E000FAA3E02401F9E43AFAEF1200869F800A9008316CE004F001D94D90080663E0FBB8
:20DA0000A3E0FAA3E0F91200864E6403600301DBB790081AF0F0A3F0900819E3E064046069
:20DA20000301DAAB90080400E0FBA3E0FAA3E0F91200877FFF9008064FE0FBA3E0FAA3E00E
:20DA4000F9E5F08FF0120087F990080652E0FBA3E0FAA3E0F91200877FFF90080660E0FB33
:20DA6000A3E0FAA3E0F9E5F08FF0120087F99008040AE0FBA3E0FAA3E0F91200877FFF90A6
:20DA8000080655E0FBA3E0FAA3E0F9E5F08FF0120087F99008040DE0FBA3E0FAA3E0F912DA
:20DAA00000877FFF9008065901DB2F9008064FE0FBA3E0FAA3E0F91200877FFF90080400EB
:20DAC000E0FBA3E0FAA3E0F9E5F08FF0120087F990080660E0FBA3E0FAA3E0F91200877FA2
:20DAE000FF90080652E0FBA3E0FAA3E0F9E5F08FF0120087F990080655E0FBA3E0FAA3E0AF
:20DB0000F91200877FFF9008040AE0FBA3E0FAA3E0F9E5F08FF0120087F990080659E0FBC3
:20DB2000A3E0FAA3E0F91200877FFF9008040DE0FBA3E0FAA3E0F9E5F08FF0120087F990E2
:20DB4000080663E0FBA3E0FAA3E02401F9E43AFA1200864E75F017A42410F582E5F0340485
:20DB6000F583759308E0FBA3E0FAA3E0F912008B9AEF6007900819E37410F01202E2EFC00F
:20DB800004C005C006C0071202E61CE4FCFD7B587A02F9F812008815D003D002D001D00007
:20DBA000EB2FFFEA3EFEE93DFDE83CFC9008040612008A6901DCA5900819E3E030E07A902C
:20DBC000080663E0FBA3E0FAA3E02402F9E43AFA1200877FC39478E5F09405402A74FA7520
:20DBE000F088120087CD90080663E0FBA3E0FAA3E02404F9E43AFA09E970010A740575F0E7
:20DC000078120087CD803290080663E0FBA3E0FAA3E02402F9E43AFAE4F5F0120087F99076
:20DC2000080663E0FBA3E0FAA3E0F91200864EB40207900819E37410F090080663E0FBA375
:20DC4000E0FAA3E02402F9E43AFA1200877FFFAEF0D39478EE940590081AF040097405F0C1
:20DC6000A37478F08005EEF0A3EFF090081AF0E0FEA3E0FF90080663E0FBA3E0FAA3E0243E
:20DC800004F9E43AFA12008AD2C003C0029008177BE0FBA3E0FAA3E0F8AC02AD03D002D07F
:20DCA00003120085D07E007F01229008064FE0FBA3E0FAA3E0F91200877FFFAEF0E5F0602F
:20DCC0000301EB1EEF12008B43DD0001E10D02E17003E19F07E1FA08E43409E4340DE4842E
:20DCE0000EE6F40FEA0B10EA0B14EA0B16EA0B19EA0B1CEA0B1FEAB320EAE1210000EB1E2F
:20DD0000900830567484F0A37433F0A374B8F09008177BE0FBA3E0FAA3E0F91200A41690AA
:20DD2000081AF0EEF0A3EFF0E490082A10F0A3F090082A10E475F00112008753AFF0FE6033
:20DD40000301E0FAEF14B40D00400301E0FA9000DD5D75F004A4C58325F0C583730200DD35
:20DD6000910200DDA70200DDBD0200DDF00200DE000200DE150200DE2A0200DE3F0200DE43
:20DD80005D0200DEF30200DF080200DF280200DF5590082A2A7484F0A37434F0A374F2F023
:20DDA0001202DF2401DF1B90082A2A7484F0A37434F0A374FFF01202DF5E01DF1B90082A2E
:20DDC0002A7484F0A37435F0A37410F0900830567484F0A37435F0A37421F0A3E4F0A374E6
:20DDE00002F0A3E4F0A304F0A3E4F0A30401E06790082A11E004F0700790082A10E004F0F9
:20DE000090082A2A7484F0A37435F0A3742EF01202E30F803D90082A2A7484F0A37435F0EA
:20DE2000A37439F01202E31F802890082A2A7484F0A37435F0A37445F01202E32F8013903F
:20DE4000082A2A7484F0A37435F0A37455F01202E33F90082A8012008A6901DFE990082ADE
:20DE60002A7484F0A37435F0A3745DF07B097A2A792D1202DBFC900830567484F0A37435E5
:20DE8000F0A37469F090082A2DE0FF3395E090083059E4F0A3EFF090082A2EE0FF3395E0BE
:20DEA0009008305BE4F0A3EFF090082A2FE0FF3395E09008305DE4F0A3EFF090082A30E024
:20DEC000FF3395E09008305FE4F0A3EFF090082A31E0FF3395E090083061E4F0A3EFF09095
:20DEE000082A32E0FF3395E090083063E4F0A3EF01E06790082A2A7484F0A37435F0A37437
:20DF000087F01202E6A9801390082A2A7484F0A37435F0A37493F01202E6B0782D7C2A7D38
:20DF20000912008D5501E07290082A2A7484F0A37435F0A374A1F01202E61C90083059EEB4
:20DF4000F0A3EFF0900830567484F0A37435F0A374B901E06790082A2A7484F0A37435F0E5
:20DF6000A374BCF0900837267409F0A3742AF0A37486F0A37409F0A3742AF0A37488F0A34B
:20DF80007409F0A3742AF0A3748AF07B097A2A79841202C69D900830567484F0A37435F074
:20DFA000A374CAF090082A84E0FFA3E090083059CFF0A3EFF090082A86E0FFA3E090083014
:20DFC0005BCFF0A3EFF090082A88E0FFA3E09008305DCFF0A3EFF090082A8AE0FFA3E09055
:20DFE00008305FCFF0A3EF807E900830567484F0A37435F0A374EEF090082A80E0FCA3E063
:20E00000FDA3E0FEA3E0FF781812008967E490083059F0A3EFF090082A80E0FCA3E0FDA3B6
:20E02000E0FEA3E0FF781012008967E49008305BF0A3EFF090082A80E0FCA3E0FDA3E0FE5E
:20E04000A3E0FF780812008967E49008305DF0A3EFF090082A80E0FCA3E0FDA3A3E0FEE49B
:20E060009008305FF0A3CEF07B097A2A792D1200A4167B097A2A792D1200BA43EF4E7010F4
:20E08000782D7C2A7D097B847A3579FA12008D559008177BE0FBA3E0FAA3E0F990081AF0FA
:20E0A000E0FEA3E0FFE92FF9EA3EFAC002C001900830567484F0A37436F0A37401F0900867
:20E0C0002A2AE0F9A3E0FAA3E090083059C9F0A3EAF0A3E9F0A37409F0A3742AF0A3742DBB
:20E0E000F0D001D0021200A41690081AF1E02FF090081AF0E03EF001DD309008064FE0FB99
:20E10000A3E0FAA3E0F9E475F00201EADA9008177BE0FBA3E0FAA3E0F990081AF0E0FEA3D5
:20E12000E0FFE92FF9EA3EFA900830567484F0A37436F0A3741BF01200A41690081AF1E019
:20E140002FF090081AF0E03EF09008064FE0FBA3E0FAA3E0F9E475F003120087F9900806B3
:20E1600060E0FBA3E0FAA3E0F9E475F00101EADAE4FFFE120159FAEF4E7002FF22900806A7
:20E180004FE0FBA3E0FAA3E0F9E475F007120087F990081AF0E07002A3E060037F002212ED
:20E1A00002E625EF4E700301E434900830567484F0A37436F0A3745CF09008177BE0FBA33B
:20E1C000E0FAA3E0F91200A41690081AF0EEF0A3EFF09008064FE0FBA3E0FAA3E0F9E47501
:20E1E000F008120087F990080660E0FBA3E0FAA3E0F9E475F001120087F990080660E0FB0E
:20E20000A3E0FAA3E0F91200877FC39401FFE5F09400FE90082A80F0A3EFF0900838BC747B
:20E2200009F0A3742AF0A37482F07B097A2A791A1202A133EF4E702B9008064FE0FBA3E065
:20E24000FAA3E0F9E475F009120087F9D390081AF1E0940090081AF0E09400500301E9F433
:20E260007F002290082A82E0FBA3E0FAA3E0F91200BA43EF4E700F90082A827484F0A374D7
:20E2800035F0A374FAF09008177BE0FBA3E0FAA3E0F990081AF0E0FEA3E0FFE92FF9EA3E1F
:20E2A000FAC002C001900830567484F0A37437F0A37400F090082A81E02401FE90082A800E
:20E2C000E0340090083059F0A3CEF090082A82E0F9A3E0FAA3E09008305BC9F0A3EAF0A39F
:20E2E000E9F0D001D0021200A41690081AF1E02FF090081AF0E03EF0E490082A16F0A3F045
:20E30000C390082D69E09401FF90082D68E09400FE90082A16E0FCA3E0FDC39FEE6480F899
:20E32000EC648098400301E3CDEDAE047803CEA2E713CE13D8F8241AF582742A3EF58375CE
:20E340009308E0FD7C0090082A17E05407FF74017E00A807088005C333CE33CED8F9FFEE04
:20E360005CFEEF5D4E60539008177BE0FBA3E0FAA3E0F990081AF0E0FEA3E0FFE92FF9EAFB
:20E380003EFA900830567484F0A37437F0A3742DF090082A17E02401FE90082A16E0340005
:20E3A00090083059F0A3CEF01200A41690081AF1E02FF090081AF0E03EF090082A17E00410
:20E3C000F0700790082A16E004F001E3009008177BE0FBA3E0FAA3E0F990081AF0E0FEA325
:20E3E000E0FFE92FF9EA3EFA900830567484F0A37437F0A37433F01200A41690081AF1E03E
:20E400002FF090081AF0E03EF090080660E0FBA3E0FAA3E0F9E475F001120087CDC3900850
:20E420001AF1E094B090081AF0E09404500301E1FA7F0022900830567484F0A37437F0A3DC
:20E440007436F09008177BE0FBA3E0FAA3E0F91200A41690081AF0EEF0A3EFF09008066058
:20E46000E0FBA3E0FAA3E0F9E475F001120087F99008064FE0FBA3E0FAA3E0F9E475F00ED4
:20E48000120087F9E490082A16F0A3F0E490082A7FF090082A17E0FF7B097A2A791A12020F
:20E4A00089B190082A17E0FF1202E38FEF60087B847A38790480067B847A38790C900830DB
:20E4C0005BEBF0A3EAF0A3E9F09008177BE0FBA3E0FAA3E0F990081AF0E0FEA3E0FFE92FF5
:20E4E000F9EA3EFA900830567484F0A37437F0A374C6F090082A17E02401FE90082A16E05C
:20E50000340090083059F0A3CEF01200A41690081AF1E02FF090081AF0E03EF090082A175E
:20E52000E025E0FF90082A16E033FE744A2FF58274323EF583759308E0FEA3E0C39401FF86
:20E54000EE940090082A10F0A3EFF090082A17E025E0FF90082A16E033FE74622FF582745F
:20E56000323EF583759308E0FEA3E0FF90082A10E0FCA3E0FDC39FEE6480F8EC6480984041
:20E580000301E62FEDAE047803CEA2E713CE13D8F8241AF582742A3EF583759308E0FD7CBB
:20E5A0000090082A11E05407FF74017E00A807088005C333CE33CED8F9FFEE5CFEEF5D4EA8
:20E5C000605A90082A7F7401F09008177BE0FBA3E0FAA3E0F990081AF0E0FEA3E0FFE92FC3
:20E5E000F9EA3EFA900830567484F0A37437F0A3742DF090082A11E02401FE90082A10E000
:20E60000340090083059F0A3CEF01200A41690081AF1E02FF090081AF0E03EF090082A1163
:20E62000E004F0700790082A10E004F001E54B90082A7FE0703C9008177BE0FBA3E0FAA3C6
:20E64000E0F990081AF0E0FEA3E0FFE92FF9EA3EFA900830567484F0A37438F0A37415F04B
:20E660001200A41690081AF1E02FF090081AF0E03EF090082A17E004F0700790082A16E0A0
:20E6800004F0C390082A17E0940490082A16E064809480500301E48C9008064FE0FBA3E0B3
:20E6A000FAA3E0F9E475F00F120087F990081AF0E0FEA3E0FFD39400EE9400500301EB21AF
:20E6C0009008177BE0FBA3E0FAA3E02FF9EA3EFA900830567484F0A37438F0A37419F01274
:20E6E00000A41690081AF1E02FF090081AF0E03EF07F00229008064FE0FBA3E0FAA3E0F9AC
:20E70000E475F00F120087F9788F7C2A7D097B817A9079987E007F0C120085D0E490082AAF
:20E7200080F0A3F0FE7F04FD7B097A2A791A12008F137E007F047D007B097A2A798A12002E
:20E740008F13900839BB7409F0A3742AF0A37486F0A37402F07B097A2A798EE4FF1202B180
:20E76000F578867C2A7D097B097A2A798A7E007F0412008E89EF601F90082A80E0F0A3E022
:20E780004402F0781A7C2A7D097B097A2A79867E007F04120085D0900839BB7409F0A374E6
:20E7A0002AF0A37482F0A37401F07B097A2A798EE4FF1202B1F578827C2A7D097B097A2A94
:20E7C000798A7E007F0412008E89EF601F90082A80E0F0A3E04401F0781A7C2A7D097B0992
:20E7E0007A2A79827E007F04120085D0900830567484F0A37438F0A37437F090082A80E06D
:20E80000FEA3E090082A8F75F00312008A86EE75F003A42583F583759308E0F9A3E0FAA379
:20E82000E090083059C9F0A3EAF0A3E9F09008177BE0FBA3E0FAA3E0F91200A41690081AA9
:20E84000F0EEF0A3EFF090082A80E07002A3E07012782D7C2A7D097B847A3579FA12008D3E
:20E8600055802A900830567484F0A37439F0A37412F090082A8EE004FFF090083059E4F022
:20E88000A3EFF07B097A2A792D1200A4169008177BE0FBA3E0FAA3E0F990081AF0E0FEA33B
:20E8A000E0FFE92FF9EA3EFA900830567484F0A37439F0A37417F0A37409F0A3742AF0A3FE
:20E8C000742DF01200A41690081AF1E02FF090081AF0E03EF090082A80E07002A3E0703FC3
:20E8E0009008177BE0FBA3E0FAA3E0F990081AF0E0FEA3E0FFE92FF9EA3EFA900830567453
:20E9000084F0A37435F0A374FAF01200A41690081AF1E02FF090081AF0E03EF001E9F4E466
:20E9200090082A16F0A3F0C390082D69E09401FF90082D68E09400FE90082A16E0FCA3E041
:20E94000FDC39FEE6480F8EC648098400301E9F4EDAE047803CEA2E713CE13D8F8241AF59D
:20E9600082742A3EF583759308E0FD7C0090082A17E05407FF74017E00A807088005C33320
:20E98000CE33CED8F9FFEE5CFEEF5D4E60539008177BE0FBA3E0FAA3E0F990081AF0E0FEC5
:20E9A000A3E0FFE92FF9EA3EFA900830567484F0A37437F0A3742DF090082A17E02401FE4E
:20E9C00090082A16E0340090083059F0A3CEF01200A41690081AF1E02FF090081AF0E03EAB
:20E9E000F090082A17E004F0700790082A16E004F001E9279008064FE0FBA3E0FAA3E0F985
:20EA0000E475F001120087CD01EB211202E57ABF013F9008177BE0FBA3E0FAA3E0F9900831
:20EA20001AF0E0FEA3E0FFE92FF9EA3EFA900830567484F0A37439F0A37473F01200A416AD
:20EA400090081AF1E02FF090081AF0E03EF001EAE19008177BE0FBA3E0FAA3E0F990081AE8
:20EA6000F0E0FEA3E0FFE92FF9EA3EFA900830567484F0A37439F0A374A5F01200A41690C5
:20EA8000081AF1E02FF090081AF0E03EF090080660E0FBA3E0FAA3E0F9E475F001120087FF
:20EAA000F99008064FE0FBA3E0FAA3E0F9E475F0208027E4FF12011785EF4E7002FF22909A
:20EAC000081AF0E07002A3E060179008064FE0FBA3E0FAA3E0F9E475F021120087F97F009C
:20EAE00022900830567484F0A37439F0A374CCF09008177BE0FBA3E0FAA3E0F91200A41611
:20EB000090081AF0EEF0A3EFF09008064FE0FBA3E0FAA3E0F9E4F5F0120087F980037F01D4
:20EB2000227F002278437C237D097B817A9179647E007F3D120085D078807C237D097B8194
:20EB40007A9179A17E007F2F120085D09008064FE0FBA3E0FAA3E0F9E475F001120087A3B6
:20EB6000AFF0FE600301F4F1EF24FE700301EC4D14700301EF6714700301F2972403600378
:20EB800001F4F1900837CE7484F0A3744FF0A374F5F09008177BE0FBA3E0FAA3E0F91202A6
:20EBA000908C90082447EBF0A3EAF0A3E9F090082447E0FBA3E0FAA3E04A4B70037F0122DA
:20EBC000900831127484F0A3744FF0A374FDF0A37409F0A37424F0A3744AF090082447E0A9
:20EBE000FBA3E0FAA3E0F91200ADE3900830567484F0A37450F0A37407F09008244AE0FE30
:20EC0000A3E0FF90083059EEF0A3EFF02401FFE43EA3F0A3EFF09008177BE0FBA3E0FAA371
:20EC2000E0F91200A41690081AF0EEF0A3EFF09008244AE0F9A3E0FF90080660E0FBA3E070
:20EC4000FAA3E0C98FF0120087F901F4F490082D90E02401FF90082D8FE03400FE90082DF0
:20EC60005FE02FFF90082D5EE03EFE90080660E0FBA3E0FAA3E0F91200877F2401FDE435C3
:20EC8000F0FCC3ED9FEC9E40181202E6D9EF4E7010FE7F98FD7B097A2379AF12008F138038
:20ECA0001B90080660E0FBA3E0FAA3E0F91200877FFF7B097A2379AF1202A96990083056C3
:20ECC0007409F0A37423F0A37443F0A37484F0A37451F0A37470F0900823AFE0FCA3E0FD33
:20ECE000A3E0FEA3E0FF9008305C12008A699008177BE0FBA3E0FAA3E0F91200A416900886
:20ED00001AF0EEF0A3EFF09008177BE0FBA3E0FAA3E0F990081AF0E0FEA3E0FFE92FF9EA8E
:20ED20003EFAC003900830567484F0A37451F0A37473F0900823C3E0FCA3E0FDA3E0FEA302
:20ED4000E0FF9008305912008A69900823B7E0FCA3E0FDA3E0FEA3E0FF9008305D12008A1C
:20ED600069D0031200A41690081AF1E02FF090081AF0E03EF09008244AE4F0A304F0900830
:20ED8000244AE0FEA3E0FFD39404EE64809480400301F4F4EE600301EEB0EF24FE604F1464
:20EDA000700301EE2914700301EE642403600301EEB09008244C7484F0A37451F0A374D78F
:20EDC000F0900823BFE0FCA3E0FDA3E0FEA3E0FF9008245212008A699008244F7484F0A3C1
:20EDE0007451F0A374E5F0900823E301EE9D9008244C7484F0A37451F0A374EFF09008234F
:20EE0000BBE0FCA3E0FDA3E0FEA3E0FF9008245212008A699008244F7484F0A37451F0A3D7
:20EE200074FDF0900823DF80749008244C7484F0A37452F0A37409F0900823D3E0FCA3E09D
:20EE4000FDA3E0FEA3E0FF9008245212008A699008244F7484F0A37452F0A3741AF090089A
:20EE600023C780399008244C7484F0A37452F0A37424F0900823D7E0FCA3E0FDA3E0FEA369
:20EE8000E0FF9008245212008A699008244F7484F0A37452F0A37432F0900823DBE0FCA3E6
:20EEA000E0FDA3E0FEA3E0FF9008245612008A699008177BE0FBA3E0FAA3E0F990081AF0BB
:20EEC000E0FEA3E0FFE92FF9EA3EFAC003C002C001900830567409F0A37423F0A37480F01D
:20EEE0009008244CE0F9A3E0FAA3E090083059C9F0A3EAF0A3E9F090082452E0FCA3E0FDF4
:20EF0000A3E0FEA3E0FF9008305C12008A699008244FE0F9A3E0FAA3E090083060C9F0A35D
:20EF2000EAF0A3E9F090082456E0FCA3E0FDA3E0FEA3E0FF9008306312008A69D001D00237
:20EF4000D0031200A41690081AF1E02FF090081AF0E03EF09008244BE004F07007900824B2
:20EF60004AE004F001ED7E90082D90E02401FF90082D8FE03400FE90082D5FE02FFF90087E
:20EF80002D5EE03EFE90080660E0FBA3E0FAA3E0F91200877F2401FDE435F0FCC3ED9FEC7E
:20EFA0009E40181202E6D9EF4E7010FE7F98FD7B097A2379AF12008F13801B90080660E043
:20EFC000FBA3E0FAA3E0F91200877FFF7B097A2379AF1202A969900830567409F0A37423F2
:20EFE000F0A37443F0A37484F0A37452F0A37445F0900823E7E0FCA3E0FDA3E0FEA3E0FFA6
:20F000009008305C12008A699008177BE0FBA3E0FAA3E0F91200A41690081AF0EEF0A3EFEB
:20F02000F09008244AE4F0A304F09008244AE0FEA3E0FFD39406EE64809480400301F4F48A
:20F04000EE600301F1E0EF24FE605B14700301F0E214700301F11E14700301F15914700377
:20F0600001F1942405600301F1E09008244C7484F0A37452F0A37448F09008242BE0FCA3AE
:20F08000E0FDA3E0FEA3E0FF9008245212008A699008244F7484F0A37452F0A37454F09046
:20F0A00008242701F1CD9008244C7484F0A37451F0A374D7F09008242FE0FCA3E0FDA3E04E
:20F0C000FEA3E0FF9008245212008A699008244F7484F0A37451F0A374E5F0900823F301B7
:20F0E000F1CD9008244C7484F0A37451F0A374EFF090082433E0FCA3E0FDA3E0FEA3E0FFC6
:20F100009008245212008A699008244F7484F0A37452F0A3745DF09008243F01F1CD9008DA
:20F12000244C7484F0A37452F0A3746CF0900823EFE0FCA3E0FDA3E0FEA3E0FF9008245294
:20F1400012008A699008244F7484F0A37452F0A3747AF09008240F80749008244C7484F02E
:20F16000A37452F0A37487F090082413E0FCA3E0FDA3E0FEA3E0FF9008245212008A6990D7
:20F1800008244F7484F0A37452F0A3748FF09008243B80399008244C7484F0A37452F0A381
:20F1A0007499F09008241BE0FCA3E0FDA3E0FEA3E0FF9008245212008A699008244F748406
:20F1C000F0A37452F0A374A3F090082437E0FCA3E0FDA3E0FEA3E0FF9008245612008A69D3
:20F1E0009008177BE0FBA3E0FAA3E0F990081AF0E0FEA3E0FFE92FF9EA3EFAC003C002C097
:20F2000001900830567409F0A37423F0A37480F09008244CE0F9A3E0FAA3E090083059C9E6
:20F22000F0A3EAF0A3E9F090082452E0FCA3E0FDA3E0FEA3E0FF9008305C12008A699008B7
:20F24000244FE0F9A3E0FAA3E090083060C9F0A3EAF0A3E9F090082456E0FCA3E0FDA3E097
:20F26000FEA3E0FF9008306312008A69D001D002D0031200A41690081AF1E02FF090081A48
:20F28000F0E03EF09008244BE004F070079008244AE004F001F02A90082D90E02401FF9040
:20F2A000082D8FE03400FE90082D5FE02FFF90082D5EE03EFE90080660E0FBA3E0FAA3E02E
:20F2C000F91200877F2401FDE435F0FCC3ED9FEC9E40181202E6D9EF4E7010FE7F98FD7BA8
:20F2E000097A2379AF12008F13801B90080660E0FBA3E0FAA3E0F91200877FFF7B097A23E7
:20F3000079AF1202A9699008244AE4F0A304F09008244AE0FEA3E0FFD39403EE6480948078
:20F32000400301F4B3EE600301F3FCEF24FE604514607D2402600301F3FC9008244C748481
:20F34000F0A37452F0A374ADF0900823F7E0FCA3E0FDA3E0FEA3E0FF9008245212008A698C
:20F360009008244F7484F0A37452F0A374B9F0900823FB80749008244C7484F0A37452F08E
:20F38000A374CCF0900823FFE0FCA3E0FDA3E0FEA3E0FF9008245212008A699008244F74EF
:20F3A00084F0A37452F0A374E0F09008240380399008244C7484F0A37452F0A374F4F0904D
:20F3C000082407E0FCA3E0FDA3E0FEA3E0FF9008245212008A699008244F7484F0A374532B
:20F3E000F0A37409F09008240BE0FCA3E0FDA3E0FEA3E0FF9008245612008A699008177BA6
:20F40000E0FBA3E0FAA3E0F990081AF0E0FEA3E0FFE92FF9EA3EFAC003C002C001900830D5
:20F42000567409F0A37423F0A37480F09008244CE0F9A3E0FAA3E090083059C9F0A3EAF020
:20F44000A3E9F090082452E0FCA3E0FDA3E0FEA3E0FF9008305C12008A699008244FE0F9B6
:20F46000A3E0FAA3E090083060C9F0A3EAF0A3E9F090082456E0FCA3E0FDA3E0FEA3E0FF41
:20F480009008306312008A69D001D002D0031200A41690081AF1E02FF090081AF0E03EF0A8
:20F4A0009008244BE004F070079008244AE004F001F30F9008177BE0FBA3E0FAA3E0F9908F
:20F4C000081AF0E0FEA3E0FFE92FF9EA3EFA900830567484F0A37453F0A3741FF01200A44B
:20F4E0001690081AF1E02FF090081AF0E03EF080037F01227F0022787D7C297D097B817A48
:20F500009079A67E007F32120085D078AF7C297D097B817A9079D87E007F06120085D0781B
:20F52000B57C297D097B817A9079DE7E007F0C120085D078C17C297D097B817A9079EA7ED3
:20F54000007F09120085D078CA7C297D097B817A9079F37E007F0F120085D078DC7C297DF4
:20F56000097B817A9179027E007F34120085D09008064FE0FBA3E0FAA3E0F91200877FFF90
:20F58000AEF0E5F0600301FDD1EF24FE700301F6CD14700301F6CD2402600301FDD1900843
:20F5A00030567484F0A3744DF0A374B4F09008177BE0FBA3E0FAA3E0F91200A41690081A52
:20F5C000F0EEF0A3EFF09008177BE0FBA3E0FAA3E0F990081AF0E0FEA3E0FFE92FF9EA3EA2
:20F5E000FA900830567484F0A3744EF0A37475F01200A41690081AF1E02FF090081AF0E04A
:20F600003EF01202E33F9008297312008A699008297BE4F0A304F09008177BE0FBA3E0FA24
:20F62000A3E0F990081AF0E0FEA3E0FFE92FF9EA3EFAC001900830567484F0A3744EF0A35A
:20F6400074B8F09008297CE075F008A4FFC374209FF990082973E0FCA3E0FDA3E0FEA3E0DE
:20F66000FFA80112008967E490083059F0A3EFF0D0011200A41690081AF1E02FF090081A78
:20F68000F0E03EF09008297CE004F070079008297BE004F0D39008297CE094049008297B10
:20F6A000E064809480500301F61790081AF1E024FEF090081AF0E034FFF09008064FE0FB0F
:20F6C000A3E0FAA3E0F9E475F00201FDCB9008177BE0FBA3E0FAA3E0F990081AF0E0FEA3FC
:20F6E000E0FFE92FF9EA3EFA900830567409F0A37429F0A3747DF0A37484F0A3744EF0A336
:20F7000074F2F01200A41690081AF1E02FF090081AF0E03EF01202E34F9008297312008A5F
:20F7200069E47F01FEFDFC9008297712008A69E49008297BF0A3F090082977E0FCA3E0FD91
:20F74000A3E0FEA3E0FF90082973E0F8A3E0F9A3E0FAA3E05FFFEA5EFEE95DFDE85CFCE413
:20F76000FBFAF9F8C31200895670087B847A4F790080067B847A4F7901900829D9EBF0A356
:20F78000EAF0A3E9F09008177BE0FBA3E0FAA3E0F990081AF0E0FEA3E0FFE92FF9EA3EFAE0
:20F7A000C003C002C001900830567409F0A37429F0A374DCF0A37484F0A3744FF0A3740964
:20F7C000F09008297BE0FEA3E0FF9008305CEEF0A3EFF0900829D9E0F9A3E0FAA3E090080E
:20F7E000305EC9F0A3EAF0A3E9F0900829AF75F003EF12008A86EE75F003A42583F5837551
:20F800009308E0F9A3E0FAA3E090083061C9F0A3EAF0A3E9F0D001D002D0031200A41690C7
:20F82000081AF1E02FF090081AF0E03EF090082977E0FCA3E0FDA3E0FEA3E0FF78011200E4
:20F84000897A9008297712008A699008297CE004F070079008297BE004F0C39008297CE0F0
:20F8600094029008297BE064809480500301F73790082DA0E0FEA3E0FF90082D55E02FFF6F
:20F8800090082D54E03EFED3EF9400EE64809480500301FA399008177BE0FBA3E0FAA3E06B
:20F8A000F990081AF0E0FEA3E0FFE92FF9EA3EFA900830567409F0A37429F0A3747DF0A338
:20F8C0007484F0A3744FF0A3740DF01200A41690081AF1E02FF090081AF0E03EF01202E3C1
:20F8E0005F9008297312008A69E47F02FEFDFC9008297712008A699008297BE4F0A304F030
:20F9000090082977E0FCA3E0FDA3E0FEA3E0FF90082973E0F8A3E0F9A3E0FAA3E05FFFEA80
:20F920005EFEE95DFDE85CFCE4FBFAF9F8C31200895670087B847A4F790080067B847A4F63
:20F940007901900829D9EBF0A3EAF0A3E9F09008177BE0FBA3E0FAA3E0F990081AF0E0FE41
:20F96000A3E0FFE92FF9EA3EFAC003C002C001900830567409F0A37429F0A374DCF0A374D7
:20F9800084F0A3744FF0A37422F09008297BE0FEA3E0FF9008305CEEF0A3EFF0900829D9BA
:20F9A000E0F9A3E0FAA3E09008305EC9F0A3EAF0A3E9F0900829B575F003EF12008A86EEB9
:20F9C00075F003A42583F583759308E0F9A3E0FAA3E090083061C9F0A3EAF0A3E9F0D00166
:20F9E000D002D0031200A41690081AF1E02FF090081AF0E03EF090082977E0FCA3E0FDA30D
:20FA0000E0FEA3E0FF78011200897A9008297712008A699008297CE004F070079008297BF7
:20FA2000E004F0C39008297CE094049008297BE064809480500301F9009008177BE0FBA371
:20FA4000E0FAA3E0F990081AF0E0FEA3E0FFE92FF9EA3EFA900830567409F0A37429F0A3BD
:20FA6000747DF0A37484F0A3744FF0A37426F01200A41690081AF1E02FF090081AF0E03E69
:20FA8000F01202E36F9008297312008A69E47F02FEFDFC9008297712008A699008297BE41E
:20FAA000F0A304F090082977E0FCA3E0FDA3E0FEA3E0FF90082973E0F8A3E0F9A3E0FAA380
:20FAC000E05FFFEA5EFEE95DFDE85CFCE4FBFAF9F8C31200895670087B847A4F7900800662
:20FAE0007B847A4F7901900829D9EBF0A3EAF0A3E9F09008177BE0FBA3E0FAA3E0F99008C0
:20FB00001AF0E0FEA3E0FFE92FF9EA3EFAC003C002C001900830567409F0A37429F0A37430
:20FB2000DCF0A37484F0A3744FF0A37442F09008297BE0FEA3E0FF9008305CEEF0A3EFF0AF
:20FB4000900829D9E0F9A3E0FAA3E09008305EC9F0A3EAF0A3E9F0900829C175F003EF126F
:20FB6000008A86EE75F003A42583F583759308E0F9A3E0FAA3E090083061C9F0A3EAF0A370
:20FB8000E9F0D001D002D0031200A41690081AF1E02FF090081AF0E03EF090082977E0FCE4
:20FBA000A3E0FDA3E0FEA3E0FF78011200897A9008297712008A699008297CE004F070076F
:20FBC0009008297BE004F0C39008297CE094039008297BE064809480500301FAA4900817E9
:20FBE0007BE0FBA3E0FAA3E0F990081AF0E0FEA3E0FFE92FF9EA3EFA900830567409F0A353
:20FC00007429F0A3747DF0A37484F0A3744FF0A37446F01200A41690081AF1E02FF090089F
:20FC20001AF0E03EF01202E37F9008297312008A69E47F01FEFDFC9008297712008A69E481
:20FC40009008297BF0A3F090082977E0FCA3E0FDA3E0FEA3E0FF90082973E0F8A3E0F9A323
:20FC6000E0FAA3E05FFFEA5EFEE95DFDE85CFCE4FBFAF9F8C31200895670087B847A4F79C9
:20FC80000080067B847A4F7901900829D9EBF0A3EAF0A3E9F09008177BE0FBA3E0FAA3E029
:20FCA000F990081AF0E0FEA3E0FFE92FF9EA3EFAC003C002C001900830567409F0A3742905
:20FCC000F0A374DCF0A37484F0A3744FF0A37451F09008297BE0FEA3E0FF9008305CEEF07A
:20FCE000A3EFF0900829D9E0F9A3E0FAA3E09008305EC9F0A3EAF0A3E9F0900829CA75F047
:20FD000003EF12008A86EE75F003A42583F583759308E0F9A3E0FAA3E090083061C9F0A347
:20FD2000EAF0A3E9F0D001D002D0031200A41690081AF1E02FF090081AF0E03EF090082918
:20FD400077E0FCA3E0FDA3E0FEA3E0FF78011200897A9008297712008A699008297CE004E1
:20FD6000F070079008297BE004F0C39008297CE094059008297BE064809480500301FC47E8
:20FD80009008177BE0FBA3E0FAA3E0F990081AF0E0FEA3E0FFE92FF9EA3EFA90083056749E
:20FDA00084F0A3744FF0A37455F01200A41690081AF1E02FF090081AF0E03EF09008064F12
:20FDC000E0FBA3E0FAA3E0F9E4F5F0120087F980037F01227F00229008064FE0FBA3E0FAE9
:20FDE000A3E0F9E475F001120087A3AFF0FE600301FFF7EF24FE700301FFA604600301FF79
:20FE0000F7900830567481F0A37493F0A374F5F09008177BE0FBA3E0FAA3E0F91200A41688
:20FE200090081AF0EEF0A3EFF090080660E0FBA3E0FAA3E0F91200877FC39401FFE5F09416
:20FE400000FE90083AFDF0A3EFF01202D8B690083AF912008A69E4FFFEFDFC90083AF9E06C
:20FE6000F8A3E0F9A3E0FAA3E0FBC312008956700301FF5A9008177BE0FBA3E0FAA3E0F994
:20FE800090081AF0E0FEA3E0FFE92FF9EA3EFAC003C002C001900830567481F0A37495F048
:20FEA000A3747FF090083AFEE02401FE90083AFDE0340090083059F0A3CEF090083AF9E0E9
:20FEC000FCA3E0FDA3E0FEA3E0FF781812008967E49008305BF0A3EFF090083AF9E0FCA34E
:20FEE000E0FDA3E0FEA3E0FF781012008967E49008305DF0A3EFF090083AF9E0FCA3E0FDF6
:20FF0000A3E0FEA3E0FF780812008967E49008305FF0A3EFF090083AF9E0FCA3E0FDA3A372
:20FF2000E0FEE490083061F0A3CEF0D001D002D0031200A41690081AF1E02FF090081AF0FF
:20FF4000E03EF090080660E0FBA3E0FAA3E0F9E475F001120087CD01FE2990083AFDE070CA
:20FF600002A3E0600301FFFA9008177BE0FBA3E0FAA3E0F990081AF0E0FEA3E0FFE92FF98E
:20FF8000EA3EFA900830567481F0A37495F0A374B1F01200A41690081AF1E02FF090081AC8
:20FFA000F0E03EF08054900830567481F0A37495F0A374F2F090080660E0FBA3E0FAA3E0FE
:20FFC000F91200877FC39401FEE5F0940090083059F0A3CEF0A3E4F0A3740AF09008177B2D
:20FFE000E0FBA3E0FAA3E0F91200A41690081AF0EEF0A3EFF080037F01227F00228F99224F
:020000040001F9
:20000000E490083CE9F02290083B47EFF0A3EBF0A3EAF0A3E9F0ED2420FFA3F0EDC3940AAC
:200020004003EF04F090083B47E0FF90083B4BE0FD900838757409F0A37432F0A3741EF096
:20004000A37408F0A37401F0E4FBFA120296BE9008321EE0FCA3E0FDA3E0FEA3E0FF900869
:200060003B48E0FBA3E0FAA3E02404F9E43AFA120089AA90083222E0FCA3E0FDA3E0FEA338
:20008000E0FF90083B48E0FBA3E0FAA3E0F9120089AA90083B47E0FF90083B4BE0FD9008C1
:2000A0003B48E0FBA3E0FAA3E02408F9E43AFA90083875EBF0A3EAF0A3E9F0A37404F0A3DE
:2000C0007401F07B087A00120296BE90083B47E0FF90083B4BE0FD90083B48E0FBA3E0FAEF
:2000E000A3E0240CF9E43AFA90083875EBF0A3EAF0A3E9F0A37404F0A37401F07B107A000B
:20010000120296BE90083B47E0FF90083B4BE0FD90083B48E0FBA3E0FAA3E02410F9E43A42
:20012000FA90083875EBF0A3EAF0A3E9F0A37404F0A37401F07B147A00120296BE90083B55
:2001400047E0FF90083B4BE0FD90083B48E0FBA3E0FAA3E02414F9E43AFA90083875EBF01F
:20016000A3EAF0A3E9F0A37404F0A37401F07B187A00120296BE90083B47E0FF90083B4BE7
:20018000E0FD90083B48E0FBA3E0FAA3E02418F9E43AFA90083875EBF0A3EAF0A3E9F0A383
:2001A0007404F0A37401F07B1C7A00120296BE90083B47E0FF90083B4BE0FD90083B48E067
:2001C000FBA3E0FAA3E0241CF9E43AFA90083875EBF0A3EAF0A3E9F0A37404F0A37401F0A7
:2001E0007B207A00120296BE90083B47E0FF90083B4BE0FD90083B48E0FBA3E0FAA3E02474
:2002000020F9E43AFA90083875EBF0A3EAF0A3E9F0A37404F0A37401F07B247A00120296BE
:20022000BE90083B47E0FF90083B4BE0FD90083B48E0FBA3E0FAA3E02424F9E43AFA900825
:200240003875EBF0A3EAF0A3E9F0A37404F0A37401F07B287A00120296BE90083B47E0FF8C
:2002600090083B4BE0FD90083B48E0FBA3E0FAA3E02428F9E43AFA90083875EBF0A3EAF093
:20028000A3E9F0A37404F0A37401F07B2C7A00120296BE90083B47E0FF90083B4BE0FD90C2
:2002A000083B48E0FBA3E0FAA3E0242CF9E43AFA90083875EBF0A3EAF0A3E9F0A37404F053
:2002C000A37401F07B307A00120296BE90083B47E0FF90083B4BE0FD90083B48E0FBA3E01C
:2002E000FAA3E02430F9E43AFA90083875EBF0A3EAF0A3E9F0A37404F0A37401F07B347AC7
:2003000000120296BE90083B47E0FF90083B4BE0FD90083B48E0FBA3E0FAA3E02434F9E456
:200320003AFA90083875EBF0A3EAF0A3E9F0A37404F0A37401F07B387A00120296BE900830
:200340003B47E0FF90083B4BE0FD900838757409F0A37432F0A3741EF0A37408F0A374010A
:20036000F07B447A00120296BE9008321EE0FCA3E0FDA3E0FEA3E0FF90083B48E0FBA3E02C
:20038000FAA3E0243CF9E43AFA120089AA90083222E0FCA3E0FDA3E0FEA3E0FF90083B48C4
:2003A000E0FBA3E0FAA3E02438F9E43AFA120089AA90083B47E0FF90083B4BE0FD90083BE9
:2003C00048E0FBA3E0FAA3E02440F9E43AFA90083875EBF0A3EAF0A3E9F0A37404F0A3744A
:2003E00001F07B4C7A00120296BE90083B47E0FF90083B4BE0FD90083B48E0FBA3E0FAA359
:20040000E02444F9E43AFA90083875EBF0A3EAF0A3E9F0A37404F0A37401F07B507A001200
:200420000296BE90083B47E0FF90083B4BE0FD90083B48E0FBA3E0FAA3E02448F9E43AFAFF
:2004400090083875EBF0A3EAF0A3E9F0A37404F0A37401F07B547A00120296BE90083B47A5
:20046000E0FF90083B4BE0FD90083B48E0FBA3E0FAA3E0244CF9E43AFA90083875EBF0A368
:20048000EAF0A3E9F0A37404F0A37401F07B587A00120296BE90083B47E0FF90083B4BE047
:2004A000FD90083B48E0FBA3E0FAA3E02450F9E43AFA90083875EBF0A3EAF0A3E9F0A37494
:2004C00004F0A37401F07B5C7A00120296BE90083B47E0FF90083B4BE0FD90083B48E0FB7D
:2004E000A3E0FAA3E02454F9E43AFA90083875EBF0A3EAF0A3E9F0A37404F0A37401F07BCC
:20050000607A00120296BE90083B47E0FF90083B4BE0FD90083B48E0FBA3E0FAA3E0245833
:20052000F9E43AFA90083875EBF0A3EAF0A3E9F0A37404F0A37401F07B647A00120296BEBD
:2005400090083B47E0FF90083B4BE0FD90083B48E0FBA3E0FAA3E0245CF9E43AFA90083850
:2005600075EBF0A3EAF0A3E9F0A37404F0A37401F07B687A00120296BE90083B47E0FF90D1
:20058000083B4BE0FD90083B48E0FBA3E0FAA3E02460F9E43AFA90083875EBF0A3EAF0A325
:2005A000E9F0A37404F0A37401F07B6C7A00120296BE90083B47E0FF90083B4BE0FD9008FA
:2005C0003B48E0FBA3E0FAA3E02464F9E43AFA90083875EBF0A3EAF0A3E9F0A37404F0A35D
:2005E0007401F07B707A00120296BE90083B47E0FF90083B4BE0FD90083B48E0FBA3E0FA62
:20060000A3E02468F9E43AFA90083875EBF0A3EAF0A3E9F0A37404F0A37401F07B747A0025
:20062000120296BE90083B47E0FF90083B4BE0FD90083B48E0FBA3E0FAA3E0246CF9E43AC1
:20064000FA90083875EBF0A3EAF0A3E9F0A37404F0A37401F07B787A00120296BE90083BCC
:2006600047E0FF90083B4BE0FD900838757409F0A37432F0A3741EF0A37408F0A37401F032
:200680007B7C7A00120296BE9008321EE0FCA3E0FDA3E0FEA3E0FF90083B48E0FBA3E0FAC7
:2006A000A3E02474F9E43AFA120089AA90083222E0FCA3E0FDA3E0FEA3E0FF90083B48E083
:2006C000FBA3E0FAA3E02470F9E43AFA120089AA90083B47E0FF90083B4BE0FD90083B4826
:2006E000E0FBA3E0FAA3E02478F9E43AFA90083875EBF0A3EAF0A3E9F0A37404F0A3740136
:20070000F07B847A00120296BE90083B47E0FF90083B4BE0FD90083B48E0FBA3E0FAA3E01E
:20072000247CF9E43AFA90083875EBF0A3EAF0A3E9F0A37404F0A37401F07B887A0012024B
:2007400096BE90083B47E0FF90083B4BE0FD90083B48E0FBA3E0FAA3E02480F9E43AFA9016
:20076000083875EBF0A3EAF0A3E9F0A37404F0A37401F07B8C7A00120296BE90083B47E0FA
:20078000FF90083B4BE0FD90083B48E0FBA3E0FAA3E02484F9E43AFA90083875EBF0A3EA03
:2007A000F0A3E9F0A37404F0A37401F07B907A00120296BE90083B47E0FF90083B4BE0FDD9
:2007C00090083B48E0FBA3E0FAA3E02488F9E43AFA90083875EBF0A3EAF0A3E9F0A3740432
:2007E000F0A37401F07B947A00120296BE90083B47E0FF90083B4BE0FD90083B48E0FBA383
:20080000E0FAA3E0248CF9E43AFA90083875EBF0A3EAF0A3E9F0A37404F0A37401F07B987B
:200820007A00120296BE90083B47E0FF90083B4BE0FD90083B48E0FBA3E0FAA3E02490F93F
:20084000E43AFA90083875EBF0A3EAF0A3E9F0A37404F0A37401F07B9C7A00120296BE90CB
:20086000083B47E0FF90083B4BE0FD90083B48E0FBA3E0FAA3E02494F9E43AFA9008387510
:20088000EBF0A3EAF0A3E9F0A37404F0A37401F07BA07A00120296BE7F002290083A79EF99
:2008A000F0E4A3F0A3F090083A79E0FE25E02448F582E4341EF583759308E0FF90083A7E40
:2008C000F0EE25E02449F582E4341EF583759308E0FE90083A7FF0FD7B097A3A797C120236
:2008E000E1E390083A7DE030E16390083A79E0FF24D8F582E4341EF583759308E070107462
:20090000D82FF582E4341EF5837593087401F090083A7EE025E024ACF582E4341DF583C04D
:2009200083C082759308E0FCA3E0FD90083A7FE075F00C8474017E00A8F0088005C333CE84
:2009400033CED8F9FFEC4EFEED4F2109E990083A79E0FF24D8F582E4341EF583759308E004
:20096000B40136EF25E025E0240CF582E4341FF583C083C082759308E0FCA3E0FDA3E0FECB
:20098000A3E02401FFE43EFEE43DFDE43CFC759308D082D08312008A6990083A79E024D875
:2009A000F582E4341EF583759308E4F090083A7EE025E024ACF582E4341DF583C083C08280
:2009C000759308E0FCA3E0FD90083A7FE075F00C8474017E00A8F0088005C333CE33CED8D0
:2009E000F9F4FFEEF45CFEED5FFF759308D082D083EEF0A3EFF090083A7CE0FEA3E0FF20A1
:200A0000E503210AE0EE20E303210AE090083A79E0FF24F4F582E4341AF583759308E0B4DD
:200A2000021074F42FF582E4341AF5837593087401F090083A79E02430F582E4341EF583D3
:200A4000759308E0FF6003B4024B90083A79E0FF2430F582E4341EF5837593087401F0EF3C
:200A600025E025E02478F582E4341EF583C083C082759308E0FCA3E0FDA3E0FEA3E0240191
:200A8000FFE43EFEE43DFDE43CFC759308D082D08312008A6990083A7EE025E0246CF58207
:200AA000E4341FF583C083C082759308E0FCA3E0FD90083A7FE075F00C8474017E00A8F0E5
:200AC000088005C333CE33CED8F9FFEC4EFEED4FFF759308D082D083EEF0A3EFF0210BA0A0
:200AE00090083A7EE025E0246CF582E4341FF583C083C082759308E0FCA3E0FD90083A7FC9
:200B0000E075F00C8474017E00A8F0088005C333CE33CED8F9F4FFEEF45CFEED5FFF7593D0
:200B200008D082D083EEF0A3EFF090083A79E0FF24F4F582E4341AF583759308E0B401128E
:200B400074F42FF582E4341AF5837593087402F0801390083A79E024F4F582E4341AF58370
:200B6000759308E4F090083A79E0FF2430F582E4341EF583759308E0B4011274302FF582ED
:200B8000E4341EF5837593087402F0801390083A79E02430F582E4341EF583759308E4F016
:200BA00090083A7CE0FEA3E0FF20E603210C8AEE20E303210C8A90083A79E0FF2432F58225
:200BC000E4341DF583759308E0B4021074322FF582E4341DF5837593087401F090083A79F9
:200BE000E024B0F582E4341DF583759308E0FF6003B4024B90083A79E0FF24B0F582E4343D
:200C00001DF5837593087401F0EF25E025E024C8F582E4341DF583C083C082759308E0FC50
:200C2000A3E0FDA3E0FEA3E02401FFE43EFEE43DFDE43CFC759308D082D08312008A699068
:200C4000083A7EE025E024F0F582E4341EF583C083C082759308E0FCA3E0FD90083A7FE094
:200C600075F00C8474017E00A8F0088005C333CE33CED8F9FFEC4EFEED4FFF759308D082FD
:200C8000D083EEF0A3EFF0210D4A90083A7EE025E024F0F582E4341EF583C083C08275932E
:200CA00008E0FCA3E0FD90083A7FE075F00C8474017E00A8F0088005C333CE33CED8F9F408
:200CC000FFEEF45CFEED5FFF759308D082D083EEF0A3EFF090083A79E0FF2432F582E4346A
:200CE0001DF583759308E0B4011274322FF582E4341DF5837593087402F0801390083A795B
:200D0000E02432F582E4341DF583759308E4F090083A79E0FF24B0F582E4341DF58375936B
:200D200008E0B4011274B02FF582E4341DF5837593087402F0801390083A79E024B0F5820E
:200D4000E4341DF583759308E4F090083A7CE0FEA3E0FF30E103210F6FEE20E203210E0976
:200D600020E503210E0920E603210E0990083A79E0FF24F4F582E4341EF583759308E0702B
:200D80004AEF25E025E0244CF582E4341DF583C083C082759308E0FCA3E0FDA3E0FEA3E087
:200DA0002401FFE43EFEE43DFDE43CFC759308D082D08312008A6990083A79E024F4F58241
:200DC000E4341EF5837593087401F090083A7EE025E0242CF582E4341EF583C083C082754C
:200DE0009308E0FCA3E0FD90083A7FE075F00C8474017E00A8F0088005C333CE33CED8F928
:200E0000FFEC4EFEED4F210ED390083A7EE025E0242CF582E4341EF583C083C0827593081E
:200E2000E0FCA3E0FD90083A7FE0FB75F00C8474017E00A8F0088005C333CE33CED8F9F493
:200E4000FFEEF45CFEED5FFF759308D082D083EEF0A3EFF090083A79E024F4F582E4341E07
:200E6000F583759308E4F090083A7CE0A320E37674017E00A803088005C333CE33CED8F90B
:200E8000FF90083A7EE0FD25E02428F582E4341EF583759308E0FAA3E0FBEA5EFEEB5F4E6A
:200EA0006041ED25E02428F582E4341EF583C083C08275930890083A7FE0FF74017E00A8CE
:200EC00007088005C333CE33CED8F9F4FFEEF45AFEEB5FFF759308D082D083EEF0A3EFF05D
:200EE0007F01227F032290083A7CA3E020E20620E50330E67790083A7FE0FF74017E00A873
:200F000007088005C333CE33CED8F9FF90083A7EE0FD25E02428F582E4341EF583759308F5
:200F2000E0FAA3E0FBEA5EFEEB5F4E703CED25E02428F582E4341EF583C083C082759308D7
:200F400090083A7FE0FF74017E00A807088005C333CE33CED8F9FFEA4EFEEB4FFF7593081E
:200F6000D082D083EEF0A3EFF07F01227F032290083A79E024F4F582E4341EF583759308AE
:200F8000E4F090083A7CE0FEA3E0FF20E20D20E50A20E607EE20E20330E3037F0122900861
:200FA0003A7FE075F00C8474017E00A8F0088005C333CE33CED8F9FF90083A7EE0FD25E0C4
:200FC000242CF582E4341EF583759308E0FAA3E0FBEA5EFEEB5F4E6041ED25E0242CF582FC
:200FE000E4341EF583C083C08275930890083A7FE075F00C8474017E00A8F0088005C3337A
:20100000CE33CED8F9F4FFEEF45AFEEB5FFF759308D082D083EEF0A3EFF07F022290080664
:201020004FE0FBA3E0FAA3E0F9E475F001120087A3AFF0FE600321177FEF24FE7003211596
:201040002E1470032116552402600321177F900837CE7484F0A3741FF0A374A8F090081706
:201060007BE0FBA3E0FAA3E0F91202908C90082EA0EBF0A3EAF0A3E9F0900831127484F0F4
:20108000A3741FF0A374B1F0A37409F0A3742EF0A374A3F01200ADE390082EA57401F0A36E
:2010A000740EF0900830567484F0A3741FF0A374BCF090082EA3E0FFA3E090083059CFF024
:2010C000A3EFF0A37401F0A3740EF09008177BE0FBA3E0FAA3E0F91200A41690081AF0EE17
:2010E000F0A3EFF09008177BE0FBA3E0FAA3E02FF9EA3EFA900830567484F0A37421F0A35E
:2011000074DFF090082EA4E02401FE90082EA3E0340090083059F0A3CEF01200A4169008CC
:201120001AF1E02FF090081AF0E03EF090082EA3E0F9A3E0FF90080660E0FBA3E0FAA3E058
:20114000C98FF0120087F990082EA4E0FF1202E06890082EA7EEF0A3EFF090082EA4E0FFFA
:201160007B097A2E79BF120235B290082EA7E07004A3E0640460032112559008177BE0FB74
:20118000A3E0FAA3E0F990081AF0E0FEA3E0FFE92FF9EA3EFA900830567484F0A37421F0F3
:2011A000A374EDF01200A41690081AF1E02FF090081AF0E03EF090082EA4E0FF1202DA7571
:2011C000EF4E70087B847A227916803190082EBFE0C4F854F0C8A3E0C4540F48540F900865
:2011E0002F5275F00312008A86E475F003A42583F583759308E0FBA3E0FAA3E0F990082E2A
:20120000A0EBF0A3EAF0A3E9F09008177BE0FBA3E0FAA3E0F990081AF0E0FEA3E0FFE92F42
:20122000F9EA3EFAC002C001900830567484F0A37422F0A37423F090082EA0E0F9A3E0FAFB
:20124000A3E090083059C9F0A3EAF0A3E9F0D001D0022113E49008177BE0FBA3E0FAA3E078
:20126000F990081AF0E0FEA3E0FFE92FF9EA3EFA900830567484F0A37422F0A3742BF012CD
:2012800000A41690081AF1E02FF090081AF0E03EF090082EA7E0FEA3E0FF64024E7003A3AB
:2012A000800AEF64034E90082EA97007F0A37405F08005E4F0A304F090082EA9E0FFA3E05D
:2012C00090082E9ECFF0A3EFF090082E9EE0FEA3E0FFD39406EE6480948040032113BA7CA5
:2012E0000090082EC0E0540FFDEFB5050CECB506087B847A22796180067B847A22796A90BB
:20130000082EA0EBF0A3EAF0A3E9F09008177BE0FBA3E0FAA3E0F990081AF0E0FEA3E0FF23
:20132000E92FF9EA3EFAC003C002C001900830567484F0A37422F0A3746BF090082E9EE04F
:20134000FEA3E0FF90083059EEF0A3EFF090082EA0E0F9A3E0FAA3E09008305BC9F0A3EAE4
:20136000F0A3E9F090082F5275F003EF12008A86EE75F003A42583F583759308E0F9A3E0E9
:20138000FAA3E09008305EC9F0A3EAF0A3E9F0D001D002D0031200A41690081AF1E02FF014
:2013A00090081AF0E03EF090082E9FE004F0700790082E9EE004F02112C99008177BE0FB94
:2013C000A3E0FAA3E0F990081AF0E0FEA3E0FFE92FF9EA3EFA900830567484F0A37422F0B0
:2013E000A37484F01200A41690081AF1E02FF090081AF0E03EF078AB7C2E7D097B847A2256
:20140000799012008D557E0090082EC0E0540FFF64056023EF6402601EEF64046019900862
:2014200039997484F0A37422F0A37495F07B097A2E79AB1202BD179008177BE0FBA3E0FA73
:20144000A3E0F990081AF0E0FEA3E0FFE92FF9EA3EFAC002C001900830567481F0A37491AD
:20146000F0A37436F0A37409F0A3742EF0A374ABF0E4A3F0A3F090082F46E0F9A3E0FAA338
:20148000E09008305EC9F0A3EAF0A3E9F0D001D0021200A41690081AF1E02FF090081AF0E1
:2014A000E03EF090082EBFE030E0087B847A22796180067B847A22796A90082EA0EBF0A344
:2014C000EAF0A3E9F09008177BE0FBA3E0FAA3E0F990081AF0E0FEA3E0FFE92FF9EA3EFA83
:2014E000C002C001900830567484F0A37422F0A3749FF0A3E4F0A304F090082EA0E0F9A3A4
:20150000E0FAA3E09008305BC9F0A3EAF0A3E9F090082F49E0F9A3E0FAA3E09008305EC9C1
:20152000F0A3EAF0A3E9F0D001D00221176B90080660E0FBA3E0FAA3E0F91200877FFF9003
:20154000082EA3E5F0F0A3EFF0A37401F0A37490F07B097A2E79C31202DB5490082EA4E0D7
:2015600024C3F582E4342EF583759308E0B401087B847A22796180067B847A22796A900891
:201580002EA0EBF0A3EAF0A3E9F09008177BE0FBA3E0FAA3E0F990081AF0E0FEA3E0FFE9C0
:2015A0002FF9EA3EFAC003C002C001900830567484F0A37422F0A374C3F090082F40E0F9C2
:2015C000A3E0FAA3E090083059C9F0A3EAF0A3E9F090082EA0E0F9A3E0FAA3E09008305CD5
:2015E000C9F0A3EAF0A3E9F090082F43E0F9A3E0FAA3E09008305FC9F0A3EAF0A3E9F0D0AD
:2016000001D002D0031200A41690081AF1E02FF090081AF0E03EF09008177BE0FBA3E0FA84
:20162000A3E0F990081AF0E0FEA3E0FFE92FF9EA3EFA900830567484F0A37423F0A3741B97
:20164000F090082EA5E0FFA3E090083059CFF0A3EFF021176B90082D90E02401FF90082DAA
:201660008FE03400FE90082D5FE02FFF90082D5EE03EFE90082D55E02FFF90082D54E03EF9
:20168000FE90080660E0FBA3E0FAA3E0F91200877FC39FE5F09E90083056402C7484F0A378
:2016A0007423F0A374E7F0A3E4F0A37406F090080660A3A3E02402F9E43AFA9008305BEBC8
:2016C000F0A3EAF0A3E9802F7484F0A37425F0A3747DF0A3E4F0A37406F090080660E0FB6D
:2016E000A3E0FAA3E0F91200877F2401FEE435F09008305BF0A3CEF0A3E4F0A37405F09026
:2017000008177BE0FBA3E0FAA3E0F91200A41690081AF0EEF0A3EFF09008177BE0FBA3E005
:20172000FAA3E0F990081AF0E0FEA3E0FFE92FF9EA3EFA900830567484F0A37427F0A374B3
:201740003BF0A3E4F0A37406F0A3E4F0A37405F0A3E4F0A37402F0A3E4F0A37404F0A3E4CE
:20176000F0A304F0A3E4F0A37403F01200A41690081AF1E02FF090081AF0E03EF080037F41
:2017800001227F002290082171EFF078A57C217D097B817A9179DC7E017F9E120085D07B62
:2017A000097A21799E1202DC2690080660E0FBA3E0FAA3E0F91200877FC39401FEE5F094AF
:2017C0000090082172F0A3CEF090082172E0FEA3E0FFC39418EE648094804003211D30EF0D
:2017E0004E70489008177BE0FBA3E0FAA3E0F990081AF0E0FEA3E0FFE92FF9EA3EFA900818
:2018000030567484F0A37400F0A374A0F0A37409F0A37421F0A374A5F01200A41690081A4A
:20182000F1E02FF090081AF0E03EF090082173E0FF1201089B90082173E0FF7B097A2179A4
:201840009C1202E27590082173E0FF7B097A21799D1202E29990082173E0FF7B097A21790F
:201860008B1202C1A790082173E0FF7B097A21799B1202C6FD90082173E0FF1202A32C90CE
:201880000821A4EFF09008219BE0D394044002E4F09008219DE0640A6006E49008219BF0B5
:2018A00090082173E025E0FD90082172E033FC74482DF582741E3CF583759308E0FF9008B3
:2018C00021A2F074492DF582741E3CF583759308E0900821A3F07B097A2179871202CF066A
:2018E000900821A3E0FF74017E00A807088005C333CE33CED8F9FF900821A2E025E024ACD9
:20190000F582E4341DF583759308E05EFEA3E05F4E7034FFFEFDFC9008218312008A69E468
:20192000FFFEFDFC9008218B12008A69E4FFFEFDFC9008218712008A69900821A4E0700795
:201940009008219B7405F09008219BE014601314601614601914601C2404701E90082FB536
:20196000801C90082FB8801690082FBB801090082FBE800A90082FC1800490082FC4E0F925
:20198000A3E0FAA3E090082180C9F0A3EAF0A3E9F09008219DE024FB600E24FC60102409DC
:2019A000701290082FDA801090082FDD800A90082FE0800490082FE3E0F9A3E0FAA3E09008
:2019C00008217AC9F0A3EAF0A3E9F09008219CE024FE600904700C90082FAF800A90082FAB
:2019E000B2800490082FACE0F9A3E0FAA3E09008217DC9F0A3EAF0A3E9F0E4FFFEFDFC9013
:201A000008218BE0F8A3E0F9A3E0FAA3E0FB120082DC601AE4FFFEFDFC90082187E0F8A344
:201A2000E0F9A3E0FAA3E0FB120082DC7007E4FFFEFDFC802A90082187E0FCA3E0FDA3E048
:201A4000FEA3E0FFA3E0F8A3E0F9A3E0FAA3E0FB12008128E4FBFA797A78441200823A9073
:201A600008218312008A6990082FC7E0FCA3E0FDA3E0FEA3E0FF90082183E0F8A3E0F9A395
:201A8000E0FAA3E0FB1200803090082FC712008A69900821A4E014601314601614601914AA
:201AA000601C2404702F90082FCB801690082FCE801090082FD1800A90082FD480049008BD
:201AC0002FD7E0F9A3E0FAA3E090082177C9F0A3EAF0A3E9F0900821A3E075F00C8474019F
:201AE0007E00A8F0088005C333CE33CED8F9FF900821A2E025E0249EF582E43421F583750F
:201B00009308E05EFEA3E05F4E60087B847A0079C080067B847A0079C790082174EBF0A3BA
:201B2000EAF0A3E9F09008177BE0FBA3E0FAA3E0F990081AF0E0FEA3E0FFE92FF9EA3EFA1C
:201B4000900830567484F0A37400F0A374CFF01200A41690081AF1E02FF090081AF0E03E74
:201B6000F090082171E09008177B6043E0FBA3E0FAA3E0F990081AF0E0FEA3E0FFE92FF9B7
:201B8000EA3EFA900830567484F0A37400F0A374E4F090082172E0FEA3E0FF90083059EE91
:201BA000F0A3EFF02401FFE43EA3F0A3EF803CE0FBA3E0FAA3E0F990081AF0E0FEA3E0FFB6
:201BC000E92FF9EA3EFA900830567484F0A37401F0A37412F090082173E02401FE900821C3
:201BE00072E0340090083059F0A3CEF01200A41690081AF1E02FF090081AF0E03EF0900837
:201C0000177BE0FBA3E0FAA3E0F990081AF0E0FEA3E0FFE92FF9EA3EFAC003C002C0019053
:201C20000830567484F0A37401F0A3741DF090082174E0F9A3E0FAA3E090083059C9F0A37F
:201C4000EAF0A3E9F09008217AE0F9A3E0FAA3E09008305CC9F0A3EAF0A3E9F09008218310
:201C6000E0FCA3E0FDA3E0FEA3E0FF9008305F12008A6990082187E0FCA3E0FDA3E0FEA319
:201C8000E0FF9008306312008A699008218BE0FCA3E0FDA3E0FEA3E0FF9008306712008AC7
:201CA0006990082180E0F9A3E0FAA3E09008306BC9F0A3EAF0A3E9F090082177E0F9A3E038
:201CC000FAA3E09008306EC9F0A3EAF0A3E9F0D001D002D0031200A41690081AF1E02FF0BB
:201CE00090081AF0E03EF090080660E0FBA3E0FAA3E0F9E475F001120087CD90080660E0D4
:201D0000FBA3E0FAA3E0F91200877FFFAEF07C007D05120086C5ED4C7003FEFF229008213B
:201D200073E004F0700790082172E004F02117C9E4FFFE7D2A7C439008218F12008A69E46D
:201D4000FFFE7D2A7C4390082FC7E0F8A3E0F9A3E0FAA3E0FB120082DC400FE4FFFE7D2AFC
:201D60007C4390082FC712008A6990082FC7E0F8A3E0F9A3E0FAA3E0FB9008218FE0FCA36D
:201D8000E0FDA3E0FEA3E0FF1200802C9008219312008A69E4FFFEFDFC90082FC7E0F8A371
:201DA000E0F9A3E0FAA3E0FB120082DC7006FFFEFDFC80229008218FE0F8A3E0F9A3E0FAB8
:201DC000A3E0FB90082FC7E0FCA3E0FDA3E0FEA3E0FF1200823A9008219712008A699008DD
:201DE000177BE0FBA3E0FAA3E0F990081AF0E0FEA3E0FFE92FF9EA3EFAC003C002C0019072
:201E00000830567484F0A37401F0A37465F09008218FE0FCA3E0FDA3E0FEA3E0FF90083069
:201E20005912008A6990082FC7E0FCA3E0FDA3E0FEA3E0FF9008305D12008A6990082193E1
:201E4000E0FCA3E0FDA3E0FEA3E0FF9008306112008A69E4FFFE7DC87C4290082197E0F8E9
:201E6000A3E0F9A3E0FAA3E0FB120081289008306512008A69D001D002D0031200A416902C
:201E8000081AF1E02FF090081AF0E03EF0E4FFFEFDFC90082FC712008A6990080660E0FB3A
:201EA000A3E0FAA3E0F9E475F001120087F97E007F0122900830B212008A69900830B6EB45
:201EC000F0A3EAF0A3E9F0900830B2A3E0FDA3E0FEA3E0F9AA06AB05900830BDEBF0A3EAD5
:201EE000F0A3E9F0900830CCEBF0A3EAF0A3E9F0900830B9E0FCA3E0FDA3E0FEA3E0FF909E
:201F00000830DA12008A69900830B6E0FBA3E0FAA3E0240EF9E43AFA1200898D7B047A03EA
:201F200079027801C312008956701C900830B2E0FCA3E0FDA3E0FEA3E0FFA3E0FBA3E0FA99
:201F4000A3E0F91201830EE4FFFEFDFC900830DAE0F8A3E0F9A3E0FAA3E0FBC312008956E2
:201F6000700574FF21259C900830B9E0FCA3E0FDA3E0FEA3E0FF900830B6E0FBA3E0FAA33E
:201F8000E0240AF9E43AFA120089AA900830CCE0FBA3E0FAA3E02406F9E43AFA1200898D0B
:201FA000900830D612008A69900830BDE0FBA3E0FAA3E0240AF9E43AFA1200898D900830EF
:201FC000B9E0F8A3E0F9A3E0FAA3E0FBD312008956401DE4FFFEFDFC900830D6E0F8A3E005
:201FE000F9A3E0FAA3E0FB120089566003212158900830CCE0FBA3E0FAA3E02406F9E43A4F
:20200000FA1200898DE4FBFAF9F8C31200895670028010900830CCE0FBA3E0FAA3E0F912A4
:20202000008AD2900830DEEBF0A3EAF0A3E9F0900830DEE0FBA3E0FAA3E04A4B7017900895
:2020400030CCE0F9A3E0FAA3E0900830DEC9F0A3EAF0A3E9F07F047E037D027C019008308B
:20206000B6E0FBA3E0FAA3E0240EF9E43AFA120089AA900830DEE0FBA3E0FAA3E0F990003D
:20208000FFFD12008BA7EBF0A3EAF0A3E9F0900830B6E0FBA3E0FAA3E0F99000FFFD12003C
:2020A0008BA7EBF0A3EAF0A3E9F0900830CCE0FBA3E0FAA3E0F99000FFFD12008BA7EBF007
:2020C000A3EAF0A3E9F0900830CCE0FBA3E0FAA3E0F91202842AE47F01FEFDFC900830D6E4
:2020E000E0F8A3E0F9A3E0FAA3E0FBC3120089564046900830BDE0FBA3E0FAA3E0240AF9D0
:20210000E43AFA1200898D900830B9E0F8A3E0F9A3E0FAA3E0FBC3EF9BFFEE9AFEED99FD5A
:20212000EC98FC900830DEE0FBA3E0FAA3E0240AF9E43AFA120089AA900830B9E0FCA3E03A
:20214000FDA3E0FEA3E0FFA3E0FBA3E0FAA3E0240AF9E43AFA212597E4900830DEF0A3F0D8
:20216000900830B9E0FCA3E0FDA3E0FEA3E0FFA3E0FBA3E0FAA3E0240AF9E43AFA12008927
:20218000E2C3EF9BFFEE9AFEED99FDEC98FC900830B912008A69900830BDE0FBA3E0FAA382
:2021A000E0F9900830CFEBF0A3EAF0A3E9F02406F9E43AFA1200898DE4FBFAF9F8C31200D9
:2021C000895670028010900830CFE0FBA3E0FAA3E0F912008AD2900830C9EBF0A3EAF0A3B9
:2021E000E9F0900830C3EBF0A3EAF0A3E9F0900830CFE0FBA3E0FAA3E02406F9E43AFA12E8
:2022000000898DE4FBFAF9F8C312008956700321237F900830CFE0FBA3E0FAA3E0F9120077
:202220008AD221237F900830C0E0FBA3E0FAA3E04A4B700321238E900830DEE07002A3E0C7
:202240007013900830DFE004F07007900830DEE004F02122F1900830C0E0FBA3E0FAA3E0F8
:20226000240AF9E43AFA1200898D900830D212008A69900830B9E0FCA3E0FDA3E0FEA3E077
:20228000FF900830D2E0F8A3E0F9A3E0FAA3E0FBD312008956400321238E900830DFE004F2
:2022A000F07007900830DEE004F0900830B9E0FCA3E0FDA3E0FEA3E0FF900830D2E0F8A348
:2022C000E0F9A3E0FAA3E0FBC3EF9BFFEE9AFEED99FDEC98FC900830B912008A6990083007
:2022E000C0E0F9A3E0FAA3E0A3C9F0A3EAF0A3E9F0900830C0E0FBA3E0FAA3E04A4B703553
:20230000900830CFE0FBA3E0FAA3E02406F9E43AFA1200898DE4FBFAF9F8C31200895670FA
:2023200002805C900830CFE0FBA3E0FAA3E0F912008AD2804A900830C0E0FBA3E0FAA3E0B9
:20234000F912008AD2C003C002C001900830CFE0FBA3E0FAA3E0F9D082D083D0E06B70082D
:20236000E965827003EA65837005FBFAF98010900830C0E0FBA3E0FAA3E0F912008AD290FB
:202380000830C0EBF0A3EAF0A3E9F0212225900830C3E0FBA3E0FAA3E04A4B7035900830A1
:2023A000CFE0FBA3E0FAA3E02406F9E43AFA1200898DE4FBFAF9F8C3120089567002805C44
:2023C000900830CFE0FBA3E0FAA3E0F912008AD2804A900830C3E0FBA3E0FAA3E0F91200E9
:2023E0008AD2C003C002C001900830CFE0FBA3E0FAA3E0F9D082D083D0E06B7008E96582C8
:202400007003EA65837005FBFAF98010900830C3E0FBA3E0FAA3E0F912008AD2900830C629
:20242000EBF0A3EAF0A3E9F0900830B9E0FCA3E0FDA3E0FEA3E0FF900830B6E0FBA3E0FA12
:20244000A3E0240AF9E43AFA120089AA7F047E037D027C01900830B6E0FBA3E0FAA3E024F8
:202460000EF9E43AFA120089AA900830C6E0FBA3E0FAA3E04A4B707E900830CFE0F9A3E019
:20248000FAA3E0900830C6C9F0A3EAF0A3E9F0900830C6E0FBA3E0FAA3E0F99000FFFD127F
:2024A000008BA7EBF0A3EAF0A3E9F0900830B6E0FBA3E0FAA3E0F99000FFFD12008BA7EB09
:2024C000F0A3EAF0A3E9F0900830C3E0FBA3E0FAA3E0F99000FFFD12008BA7EBF0A3EAF08C
:2024E000A3E9F0900830CFE0FBA3E0FAA3E0F91202842A21259B900830C6E0FBA3E0FAA3C9
:20250000E0F99000FFFD12008BA7EBF0A3EAF0A3E9F0900830B6E0FBA3E0FAA3E0F990005C
:20252000FFFD12008BA7EBF0A3EAF0A3E9F0900830C3E0FBA3E0FAA3E0F99000FFFD12008A
:202540008BA7EBF0A3EAF0A3E9F0900830CFE0FBA3E0FAA3E0F91202842A900830C6E0FBDF
:20256000A3E0FAA3E0240AF9E43AFAC003C002C0011200898D900830B9E0F8A3E0F9A3E056
:20258000FAA3E0FBC3EF9BFFEE9AFEED99FDEC98FCD001D002D003120089AAE4FFFEFDFC59
:2025A000229008064FE0FBA3E0FAA3E0F91200877FFFAEF0E5F06003212C33EF24FE603723
:2025C0001460701470032127DC14700321291C147003212BB724056003212C337F017E00EB
:2025E000120299A49008064FE0FBA3E0FAA3E0F9E475F002212C2C900830567484F0A374E8
:202600002CF0A3741AF09008177BE0FBA3E0FAA3E0F91200A41690081AF0EEF0A3EFF09021
:2026200008064FE0FBA3E0FAA3E0F9E475F003120087F990080660E0FBA3E0FAA3E0F912A7
:2026400000877FC39401FFE5F09400FE7B097A3479111202C505EF4E705090080660E0FB46
:20266000A3E0FAA3E0F91200877FFF90080655E0FBA3E0FAA3E0F9E5F08FF0120087F9900D
:2026800008064FE0FBA3E0FAA3E0F9E475F004120087F9D390081AF1E0940090081AF0E0BE
:2026A000940050032127DC7F002290080660E0FBA3E0FAA3E0F91200877FC39401FFE5F058
:2026C0009400FE90083CCAE0B50616A3E0B507119008341B7484F0A3742CF0A374C5F0807B
:2026E0000F9008341B7484F0A3742CF0A374CEF090083411E0FEA3E0FF64014E9008341E1A
:20270000700D7484F0A3742CF0A374CFF0800B7484F0A3742CF0A374CEF09008177BE0FBCB
:20272000A3E0FAA3E0F990081AF0E0FCA3E0FDE92DF9EA3CFAC003C002C00190083056749B
:2027400084F0A3742CF0A374DFF090080660E0FBA3E0FAA3E0F91200877FFD90083059E5FF
:20276000F0F0A3EDF09008341BE0F9A3E0FAA3E09008305BC9F0A3EAF0A3E9F0A3EEF0A340
:20278000EFF09008341EE0F9A3E0FAA3E090083060C9F0A3EAF0A3E9F0D001D002D0031235
:2027A00000A41690081AF1E02FF090081AF0E03EF090080660E0FBA3E0FAA3E0F9E475F0F2
:2027C00001120087CDC390081AF1E0948490081AF0E0940350032126337F0022C390082D25
:2027E00069E09401FF90082D68E09400F990080659E0FBA3E0FAA3E0C98FF0120087F99026
:2028000008177BE0FBA3E0FAA3E0F990081AF0E0FEA3E0FFE92FF9EA3EFA900830567484FF
:20282000F0A3742CF0A374FBF01200A41690081AF1E02FF090081AF0E03EF09008340DE498
:20284000F0A304F090080659E0FBA3E0FAA3E0F91200877FFF9008340DE0FCA3E0FDD39F68
:20286000EC95F050549008177BE0FBA3E0FAA3E0F990081AF0E0FEA3E0FFE92FF9EA3EFA10
:20288000900830567484F0A3742DF0A374B9F0A3ECF0A3EDF01200A41690081AF1E02FF0D1
:2028A00090081AF0E03EF09008340EE004F070949008340DE004F0808B9008177BE0FBA356
:2028C000E0FAA3E0F990081AF0E0FEA3E0FFE92FF9EA3EFA900830567484F0A3742DF0A390
:2028E00074C7F01200A41690081AF1E02FF090081AF0E03EF090080660E0FBA3E0FAA3E0B6
:20290000F9E475F001120087F99008064FE0FBA3E0FAA3E0F9E475F005212C2C90083CCABC
:20292000E0FEA3E0FF7B097A3479111202C505EF4E700EFE7F0AFD7B097A34791112008F01
:202940001390080659E0FBA3E0FAA3E0F91200877FFFAEF090080660E0FBA3E0FAA3E0F912
:202960001200877FFDACF0D39FEC9E402B9008064FE0FBA3E0FAA3E0F9E475F00612008796
:20298000F9D390081AF1E0940090081AF0E094005003212BB77F0022C3ED9401FEEC940084
:2029A0009008340FF0A3CEF0E490083421F0A3F09008340FE0FEA3E07803CEA2E713CE1395
:2029C000D8F82413F58274343EF583759308E0FD7C0090083410E05407F974017E00A80106
:2029E000088005C333CE33CED8F9FBAA06EA5CFEEB5D4E601090083422E004F070079008EE
:202A00003421E004F09008340FE0FEA3E07803CEA2E713CE13D8F82417F58274343EF583AB
:202A2000759308E0FFEB5F601090083422E004F0700790083421E004F09008177BE0FBA34B
:202A4000E0FAA3E0F990081AF0E0FEA3E0FFE92FF9EA3EFA900830567484F0A3742EF0A30D
:202A6000740FF01200A41690081AF1E02FF090081AF0E03EF09008340DE4F0A37402F0907F
:202A800008340DE0FEA3E0FFC3EE648094805003212B8C90083421E0FCA3E0FDEFB50515B2
:202AA000EEB504119008341B7484F0A3742EF0A37417F0800F9008341B7484F0A3742CF0AB
:202AC000A374CEF09008340DE0FEA3E0FF4E9008341E600D7484F0A3742EF0A3741FF08080
:202AE0000B7484F0A3742CF0A374CEF09008177BE0FBA3E0FAA3E0F990081AF0E0FCA3E0DC
:202B0000FDE92DF9EA3CFAC003C002C001900830567484F0A3742EF0A37424F09008340F02
:202B2000E0FDA3E090083059CDF0A3EDF0A3EEF0A3EFF09008341BE0F9A3E0FAA3E090087C
:202B4000305DC9F0A3EAF0A3E9F09008341EE0F9A3E0FAA3E090083060C9F0A3EAF0A3E989
:202B6000F0D001D002D0031200A41690081AF1E02FF090081AF0E03EF09008340EE024FFF4
:202B8000F09008340DE034FFF0212A7F90080660E0FBA3E0FAA3E0F9E475F001120087CD1D
:202BA000C390081AF1E0948490081AF0E0940350032129417F002290083CCAE07002A3E0AC
:202BC0009008341B700D7484F0A3742EF0A37450F0800B7484F0A3742CF0A374CEF090080A
:202BE00030567484F0A3742EF0A37459F09008341BE0F9A3E0FAA3E090083059C9F0A3EAAB
:202C0000F0A3E9F09008177BE0FBA3E0FAA3E0F91200A41690081AF0EEF0A3EFF0900806DE
:202C20004FE0FBA3E0FAA3E0F9E4F5F0120087F97F00227F01229008064FE0FBA3E0FAA3EB
:202C4000E0F91200877FFFE5F06003213272EF24FE7003212EC3147003213116147003215A
:202C6000321C24036003213272E49008334BF0A3F0FE7F04FD7B097A33794712008F137E99
:202C8000007F047D007B097A33794212008F13900839BB7409F0A37433F0A3743EF0A37405
:202CA00002F07B097A337946E4FF1202B1F5783E7C337D097B097A3379427E007F041200AB
:202CC0008E89EF601F9008334BE0F0A3E04402F078477C337D097B097A33793E7E007F04F3
:202CE000120085D0900839BB7409F0A37433F0A3743AF0A37401F07B097A337946E4FF120C
:202D000002B1F5783A7C337D097B097A3379427E007F0412008E89EF601F9008334BE0F0BA
:202D2000A3E04401F078477C337D097B097A33793A7E007F04120085D0900830567484F095
:202D4000A3743FF0A3740FF09008177BE0FBA3E0FAA3E0F91200A41690081AF0EEF0A3EF3B
:202D6000F0E490083352F0A3F090083352E0FEA3E0FFD39403EE648094804003212E5F9091
:202D800008334BE0FCA3E0FDEFB50515EEB504119008334F7484F0A37440F0A3746EF0809D
:202DA0000F9008334F7484F0A37440F0A37477F09008177BE0FBA3E0FAA3E0F990081AF09D
:202DC000E0FEA3E0FFE92FF9EA3EFAC003C002C001900830567484F0A37440F0A37478F04E
:202DE00090083352E0FEA3E0FF90083059EEF0A3EFF09008334FE0F9A3E0FAA3E09008301A
:202E00005BC9F0A3EAF0A3E9F09008374775F003EF12008A86EE75F003A42583F5837593F4
:202E200008E0F9A3E0FAA3E09008305EC9F0A3EAF0A3E9F0D001D002D0031200A4169008FF
:202E40001AF1E02FF090081AF0E03EF090083353E004F0700790083352E004F0212D699017
:202E600008177BE0FBA3E0FAA3E0F990081AF0E0FEA3E0FFE92FF9EA3EFA90083056748499
:202E8000F0A37440F0A37493F01200A41690081AF1E02FF090081AF0E03EF09008064FE076
:202EA000FBA3E0FAA3E0F9E475F002120087F990080660E0FBA3E0FAA3E0F9E475F0011213
:202EC0000087F9E49008334BF0A3F0FE7F04FD7B097A33794712008F137E007F047D007BD9
:202EE000097A33794212008F13900839BB7409F0A37433F0A3743EF0A37402F07B097A33FB
:202F00007946E4FF1202B1F5783E7C337D097B097A3379427E007F0412008E89EF601F9056
:202F200008334BE0F0A3E04402F078477C337D097B097A33793E7E007F04120085D09008A6
:202F400039BB7409F0A37433F0A3743AF0A37401F07B097A337946E4FF1202B1F5783A7CD2
:202F6000337D097B097A3379427E007F0412008E89EF601F9008334BE0F0A3E04401F078FE
:202F8000477C337D097B097A33793A7E007F04120085D090080660E0FBA3E0FAA3E0F91285
:202FA00000877FFFAEF090083354EEF0A3EFF0C390082D69E09401FD90082D68E09400FCEF
:202FC000D3EF9DEC6480F8EE64809840032130B3C390083355E09401FF90083354E094002F
:202FE000FE90083346E07C00B50715ECB506119008334F7484F0A37440F0A3746EF0800F90
:203000009008334F7484F0A37440F0A37477F09008177BE0FBA3E0FAA3E0F990081AF0E069
:20302000FEA3E0FFE92FF9EA3EFAC002C001900830567484F0A37440F0A374F5F090083346
:2030400054E0FCA3E0FDC39401FEEC940090083059F0A3CEF09008334FE0F9A3E0FAA3E085
:203060009008305BC9F0A3EAF0A3E9F0A3ECF0A3EDF0D001D0021200A41690081AF1E02F5B
:20308000F090081AF0E03EF090080660E0FBA3E0FAA3E0F9E475F001120087CDC390081A99
:2030A000F1E094B090081AF0E094045003212F937F00229008177BE0FBA3E0FAA3E0F9907C
:2030C000081AF0E0FEA3E0FFE92FF9EA3EFA900830567484F0A37441F0A37412F01200A42E
:2030E0001690081AF1E02FF090081AF0E03EF09008064FE0FBA3E0FAA3E0F9E475F0031249
:203100000087F990080660E0FBA3E0FAA3E0F9E475F00121326BE49008334BF0A3F0FE7F5B
:2031200004FD7B097A33794712008F137E007F047D007B097A33794212008F13900839BB3F
:203140007409F0A37433F0A3743EF0A37402F07B097A337946E4FF1202B1F5783E7C337D0B
:20316000097B097A3379427E007F0412008E89EF601F9008334BE0F0A3E04402F078477CE8
:20318000337D097B097A33793E7E007F04120085D0900839BB7409F0A37433F0A3743AF0B2
:2031A000A37401F07B097A337946E4FF1202B1F5783A7C337D097B097A3379427E007F04A6
:2031C00012008E89EF601F9008334BE0F0A3E04401F078477C337D097B097A33793A7E0064
:2031E0007F04120085D090083AD27484F0A37441F0A3745FF07B097A3379471202D4DAEF09
:2032000064014E70149008064FE0FBA3E0FAA3E0F9E475F004120087F97F00229008305618
:203220007484F0A37441F0A37463F0C390082D69E09401FE90082D68E0940090083059F0DE
:20324000A3CEF09008177BE0FBA3E0FAA3E0F91200A41690081AF0EEF0A3EFF09008064F54
:20326000E0FBA3E0FAA3E0F9E4F5F0120087F97F00227F0122787C7C067D097B817A93795E
:203280007A7E007F7B120085D07B097A0679701202DC26900837CE7484F0A37407F0A37428
:2032A00015F09008177BE0FBA3E0FAA3E0F91202908C9008066AEBF0A3EAF0A3E9F0900867
:2032C00031127484F0A37407F0A3741DF0A37409F0A37406F0A37466F01200ADE3900806C7
:2032E0004FE0FBA3E0FAA3E0F91200877FFFAEF0E5F06003213862EF24FE70032134831493
:2033000070032138252402600321386290080667E0FF7B097A0679741202E2759008066733
:20332000E0FF7B097A0679751202E2879008067BE075F00C8474017E00A8F0088005C33343
:20334000CE33CED8F9FF9008067AE075F00C8425E02470F582E43406F583759308E05EFEEF
:20336000A3E05FFF4E60087B847A07792780067B847A0779309008066AEBF0A3EAF0A3E9FB
:20338000F0EF4E60087B847A07793080067B847A0779279008066DEBF0A3EAF0A3E9F0905A
:2033A000080667E025E0FF90080666E033FE74482FF582741E3EF583759308E0FD9008066A
:2033C0007AF074492FF582741E3EF583759308E09008067BF075F00C8474017E00A8F00857
:2033E0008005C333CE33CED8F9FFED75F00C8425E02470F582E43406F583759308E05EFEDF
:20340000A3E05F4E600B90080668E4F0A304F08008E490080668F0A3F0900830567484F0A5
:20342000A37407F0A37431F090080668E0FFA3E090083059CFF0A3EFF090080666E0FFA3F6
:20344000E09008305BCFF0A3EFF0A37409F0A37406F0A3747CF09008177BE0FBA3E0FAA363
:20346000E0F91200A41690081AF0EEF0A3EFF09008064FE0FBA3E0FAA3E0F9E475F0021287
:203480000087F99008177BE0FBA3E0FAA3E0F990081AF0E0FEA3E0FFE92FF9EA3EFAC003B6
:2034A000C002C001900830567484F0A37408F0A3744EF090080667E02401FE90080666E033
:2034C000340090083059F0A3CEF09008066AE0F9A3E0FAA3E09008305BC9F0A3EAF0A3E980
:2034E000F09008066DE0F9A3E0FAA3E09008305EC9F0A3EAF0A3E9F0D001D002D003120098
:20350000A41690081AF1E02FF090081AF0E03EF09008177BE0FBA3E0FAA3E0F990081AF0FF
:20352000E0FEA3E0FFE92FF9EA3EFA900830567484F0A37408F0A374DFF01200A416900899
:203540001AF1E02FF090081AF0E03EF0E490080668F0A3F090080668E0FEA3E0FFC3940B7C
:20356000EE64809480400321380E90080675E0FD7C00EFB5050CECB506087B847A077927CB
:2035800080067B847A0779309008066AEBF0A3EAF0A3E9F090080668E0FEA3E0FFEE6003E9
:2035A0002137FBEF24FB700321363F24FC70032136CE14700321375D240A60032137FB9039
:2035C000082FDAE0F9A3E0FAA3E09008066DC9F0A3EAF0A3E9F09008177BE0FBA3E0FAA31F
:2035E000E0F990081AF0E0FCA3E0FDE92DF9EA3CFAC002C001900830567484F0A37409F02C
:20360000A3740AF09008066AE0F9A3E0FAA3E090083059C9F0A3EAF0A3E9F0A3EEF0A3EFD2
:20362000F09008066DE0F9A3E0FAA3E09008305EC9F0A3EAF0A3E9F0D001D0022137E9906A
:20364000082FDDE0F9A3E0FAA3E09008066DC9F0A3EAF0A3E9F09008177BE0FBA3E0FAA39B
:20366000E0F990081AF0E0FEA3E0FFE92FF9EA3EFAC003C002C001900830567484F0A374D9
:2036800009F0A3740AF09008066AE0F9A3E0FAA3E090083059C9F0A3EAF0A3E9F0900806CE
:2036A00068E0FFA3E09008305CCFF0A3EFF09008066DE0F9A3E0FAA3E09008305EC9F0A375
:2036C000EAF0A3E9F0D001D002D0032137E990082FE0E0F9A3E0FAA3E09008066DC9F0A3F6
:2036E000EAF0A3E9F09008177BE0FBA3E0FAA3E0F990081AF0E0FEA3E0FFE92FF9EA3EFA41
:20370000C003C002C001900830567484F0A37409F0A3740AF09008066AE0F9A3E0FAA3E05B
:2037200090083059C9F0A3EAF0A3E9F090080668E0FFA3E09008305CCFF0A3EFF09008064B
:203740006DE0F9A3E0FAA3E09008305EC9F0A3EAF0A3E9F0D001D002D0032137E990082FCD
:20376000E3E0F9A3E0FAA3E09008066DC9F0A3EAF0A3E9F09008177BE0FBA3E0FAA3E0F9D2
:2037800090081AF0E0FEA3E0FFE92FF9EA3EFAC003C002C001900830567484F0A37409F098
:2037A000A3740AF09008066AE0F9A3E0FAA3E090083059C9F0A3EAF0A3E9F090080668E05E
:2037C000FFA3E09008305CCFF0A3EFF09008066DE0F9A3E0FAA3E09008305EC9F0A3EAF0C2
:2037E000A3E9F0D001D002D0031200A41690081AF1E02FF090081AF0E03EF090080669E0D2
:2038000004F0700790080668E004F02135549008064FE0FBA3E0FAA3E0F9E475F00312009A
:2038200087F97F0022900830567484F0A37409F0A37425F09008177BE0FBA3E0FAA3E0F927
:203840001200A41690081AF0EEF0A3EFF09008064FE0FBA3E0FAA3E0F9E4F5F0120087F97E
:2038600080037F01227F0022900833F5EFF0A3EDF0A3EBF0A3EAF0A3E9F0E4900833FBF052
:20388000A3F0A3F0A304F0E4A3F0A3F0A3F0A3F0A3F0A3F0A3F0A3F01200877F540F64060A
:2038A00060032139BE900833FA7403F0900833F6E0FEC3940A507F900833F5E0FFEEFB7A90
:2038C00000900806FB7409F0A37433F0A374FAF0A37401F0A3F0E4FD1202A1DD900833F5D9
:2038E000E0FFA3E02410FD900806FB7409F0A37433F0A374FDF0A37402F0A314F07B087A44
:20390000001202A1DD900833FB7412F0A3E4F0900833F5E0FFA3E02410FD900806FB7409F9
:20392000F0A37433F0A374FBF0A37402F0A314F0E4FBFA213E2C900833F5E0FFA3E02412EF
:20394000FB7A00900806FB7409F0A37433F0A374FAF0A37401F0A3F0E4FD1202A1DD90080B
:2039600033F6E0640A6003213E30900833F5E0FF900838757409F0A37433F0A374FBF0A3AE
:203980007402F0A314F0E4FBFA7D1A120296BE900833FBE04408F0A3E0F0900833F5E0FF4E
:2039A000900806FB7409F0A37433F0A374FBF0A37402F0A314F0E4FBFA7D1A213E2CE490A6
:2039C0000833FAF0900833F6E0FEC3940A900833F5E0FF5003EE8004A3E02412FB7A0090A0
:2039E0000806FB7409F0A37433F0A374FAF0A37401F0A3F0E4FD1202A1DD900833F6E0FD6A
:203A0000C3940A4003213A9A900833FDE04401F0A3E044E0F0900833F7E0FBA3E0FAA3E0FC
:203A2000F91200877FE5F030E00B900833FDE04404F0A3E0F0900833F5E0FFED2410FD90E5
:203A40000806FB7409F0A37433F0A374FDF0A37402F0A314F07B087A001202A1DD900833A8
:203A6000FBE04410F0A3E0F0900833FBE04402F0A3E0F0900833F5E0FFA3E02410FD90087A
:203A800006FB7409F0A37433F0A374FBF0A37402F0A314F0E4FBFA213BE7900833F6E064AB
:203AA0000A6003213BEB900833F5E0FF900838757409F0A37434F0A37407F0A37402F0A30C
:203AC00014F0E4FBFA7D1A120296BE90083407E054F7F0A3E0F0900833F5E0FF900806FB71
:203AE0007409F0A37434F0A37407F0A37402F0A314F0E4FBFA7D1A1202A1DD900833FDE0B6
:203B00004401F0A3E044E0F0900833F7E0FBA3E0FAA3E0F91200877FE5F030E00B90083370
:203B2000FDE0440CF0A3E0F0900833F5E0FF900806FB7409F0A37433F0A374FDF0A37402F9
:203B4000F0A314F07B087A007D1A1202A1DD900833F5E0FF900838757409F0A37433F0A37A
:203B600074FDF0A37402F0A314F07B127A007D1A120296BE900833FDE04403F0A3E0F0904C
:203B80000833F5E0FF900806FB7409F0A37433F0A374FDF0A37402F0A314F07B127A007D9E
:203BA0001A1202A1DD900833FBE04410F0A3E0F0900833FBE04402F0A3E0F0900833FBE007
:203BC000F0A3E04440F0900833F5E0FF900806FB7409F0A37433F0A374FBF0A37402F0A371
:203BE00014F0E4FBFA7D1A1202A1DD900833F7E0FBA3E0FAA3E0F91200877F540F640570D5
:203C000003213D451202E2EFEF240AFFE43EFEE43DFDE43CFC9008340912008A691202E2D3
:203C2000EF90083409E0F8A3E0F9A3E0FAA3E0FBD31200895650E6900833F6E0FEC3940A77
:203C40005064A3E0FBA3E0FAA3E0F91200877F540F24FE600F1460142402701C900833FB2D
:203C60007421800E900833FB74208006900833FB7401F0A3E4F08008E4900833FBF0A3F0EA
:203C8000900833F5E0FFEE2410FD900806FB7409F0A37433F0A374FBF0A37402F0A314F074
:203CA000E4FBFA213D41900833F6E0640A6003213D45A3E0FBA3E0FAA3E0F91200877F5494
:203CC0000F24FE600F1460142402701C900833FB7421800E900833FB74208006900833FB7B
:203CE0007401F0A3E4F08008E4900833FBF0A3F0900833F5E0FF900806FB7409F0A3743344
:203D0000F0A374FBF0A37402F0A314F0E4FBFA7D1A1202A1DD90083405E4F0A37480F09043
:203D20000833F5E0FF900806FB7409F0A37434F0A37405F0A37402F0A314F07B3C7A007DC9
:203D40001A1202A1DD900833F5E0FF900838757409F0A37434F0A37401F0A37402F0A31463
:203D6000F07B137A007D30120296BE900833F7E0FBA3E0FAA3E0F91200877FE5F030E0445F
:203D8000900833F6E0FFC3940A501274017E00A807088005C333CE33CED8F9801990083397
:203DA000F6E0C39401FF74017E00A807088005C333CE33CED8F9FF90083401E04EF0A3E0A4
:203DC0004FF08046900833F6E0FFC3940A501274017E00A807088005C333CE33CED8F98036
:203DE00019900833F6E0C39401FF74017E00A807088005C333CE33CED8F9F4FFEEF4FE908A
:203E0000083401E05EF0A3E05FF0900833F5E0FF900806FB7409F0A37434F0A37401F0A3DA
:203E20007402F0A314F07B137A007D301202A1DD2290082552EBF0A3EAF0A3E9F0E49008AD
:203E40002609F0A3F0FE7F51FD7B097A25795F12008F137E007F517D007B097A2579B0120D
:203E6000008F137E007F047D007B097A25795B12008F13900834C37481F0A3749FF0A37446
:203E80001DF0A37481F0A3749EF0A3742CF0A37409F0A37425F0745512025957900834C35D
:203EA0007481F0A3749FF0A37422F0A37481F0A3749EF0A3742CF0A37409F0A37425F0743E
:203EC0005F12025957900834C37481F0A3749FF0A37427F0A37481F0A3749EF0A3742CF017
:203EE000A37409F0A37425F0A374B012025958900834C37481F0A3749FF0A3742CF0A37496
:203F000081F0A3749EF0A3742CF0A37409F0A37425F0A3745B120259587B097A25795F12D8
:203F200002551D7B097A2579B01202551D7B097A2579551202851F90082601EEF0A3EFF073
:203F4000D39400EE9400400CE094FF90082601E094FF40119008395A7481F0A3749FF0A3DD
:203F600074422142847B097A25795B1202851F90082603EEF0A3EFF0C39403EE6480948094
:203F8000400FD3E0941E90082603E06480948040119008395A7481F0A3749FF0A374632132
:203FA0004284E490082617F0A3F090082617E0FEA3E0FFD39402EE648094804003214214C1
:203FC000EE7060EF14602414603E24027055900826217481F0A3749FF0A3747FF0A3748177
:203FE000F0A3749FF0A37483F08038900826217481F0A3749FF0A37496F0A37481F0A37443
:204000009FF0A3749AF0801B900826217481F0A3749FF0A374AEF0A37481F0A3749FF0A3E5
:2040200074B2F0E490082605F0A3F090082621E0F9A3E0FAA3E0900837CEC9F0A3EAF0A312
:20404000E9F090082552E0FBA3E0FAA3E0F91202908C90082552EBF0A3EAF0A3E9F0C002CF
:20406000C00190082621E0F9A3E0FAA3E0900834C3C9F0A3EAF0A3E9F0A37481F0A3749E49
:20408000F0A3742CF0A37409F0A37426F0A37427F0D001D00212025965E490082607F0A3E1
:2040A000F07B097A2679271200BA43C390082608E09FEE6480F890082607E06480985041B9
:2040C000A3E02427F582E43426F583759308E0FF1202E4A5401990082624E0F9A3E0FAA325
:2040E000E09008395AC9F0A3EAF0A3E921428490082608E004F070A990082607E004F08040
:20410000A07B097A2679271202851FAC06AD0790082606E025E0FF90082605E033FE741914
:204120002FF58274263EF583759308ECF0A3EDF090082553E475F001120087539008260613
:20414000E004F0700790082605E004F0C390082606E0940490082605E0648094805003216F
:20416000402B90082617E0FEA3E0FF64014E7045EF7802C333CE33CED8F9240BF974263E38
:20418000FA900836CA7409F0A3EAF0A3E9F07B097A2679191202175EEF4E706590082624F4
:2041A000E0F9A3E0FAA3E09008395AC9F0A3EAF0A3E921428490082617E0FEA3E07802C3DF
:2041C00033CE33CED8F9240BF974263EFA900837627409F0A3EAF0A3E9F07B097A267919C5
:2041E0001202448EEF4E701990082624E0F9A3E0FAA3E09008395AC9F0A3EAF0A3E9214208
:204200008490082618E004F0700790082617E004F0213FAA9008260FE0FCA3E0FDA3E0FE9C
:20422000A3E0FFA3E0F8A3E0F9A3E0FAA3E05FFFEA5EFEE95DFDE85CFCC004C005C006ABE4
:20424000079008260FE0FCA3E0FDA3E0FEA3E0FF9008260BE0F8A3E0F9A3E0FAA3E05FFFB0
:20426000EA5EFEE95DFDE85CFCD002D001D000C31200895660299008395A7481F0A3749FFF
:20428000F0A374C5F0A37481F0A3749FF0A3745BF07B817A9F79331202A5C0E4FEFF221283
:2042A00002E30F9008260BE0F8A3E0F9A3E0FAA3E0FBC31200895660279008260BE0FCA36F
:2042C000E0FDA3E0FEA3E0FF90082D5612008A6990082D50E4F0A304F0900819E37410F056
:2042E0001202E31F9008260FE0F8A3E0F9A3E0FAA3E0FBC31200895660209008260FE0FCAF
:20430000A3E0FDA3E0FEA3E0FF90082D6C12008A6990082D50E4F0A304F01202E32F9008A6
:204320002613E0F8A3E0F9A3E0FAA3E0FBC312008956602090082613E0FCA3E0FDA3E0FE13
:20434000A3E0FF90082D5A12008A6990082D50E4F0A304F0E4FFFE1202E6A21202E5CC9065
:20436000082601E0FCA3E0FD6F7002EC6E601290082D9CECF0A3EDF090082D50E4F0A304B8
:20438000F07B097A25795F1202E5B87B097A2579B01202E5C290082603E0FEA3E0FF120245
:2043A000E69B90082D9CE07002A3E070041202D3E81202E2EFC004A905AA06AB079008268C
:2043C00003E0FEA3E0FF7C027D58120086B3EE3395E0FDFCD000EB2FFFEA3EFEE93DFDE833
:2043E0003CFC9008040612008A697E007F0122E4900835F9F0A3F090081D4AE0FEA3E0FF32
:20440000C3900835FAE09F900835F9E09E40032149887B097A1979EE90081AEDEBF0A3EA95
:20442000F0A3E9F02414F9E43AFA74111200869F1202E33F90081AEDE0FBA3E0FAA3E02437
:2044400004F9E43AFA120089AA90081AEDE0FBA3E0FAA3E0F974FC75F003120087F990088D
:204460001AEDE0FBA3E0FAA3E02402F9E43AFA74FC75F002120087F990081AEDE0FBA3E0BD
:20448000FAA3E0242AF9E43AFAE41200869F12028A941202E5FE90082D97E0FBA3E0FAA3A5
:2044A000E0C39404F9EA9400FAEE8FF0120087F990081781E0FBA3E0FAA3E02408F9E43A03
:2044C000FA900835F3EBF0A3EAF0A3E9F02428F9E43AFAA3EBF0A3EAF0A3E9F01202E30F74
:2044E000900835F6E0FBA3E0FAA3E0F9120089AA900835F7E475F004120087531202DF24CC
:20450000C003C002900835F6E0FBA3E0FAA3E0F8AC02AD03D002D00312008D557B817AB261
:2045200079D31200BA43900835F7EE8FF012008753900835F6E0FBA3E475F0011200876976
:20454000A9F0FA74201200869F900835F6E0FBA3E475F00112008769A9F0FA7420120086B1
:204560009F900835F9E475F00112008769FEE5F025E0FFEE33FE74242FF582741B3EF58311
:20458000759308E0FFA3E0900835FBCFF0A3EFF0900830567481F0A374B3F0A37404F09048
:2045A0000835FBE0FFA3E090083059CFF0A3EFF0900835F6E0FBA3E0FAA3E0F91200A4169C
:2045C000900835F7EE8FF012008753900835FBE0FCA3E0FDC394D0EC6480948740032147DD
:2045E00027ED64EA7003EC640360032146E2900835FAE025E0FF900835F9E033FE74242F9E
:20460000F582741B3EF583759308E0FCA3E0FDA3E0FEA3E0FF900835FF12008A69900835D1
:20462000FAE02402F0900835F9E03400F0C3900835FCE094E8FF900835FBE09403CFC39474
:2046400001CF9400FE90081BEF75F003EF12008A86EE75F003A42583F583759308E0F9A337
:20466000E0FAA3E090083056C9F0A3EAF0A3E9F0900835FFE0FCA3E0FDA3E0FEA3E0FF786A
:204680001812008967E490083059F0A3EFF0900835FFE0FCA3E0FDA3E0FEA3E0FF781012C4
:2046A000008967E49008305BF0A3EFF0900835FFE0FCA3E0FDA3E0FEA3E0FF78081200894B
:2046C00067E49008305DF0A3EFF0900835FFE0FCA3E0FDA3A3E0FEE49008305FF0A3CE211F
:2046E00048FCC3900835FCE094E8FF900835FBE09403CFC39401CF9400FE90081BEF75F0C1
:2047000003EF12008A86EE75F003A42583F583759308E0F9A3E0FAA3E090083056C9F0A308
:20472000EAF0A3E92148FC900835FBE0FCA3E0FDC394B8EC6480948B506CC3ED94D0FFECD1
:204740009407CFC39401CF9400FE90081D1375F003EF12008A86EE75F003A42583F5837566
:204760009308E0F9A3E0FAA3E090083056C9F0A3EAF0A3E9F0900835F9E475F0011200874C
:2047800069FEE5F025E0FFEE33FE74242FF582741B3EF583759308E0FFA3E090083059CFD5
:2047A000F0A3EF2148FC900835FBE0FCA3E0FDC394A0EC6480948F506CC3ED94B8FFEC94CD
:2047C0000BCFC39401CF9400FE90081D2575F003EF12008A86EE75F003A42583F5837593D1
:2047E00008E0F9A3E0FAA3E090083056C9F0A3EAF0A3E9F0900835F9E475F00112008769F6
:20480000FEE5F025E0FFEE33FE74242FF582741B3EF583759308E0FFA3E090083059CFF0CD
:20482000A3EF2148FC900835FBE0FCA3E0FD64A17003EC640F6010ED64A67003EC640F60ED
:2048400006BC0F47BDA744C3900835FCE094A0FF900835FBE0940FCFC39401CF9400FE9096
:20486000081B0E75F003EF12008A86EE75F003A42583F583759308E0F9A3E0FAA3E09008F3
:204880003056C9F0A3EAF0A3E98071C3900835FCE094A0FF900835FBE0940FCFC39401CFFF
:2048A0009400FE90081B0E75F003EF12008A86EE75F003A42583F583759308E0F9A3E0FAAC
:2048C000A3E090083056C9F0A3EAF0A3E9F0900835F9E475F00112008769FEE5F025E0FF9C
:2048E000EE33FE74242FF582741B3EF583759308E0FFA3E090083059CFF0A3EFF090083575
:20490000F6E0FBA3E0FAA3E0F91200A416900835F7EE8FF012008753900835F3A3E0FAA304
:20492000E0AE02FFA3A3E0FAA3E0C39FFFEA9E90081AF0F0A3EFF0900835F3E0FBA3E0FA30
:20494000A3E0F91202A7001202E625EF64014E700C1202E5FEAC06AD07E4FF800A1202E520
:20496000FEAC06AD077F011202D58C7F027E0012016904900835FDEEF0A3EFF0F47002EEE1
:20498000F460032143F78000900835FDE0FEA3E0FF229008064FE0FBA3E0FAA3E0F91200C6
:2049A000877FFFAEF0E5F06003214F22EF24FE7003214BFF147003214BFF147003214E783B
:2049C00024036003214F22900830567484F0A37444F0A37407F09008177BE0FBA3E0FAA337
:2049E000E0F91200A41690081AF0EEF0A3EFF0E490082F9EF0A3F090082F9EE0FEA3E0FF7F
:204A0000D39403EE648094804003214BB0EE6003214B0AEF14603F14606A147003214ABCF2
:204A200024036003214B0A90082F9CE4F0A37405F090082F997484F0A37444F0A374CEF0CB
:204A400090082F967484F0A37444F0A374DEF01202E5CC214AE890082F9CE4F0A37414F077
:204A600090082F997484F0A37444F0A374E5F090082F967484F0A37444F0A374F1F012021B
:204A8000E6A9802C90082F9CE4F0A37414F090082F997484F0A37444F0A374F5F090082F33
:204AA000967484F0A37445F0A37403F01202E6B0786E7C2F7D0912008D55804E90082F9C3C
:204AC000E4F0A37402F090082F997484F0A37445F0A37407F090082F967484F0A37445F0C6
:204AE000A37430F01202E61C90083059EEF0A3EFF0900830567484F0A37444F0A374E2F0AE
:204B00007B097A2F796E1200A4169008177BE0FBA3E0FAA3E0F990081AF0E0FEA3E0FFE9CC
:204B20002FF9EA3EFAC003C002C001900830567484F0A37445F0A37436F090082F99E0F91D
:204B4000A3E0FAA3E090083059C9F0A3EAF0A3E9F090082F96E0F9A3E0FAA3E09008305C28
:204B6000C9F0A3EAF0A3E9F0A37409F0A3742FF0A3746EF090082F9CE0FFA3E090083062D9
:204B8000CFF0A3EFF0D001D002D0031200A41690081AF1E02FF090081AF0E03EF090082F79
:204BA0009FE004F0700790082F9EE004F02149F79008177BE0FBA3E0FAA3E0F990081AF0D1
:204BC000E0FEA3E0FFE92FF9EA3EFA900830567484F0A37445F0A37494F01200A4169008F1
:204BE0001AF1E02FF090081AF0E03EF09008064FE0FBA3E0FAA3E0F9E475F002214F1C90D3
:204C0000082FA0E4F0A304F090082FA0E0FEA3E0FFD39403EE648094804003214E29EE7002
:204C20007EEF24FE602B14604C2402707290082F997484F0A37445F0A374BCF090082F96DE
:204C40007484F0A37445F0A374C7F01202E30F804690082F997484F0A37445F0A374CAF021
:204C600090082F967484F0A37445F0A374D6F01202E31F802290082F997484F0A37445F07A
:204C8000A374D9F090082F967484F0A37445F0A374E1F01202E32F90082F6A12008A6990CF
:204CA00008177BE0FBA3E0FAA3E0F990081AF0E0FEA3E0FFE92FF9EA3EFAC002C001900836
:204CC00030567484F0A37445F0A374E4F090082F99E0F9A3E0FAA3E090083059C9F0A3EA8F
:204CE000F0A3E9F0D001D0021200A41690081AF1E02FF090081AF0E03EF090082F9EE4F04E
:204D0000A304F01202E62EEF64014E9008177B7047E0FBA3E0FAA3E0F990081AF0E0FEA35A
:204D2000E0FFE92FF9EA3EFAC002C001900830567484F0A37446F0A37401F090082F96E046
:204D4000F9A3E0FAA3E090083059C9F0A3EAF0A3E9F0D001D0028076E0FBA3E0FAA3E0F91A
:204D600090081AF0E0FEA3E0FFE92FF9EA3EFAC003C002C001900830567484F0A37446F065
:204D8000A37432F090082F96E0F9A3E0FAA3E090083059C9F0A3EAF0A3E9F090082F9FE08B
:204DA00075F008A4FFC374209FF990082F6AE0FCA3E0FDA3E0FEA3E0FFA80112008967E4D5
:204DC0009008305CF0A3EFF0D001D002D0031200A41690081AF1E02FF090081AF0E03EF0A9
:204DE00090082F9FE004F0700790082F9EE004F0D390082F9FE0940490082F9EE06480945B
:204E0000805003214D0390081AF1E024FEF090081AF0E034FFF090082FA1E004F0700790D1
:204E2000082FA0E004F0214C089008177BE0FBA3E0FAA3E0F990081AF0E0FEA3E0FFE92F3A
:204E4000F9EA3EFA900830567484F0A37446F0A3746CF01200A41690081AF1E02FF090086B
:204E60001AF0E03EF09008064FE0FBA3E0FAA3E0F9E475F004214F1C900830567484F0A3D7
:204E80007447F0A37405F09008177BE0FBA3E0FAA3E0F91200A41690081AF0EEF0A3EFF08F
:204EA0009008177BE0FBA3E0FAA3E02FF9EA3EFA900830567484F0A37447F0A374FCF0123A
:204EC00000A41690081AF1E02FF090081AF0E03EF09008177BE0FBA3E0FAA3E0F990081A16
:204EE000F0E0FEA3E0FFE92FF9EA3EFA900830567484F0A37448F0A3749FF01200A41690D8
:204F0000081AF1E02FF090081AF0E03EF09008064FE0FBA3E0FAA3E0F9E4F5F0120087F9B3
:204F200080037F01227F002290082DA0E0FEA3E0FF90082D55E02FFF90082D54E03EFED3B6
:204F4000EF9400EE6480948050032151421202E35FEF5402FFE4FDFCEF70032151429008BC
:204F60002D90E02401FF90082D8FE03400FE90082D5FE02FFF90082D5EE03E9008377DF05B
:204F8000A3EFF090082D90E02401FF90082D8FE03400FE90082D5FE02FFF90082D5EE03E5D
:204FA000FE90082D55E02FFF90082D54E03EFE90082DA1E02FFF90082DA0E03EFEC3900846
:204FC000377EE09FEE6480F89008377DE06480984003215142A3E0C39401FF7B097A3779AC
:204FE0007F120235B29008377FE0C4F854F0C8A3E0C4540F48540F6407600321508B90088A
:205000002D90E004FF90082D5FE02FFF9008377EE0C39FFF74017E00A807088005C333CE3D
:2050200033CED8F9FF90081BECE0FDEF5D700321512F9008377EE02401FF9008377DE03412
:2050400000FE3395E0FDFC90083A0112008A69E490083A05F0A3F07FD47E07120278609047
:20506000081BECE0FF90082D90E004FE90082D5FE02EFE9008377EE0C39EFE7401A8060824
:205080008002C333D8FCF45F21512A9008377FE0C4F854F0C8A3E0C4540F48540F640670B0
:2050A0000321512F90082D90E004FF90082D5FE02FFF9008377EE0C39FFF74017E00A807B2
:2050C000088005C333CE33CED8F9FF90081BECE0FDEF5D705A9008377EE02401FF900837FC
:2050E0007DE03400FE3395E0FDFC90083A0112008A69E490083A05F0A3F07FD37E0712027F
:20510000786090081BECE0FF90082D90E004FE90082D5FE02EFE9008377EE0C39EFE7401D1
:20512000A806088002C333D8FC4F90081BECF09008377EE004F070079008377DE004F021B6
:205140004F8390081AF2E475F00112008753FED3E5F0940AEE648094804010E490081AF2A1
:20516000F0A3F01201B81F1201A0E81202E37FEF5401FFE4FEFDFCEF602F90081B23E0B4AB
:20518000012790081C10E07020FF90083A0112008A69E490083A05F0A3F07FA17E0F1202DD
:2051A000786090081C107401F090081B23E060032154B590083779F0A3F090083779E0FEBA
:2051C000A3E0FFC39418EE648094804003215443EF25E0FFEE33FE74482FF582741E3EF5C4
:2051E00083759308E090083777F074492FF582741E3EF583759308E090083778F01202E33D
:205200007FEF5402FFE4FEFDFCEF700321530090083778E0FF7401A807088005C333CE334C
:20522000CED8F9FF90083777E025E024ACF582E4341DF583759308E05EFEA3E05F4E60389D
:205240009008377AE024F8F582E4341BF583759308E070249008377AE09008377912027866
:20526000409008377AE024F8F582E4341BF5837593087401F021530090083778E0FF740103
:205280007E00A807088005C333CE33CED8F9FF90083777E025E024ACF582E4341DF583752B
:2052A0009308E05EFEA3E05F4E70559008377AE024F8F582E4341BF583759308E0B40140D6
:2052C0009008377AE02401FF90083779E03400FE3395E0FDFC90083A0112008A69E4900832
:2052E0003A05F0A3F07FA37E0F120278609008377AE024F8F582E4341BF583759308E4F006
:205300001202E37FEF5404FFE4FEFDFCEF700321539890083778E0FF7401A807088005C3EE
:2053200033CE33CED8F9FF90083777E025E0246CF582E4341FF583759308E05EFEA3E05F8C
:205340004E60559008377AE024F4F582E4341AF583759308E070419008377AE02401FF906A
:20536000083779E03400FE3395E0FDFC90083A0112008A69E490083A05F0A3F07FA47E0FFC
:20538000120278609008377AE024F4F582E4341AF5837593087401F01202E37FEF5408FF8A
:2053A000E4FEFDFCEF700321543090083778E0FF7401A807088005C333CE33CED8F9FF900F
:2053C000083777E025E024F0F582E4341EF583759308E05EFEA3E05F4E60559008377AE09F
:2053E0002432F582E4341DF583759308E070419008377AE02401FF90083779E03400FE33B8
:2054000095E0FDFC90083A0112008A69E490083A05F0A3F07FA57E0F120278609008377A22
:20542000E02432F582E4341DF5837593087401F09008377AE004F0700790083779E004F0ED
:205440002151BA1202E37FEF5410FFE4FEFDFCEF60631202D074BF012A90081D31E0702330
:20546000FFFEFDFC90083A0112008A69E490083A05F0A3F07FA67E0F1202786090081D319C
:205480007401F01202D074EF702B90081D31E0B40123E4FFFEFDFC90083A0112008A69E491
:2054A00090083A05F0A3F07FA77E0F12027860E490081D31F022E49008335EF0A3F09008EF
:2054C000064FE0FBA3E0FAA3E0F91200877FFFAEF0E5F060032159F4EF24FE7003215594BA
:2054E0001470032159A3240260032159F4900830567484F0A3745FF0A374DBF09008177B99
:20550000E0FBA3E0FAA3E0F91200A41690081AF0EEF0A3EFF090083356E4F0A304F09008C5
:20552000177BE0FBA3E0FAA3E0F990081AF0E0FEA3E0FFE92FF9EA3EFA900830567484F0CA
:20554000A37461F0A3741BF01200A41690081AF1E02FF090081AF0E03EF090083357E0049D
:20556000F0700790083356E004F0D390083357E0940290083356E06480948040A1900806EC
:205580004FE0FBA3E0FAA3E0F9E475F002120087F97F002290080660E0FBA3E0FAA3E0F998
:2055A0001200877FC39401FEE5F0940090083356F0A3CEF0C390082D69E09401FF90082D78
:2055C00068E09400FEC390083357E09FEE6480F890083356E0648098400321597BA3E0FF8C
:2055E0001202E0689008335CEEF0A3EFF090083356E07002A3E0601A90083357E0C39401FE
:20560000FF1202E0689008335CE06E7003A3E06F60119008335CE0FEA3E0FF7D0A7C001248
:2056200002B3089008177BE0FBA3E0FAA3E0F990081AF0E0FEA3E0FFE92FF9EA3EFA9008E2
:2056400030567484F0A37461F0A37492F01200A41690081AF1E02FF090081AF0E03EF0902D
:20566000083358E4F0A304F090083358E0FEA3E0FFD39402EE648094804003215905900800
:205680003356E0FDA3E09008335ACDF0A3EDF0EF64024E60032157F8A3E0FEA3E0FF120232
:2056A000D9B1EFC313FF90083357E02FFE90083356E034009008335AF0A3CEF0E0FF1202CF
:2056C000E0689008335CEEF0A3EFF090082D90E02401FF90082D8FE03400FE90082D5FE038
:2056E0002FFF90082D5EE03EFE90082D55E02FFF90082D54E03EFE90082DA1E02FFF9008D4
:205700002DA0E03ECFC39401CF9400FE9008335AE06E7003A3E06F601A9008335BE0C39467
:2057200001FF1202E0689008335CE06E7003A3E06F60769008177BE0FBA3E0FAA3E0F990CF
:20574000081AF0E0FEA3E0FFE92FF9EA3EFA900830567484F0A37461F0A37499F01200A4E0
:205760001690081AF1E02FF090081AF0E03EF090083356E0FEA3E0FF9008335AE0FCA3E0BC
:20578000FDB50709ECB50605ED24028003ED2401FFE43CF990080660E0FBA3E0FAA3E0C939
:2057A0008FF0120087F97F00229008335BE004FF1202E0689008335CE06E7003A3E06F6098
:2057C000099008335EE4F0A304F090082D68E0FEA3E0FFC39402FDEE9400FC9008335AE0C6
:2057E000B50415A3E0B50510C3EF9401FFEE940090083356F0A3EFF09008335AE0FEA3E0AD
:20580000FF9008278A7409F0A37433F0A37466F0A37409F0A37433F0A3746AF0A37409F061
:20582000A37433F0A3746EF07B097A3379621202376A9008177BE0FBA3E0FAA3E0F9900862
:205840001AF0E0FEA3E0FFE92FF9EA3EFAC003C002C001900830567484F0A37461F0A374E0
:20586000B0F09008335AE0FEA3E0FF90083059EEF0A3EFF02401FFE43EA3F0A3EFF090088F
:205880003366E0FCA3E0FDA3E0FEA3E0FF9008305D12008A699008336EE0FCA3E0FDA3E0CE
:2058A000FEA3E0FF9008306112008A6990083362E0FCA3E0FDA3E0FEA3E0FF90083065126F
:2058C000008A699008336AE0FCA3E0FDA3E0FEA3E0FF9008306912008A69D001D002D00395
:2058E0001200A41690081AF1E02FF090081AF0E03EF090083359E004F0700790083358E018
:2059000004F02156689008335EE07002A3E0701690080660E0FBA3E0FAA3E0F9E475F00114
:20592000120087CD802C9008335BE02402FF9008335AE03400F990080660E0FBA3E0FAA3FF
:20594000E0C98FF0120087F9E49008335EF0A3F0FF2290080660E0FBA3E0FAA3E0F91200F8
:20596000877F54037002FF2290083357E004F0700790083356E004F02155B49008064FE0DE
:20598000FBA3E0FAA3E0F9E475F003120087F990080660E0FBA3E0FAA3E0F9E475F0011207
:2059A0000087F99008177BE0FBA3E0FAA3E0F990081AF0E0FEA3E0FFE92FF9EA3EFA90089C
:2059C00030567484F0A37462F0A37409F01200A41690081AF1E02FF090081AF0E03EF09032
:2059E00008064FE0FBA3E0FAA3E0F9E4F5F0120087F980037F01227F002290082FE6EEF0CA
:205A0000A3EFF0E490083014F0A3F07B097A2F79F41202DB5490080660E0FBA3E0FAA3E00B
:205A2000F91200877FC39401FEE5F0940090082FE8F0A3CEF0C390082D69E09401FF900899
:205A40002D68E09400FEC390082FE9E09F90082FE8E09E4003215F21A3E0FF1202E06890CE
:205A6000082FF0EEF0A3EFF090082FE8E07002A3E0601A90082FE9E0C39401FF1202E0685E
:205A800090082FF0E06E7003A3E06F601F90082FF2E4F0A3740AF090082FF0E0FEA3E0FF68
:205AA0007D0A7C001202B3081202A3D29008177BE0FBA3E0FAA3E0F990081AF0E0FEA3E08A
:205AC000FFE92FF9EA3EFA900830567484F0A3741DF0A374CFF01200A41690081AF1E02F16
:205AE000F090081AF0E03EF090082FEAE4F0A304F090082FEAE0FEA3E0FFD39402EE9400EE
:205B00004003215EA990082FE8E0FDA3E090082FECCDF0A3EDF0EF64024E6003215C709098
:205B2000082FF0E0FEA3E0FF1202D9B1EFC313FF90082FE9E02FFE90082FE8E03400900864
:205B40002FECF0A3CEF0E0FF1202E06890082FF0EEF0A3EFF0C390082D69E09401FF90088A
:205B60002D68E09400FE90082FECE06E7003A3E06F601D90082FEDE0C39401FF1202E068F4
:205B800090082FF0E06E7003A3E06F7003215C219008177BE0FBA3E0FAA3E0F990081AF0EA
:205BA000E0FEA3E0FFE92FF9EA3EFA900830567484F0A3741DF0A374D6F090082FF2E0FEB4
:205BC000A3E0FF7C007D021200871B90083059EEF0A3EFF01200A41690081AF1E02FF09015
:205BE000081AF0E03EF090082FE8E0FEA3E0FF90082FECE0FCA3E0FDB50709ECB50605ED09
:205C000024028003ED2401FFE43CF990080660E0FBA3E0FAA3E0C98FF0120087F9E4FEFF1D
:205C20002290082FEDE004FF1202E06890082FF0E06E7003A3E06F600990083014E4F0A329
:205C400004F090082D68E0FEA3E0FFC39402FDEE9400FC90082FECE0B50415A3E0B5051041
:205C6000C3EF9401FFEE940090082FE8F0A3EFF090082FEDE0FF7B097A307916120235B2F0
:205C800090082FF0E07004A3E06404703190082FEDE0FF1202DA75EF4E70119008301A7463
:205CA00084F0A3741DF0A374EEF0804390083016E0C4F854F0C8A3E0C4540F4880059008FF
:205CC0003017E0540F90082F5275F00312008A86E475F003A42583F583759308E0F9A3E01B
:205CE000FAA3E09008301AC9F0A3EAF0A3E9F090082FE6E07004A3E064019008177B7043CD
:205D0000E0FBA3E0FAA3E0F990081AF0E0FEA3E0FFE92FF9EA3EFA900830567484F0A3745D
:205D20001DF0A374FAF090082FECE0FEA3E0FF90083059EEF0A3EFF02401FFE43EA3F0A345
:205D4000EF803CE0FBA3E0FAA3E0F990081AF0E0FEA3E0FFE92FF9EA3EFA90083056748479
:205D6000F0A3741EF0A3742EF090082FEDE02401FE90082FECE0340090083059F0A3CEF0E9
:205D80001200A41690081AF1E02FF090081AF0E03EF09008177BE0FBA3E0FAA3E0F990084F
:205DA0001AF0E0FEA3E0FFE92FF9EA3EFAC003C002C001900830567484F0A3741EF0A374BE
:205DC00049F09008301AE0F9A3E0FAA3E090083059C9F0A3EAF0A3E9F090083016E0FCA39F
:205DE000E0FDEC540190082F4675F00312008A86E475F003A42583F583759308E0F9A3E072
:205E0000FAA3E09008305CC9F0A3EAF0A3E9F090082FECE0FEA3E024F4F582742F3EF58333
:205E2000759308E075F003A42440F582E4342FF583759308E0F9A3E0FAA3E09008305FC9F3
:205E4000F0A3EAF0A3E9F0ECC4F854F0C8EDC4540F48540F90082F5275F00312008A86E45F
:205E600075F003A42583F583759308E0F9A3E0FAA3E090083062C9F0A3EAF0A3E9F0D00160
:205E8000D002D0031200A41690081AF1E02FF090081AF0E03EF090082FEBE004F0700790B2
:205EA000082FEAE004F0215AF190083014E07002A3E0701690080660E0FBA3E0FAA3E0F978
:205EC000E475F001120087CD802D90082FEDE02402FF90082FECE03400F990080660E0FB13
:205EE000A3E0FAA3E0C98FF0120087F9E490083014F0A3F0FEFF2290080660E0FBA3E0FA10
:205F0000A3E0F91200877F54037003FEFF2290082FE9E004F0700790082FE8E004F0215A0B
:205F20003590080660E0FBA3E0FAA3E0F9E475F001120087F97E007F01221202E33F900890
:205F400034D812008A697E007F807D007B097A1C799312008F137E007F807D007B097A1C48
:205F6000791312008F13E4FFFEFDFC900834D8E0F8A3E0F9A3E0FAA3E0FBC3120089566000
:205F8000291202E34FEF5401FFE4FEFDFCEF601AE4FF90083A0112008A69E490083A05F0A5
:205FA000A3F07FE97E03120278601202E35F900834D412008A691202E6D990081B0CEEF00E
:205FC000A3EFF090082DA0E0FEA3E0FF90082D55E02FFF90082D54E03EFED3EF9400EE6475
:205FE00080948050032161DE1202E35FEF5402FFE4FEFDFCEF70032161DE90082D90E024CA
:2060000001FF90082D8FE03400FE90082D5FE02FFF90082D5EE03E900834E2F0A3EFF090F7
:20602000082D90E02401FF90082D8FE03400FE90082D5FE02FFF90082D5EE03EFE90082DFB
:2060400055E02FFF90082D54E03EFE90082DA1E02FFF90082DA0E03EFEC3900834E3E09FC2
:20606000EE6480F8900834E2E064809840032161DEA3E0C39401FF7B097A3479E4120235F7
:20608000B2900834E4E0C4F854F0C8A3E0C4540F48540F6407600321612790082D90E004F1
:2060A000FF90082D5FE02FFF900834E3E0C39FFF74017E00A807088005C333CE33CED8F9FA
:2060C000FF90081BECE0FDEF5D70032161CB900834E3E02401FF900834E2E03400FE3395FE
:2060E000E0FDFC90083A0112008A69E490083A05F0A3F07FD47E071202786090081BECE06E
:20610000FF90082D90E004FE90082D5FE02EFE900834E3E0C39EFE7401A806088002C33388
:20612000D8FCF45F2161C6900834E4E0C4F854F0C8A3E0C4540F48540F640670032161CB19
:2061400090082D90E004FF90082D5FE02FFF900834E3E0C39FFF74017E00A807088005C3F3
:2061600033CE33CED8F9FF90081BECE0FDEF5D705A900834E3E02401FF900834E2E0340046
:20618000FE3395E0FDFC90083A0112008A69E490083A05F0A3F07FD37E07120278609008EF
:2061A0001BECE0FF90082D90E004FE90082D5FE02EFE900834E3E0C39EFE7401A8060880F9
:2061C00002C333D8FC4F90081BECF0900834E3E004F07007900834E2E004F021601F1202E5
:2061E000D36A1202E37FEF5401FFE4FEFDFCEF602990081B23E0B40121E4FF90083A011202
:20620000008A69E490083A05F0A3F07FA17E0F1202786090081C107401F090081B23E06075
:206220000321642D900834DEF0A3F0900834DFE0FF1201089B900834DFE025E0FF900834E1
:20624000DEE033FE74482FF582741E3EF583759308E0900834DCF074492FF582741E3EF5F5
:2062600083759308E0900834DDF01202E37FEF5402FFE4FEFDFCEF6052900834DDE0FF74E0
:2062800001A807088005C333CE33CED8F9FF900834DCE025E024ACF582E4341DF5837593A3
:2062A00008E05EFEA3E05F4E6021900834DFE0900834DE12027840900834DFE024F8F582CA
:2062C000E4341BF5837593087401F01202E37FEF5404FFE4FEFDFCEF6072900834DDE0FFBE
:2062E0007401A807088005C333CE33CED8F9FF900834DCE025E0246CF582E4341FF58375A0
:206300009308E05EFEA3E05F4E6041900834DFE02401FF900834DEE03400FE3395E0FDFCC9
:2063200090083A0112008A69E490083A05F0A3F07FA47E0F12027860900834DFE024F4F513
:2063400082E4341AF5837593087401F01202E37FEF5408FFE4FEFDFCEF6072900834DDE0B7
:20636000FF7401A807088005C333CE33CED8F9FF900834DCE025E024F0F582E4341EF58312
:20638000759308E05EFEA3E05F4E6041900834DFE02401FF900834DEE03400FE3395E0FDD0
:2063A000FC90083A0112008A69E490083A05F0A3F07FA57E0F12027860900834DFE024324D
:2063C000F582E4341DF5837593087401F0900834DFE004F07007900834DEE004F0C3900855
:2063E00034DFE09418900834DEE064809480500321622B1202E37FEF5410FFE4FEFDFCEFE9
:20640000602B1202D074BF0124E4FFFEFDFC90083A0112008A69E490083A05F0A3F07FA6A0
:206420007E0F1202786090081D317401F022900833DB12008A69900833DFEBF0A3EAF0A326
:20644000E9F01202E32F900833ED12008A691202E31F900833F112008A69900833F1E0FC11
:20646000A3E0FDA3E0FEA3E0FF900833EDE0F8A3E0F9A3E0FAA3E05FFFEA5EFEE95DFDE8BE
:206480005CFCC004C005C006AB07A3E0FCA3E0FDA3E0FEA3E0FF900833DBE0F8A3E0F9A304
:2064A000E0FAA3E05FFFEA5EFEE95DFDE85CFCD002D001D000C3120089566017900833ED02
:2064C000E0FCA3E0FDA3E0FEA3E0FF900833DB12008A69E4900833E9F0A3F0900833E9E003
:2064E000FEA3E0FFC39408EE6480948040032165AD90082DFA75F00AEF12008A86EE75F0CF
:206500000AA42583F583759308E0FCA3E0FDA3E0FEA3E0FF900833DBE0F8A3E0F9A3E0FAC7
:20652000A3E0FBC3120089567070900833E9E0FEA3E090082DFA75F00A12008A86EE75F091
:206540000AA42583F583759308E0FCA3E0FDA3E0FEA3E0FFE4FBFAF9F8C312008956603AE6
:20656000900833E9E0FEA3E0FF7C007D0A120086B374FE2FF9742D3EFA7B09C003C00290AD
:206580000833DFE0FBA3E0FAA3E0F8AC02AD03D002D0037E007F062168F7900833EAE004EF
:2065A000F07007900833E9E004F02164DB90081AF0E0FEA3E0FF78007C077D0990082D97AD
:2065C000E0FBA3E0FAA3E0F9120085D090081AF0E0FFA3E0900833EBCFF0A3EFF090082EBF
:2065E0004CE4F0A3743CF0900833E9E4F0A304F090081784E0FBA3E0FAA3E0F9900833E661
:20660000EBF0A3EAF0A3E9F0E475F001120087F9900833E6E0FBA3E0FAA3E02402F9E43A01
:20662000FA740875F000120087F9900833E6E0FBA3E0FAA3E02404F9E43AFA740675F00445
:20664000120087F9900833E6E0FBA3E0FAA3E02406F9E43AFAE475F001120087F99008333A
:20666000E6E0FBA3E0FAA3E02408F9E43AFA1202DBFC1202E30F900833E6E0FBA3E0FAA37F
:20668000E0240EF9E43AFA120089AA7E007F067D00900833E6E0FBA3E0FAA3E02412F9E473
:2066A0003AFA12008F13900833DBE0FCA3E0FDA3E0FEA3E0FF900833E6E0FBA3E0FAA3E061
:2066C0002418F9E43AFA120089AA90081778E0FBA3E0FAA3E0240CF9E43AFA740875F006FE
:2066E000120087F97E007F067DFF90081778E0FBA3E0FAA3E0F912008F13900833E6E0FB4E
:20670000A3E0FAA3E02408F9E43AFAC003C002C00190081778E0FBA3E0FAA3E02406F9E4ED
:206720003AA801FCAD03D001D002D0037E007F06120085D090082D97E0FBA3E0FAA3E0F9BA
:206740007D2A7C001201B1BC12028A94900833EAE004F07007900833E9E004F0D39008333E
:20676000EAE09403900833E9E06480948050032165F01202E2EFEF240AFFE43EFEE43DFD24
:20678000E43CFC900833E212008A691202E2EF900833E2E0F8A3E0F9A3E0FAA3E0FBD31265
:2067A00000895650032168FF7B097A1A79F01202026E90082D97EBF0A3EAF0A3E9F0900852
:2067C0002D97E0FBA3E0FAA3E04A4B60BE90082D97E0FBA3E0FAA3E0F990081778EBF0A392
:2067E000EAF0A3E9F0240CF9E43AFA1200877F64067004E5F06408600321687D900817783B
:20680000E0FBA3E0FAA3E0240EF9E43AFA900833E6EBF0A3EAF0A3E9F01202E30F90083304
:20682000E6E0FBA3E0FAA3E02418F9E43AFA120089E2C3120089567044900833E6E0FBA336
:20684000E0FAA3E02406F9E43AFA1200877F640245F07029900833E6A3E0FAA3E0240EF978
:20686000E43AFA1200898D900833DBE0F8A3E0F9A3E0FAA3E0FBC31200895660071202E7CD
:206880004F21678B900833DBE0FCA3E0FDA3E0FEA3E0FF90081778E0FBA3E0FAA3E0240665
:2068A000F9E43AFA120233F3900833EBE0FFA3E090081AF0CFF0A3EFF090081778E0FBA3ED
:2068C000E0FAA3E02406F9E43AFA78007C077D097E007F06120085D090081AF0E0FEA3E032
:2068E000FF90082D97E0FBA3E0FAA3E0F8AC02AD037B097A077900120085D0E4FEFF227EA6
:20690000FF7FFF2290083546EEF0A3EFF064014E701B74FFFFFEFDFC90081AEDE0FBA3E0C1
:20692000FAA3E02404F9E43AFA120089AA90081AEDE0FBA3E0FAA3E02414F9E43AFA120087
:20694000864E147003216B1724FB7003216A0124F56003216A1B90081AEDE0FBA3E0FAA35F
:20696000E0F91200877FFF90081781E0FBA3E0FAA3E0F9E5F08FF0120087F990081AEDE0BE
:20698000FBA3E0FAA3E02402F9E43AFA1200877FFF90081781E0FBA3E0FAA3E02402F9E4A0
:2069A0003AFAE5F08FF0120087F990081AF1E02408F090081AF0E03400F0E0FEA3E0FF9088
:2069C000081781E0FBA3E0FAA3E02404F9E43AFAEE8FF0120087F990081781E0FBA3E0FA7C
:2069E000A3E02406F9E43AFAE4F5F0120087F990081AF1E02414F090081AF0E03400F080AD
:206A00001D9008177EE0FBA3E0FAA3E02410F9E43AFAE4F5F0120087F98003216DAAC390A3
:206A2000081AF1E09414FE90081AF0E0940090083548F0A3CEF01202E30F9008354A120012
:206A40008A6990081AEDE0FBA3E0FAA3E02404F9E43AFA1200898D9008354E12008A69E464
:206A600090083552F090081AEDE0FBA3E0FAA3E02414F9E43AFA1200864E90083553F090BE
:206A8000083548E0FCA3E0FD90083554ECF0A3EDF090081784E0FBA3E0FAA3E02414F9E475
:206AA0003AFA120253BE90083556EEF0A3EFF07B097A35794A7D0E7C00120253BEEFF4FFF6
:206AC000EEF490083556F0A3EFF090081AEDE0FBA3E0FAA3E02414F9E43AFA1200864E9006
:206AE000083556B41114E0FEA3E0FF90081781E0FBA3E0FAA3E024068012E0FEA3E0FF9013
:206B000008177EE0FBA3E0FAA3E02410F9E43AFAEE8FF0120087F91202E30F90081784E0A0
:206B2000FBA3E0FAA3E0240CF9E43AFA120089AA90081AEDE0FBA3E0FAA3E02404F9E43A1B
:206B4000FA1200898D90081784E0FBA3E0FAA3E02410F9E43AFA120089AA90081AEDE0FB01
:206B6000A3E0FAA3E02414F9E43AFA1200864EFF90081784E0FBA3E0FAA3E02409F9E43A95
:206B8000FAEF1200869F90081784E0FBA3E0FAA3E0F974451200869F90081784E0FBA3E04D
:206BA000FAA3E02401F9E43AFAE41200869F900819E1E0FEA3E08EF012008B6B6BC800005B
:206BC0006BFCFFFF00006C1190081784E0FBA3E0FAA3E02406F9E43AFAE475F0A112008707
:206BE000F974FF900819E1F0A3F07E027F587D007B097A17798912008F13802F9008178493
:206C0000E0FBA3E0FAA3E02406F9E43AFA7440801390081784E0FBA3E0FAA3E02406F9E402
:206C20003AFA742075F000120087F91202E6B790081784E0FBA3E0FAA3E02408F9E43AFA99
:206C4000EF1200869F90081AF0E0FEA3E0FF90081784E0FBA3E0FAA3E02402F9E43AFAEED9
:206C60008FF0120087F990081787E475F00112008753FE90081784E0FBA3E0FAA3E0240463
:206C8000F9E43AFAEE120087F990081784E0FBA3E0FAA3E0240AF9E43AFAE4F5F0120087B4
:206CA000F9120253AEEFF4FFEEF4FE90081784E0FBA3E0FAA3E0240AF9E43AFAEE8FF01238
:206CC0000087F990081AF1E0240EF090081AF0E03400F090081778E0FBA3E0FAA3E0240CB7
:206CE000F9E43AFA740875F000120087F990081778E0FBA3E0FAA3E02406F9E43AFA1202BF
:206D0000DBFC90083546E07004A3E06401703090081778E0FBA3E0FAA3E0F8AC02AD037BDA
:206D2000097A1979E47E007F06120085D090082D97E0FBA3E0FAA3E0F91202BF6F807090FE
:206D4000083546E07004A3E06404703378487C357D097B817A90798CFE7F06120085D09052
:206D6000081778E0FBA3E0FAA3E0F8AC02AD037B097A3579487E007F06120085D0803090AD
:206D8000081AEDE0FBA3E0FAA3E02404F9E43AFA1200898D90081778E0FBA3E0FAA3E0F9AD
:206DA0001201642EBEFF08BFFF057EFF7FFF221202750A90082D97E0FBA3E0FAA3E0F99036
:206DC000081AF0E0FCA3E0FD1201B1BCE4FEFF2290081781E0FBA3E0FAA3E02408F9E43A74
:206DE000FA900836D5EBF0A3EAF0A3E9F090083A127481F0A374B8F0A374F1F0A3E4F0A388
:206E00007410F01202B7AEEF706F900837267409F0A37436F0A374DAF0A37409F0A37436DA
:206E2000F0A374DCF0A37409F0A37436F0A374DEF07B097A3679D81202C69D900836DAE0C9
:206E40007002A3E060032171E2900836DCE07002A3E060032171E2D3900836DFE09432905A
:206E60000836DEE06480948040032171E290083BCFE4F0A304F021721790083A127481F0E7
:206E8000A374B8F0A374FAF0A3E4F0A37410F0900836D5E0FBA3E0FAA3E0F91202B7AEEFC5
:206EA000700321721790083A127481F0A374B9F0A37402F0A3E4F0A37409F0900836D5E019
:206EC000FBA3E0FAA3E0F91202B7AEEF705090083BCFE07004A3E0640160032171E2900849
:206EE00036D5E0FBA3E0FAA3E0240AF9E43AFA7D087C00120253BEEFF47002EEF46003218C
:206F000071E2900836D5E0FBA3E0FAA3E0240AF9E43AFA1202E2091202D4622172179008D6
:206F20003A127481F0A374B9F0A3740CF0A3E4F0A37409F0900836D5E0FBA3E0FAA3E0F94F
:206F40001202B7AEEF701790083BCFE07004A3E0640160032171E21202D8832172179008DC
:206F60003A127481F0A374B9F0A37416F0A3E4F0A37407F0900836D5E0FBA3E0FAA3E0F907
:206F80001202B7AEEF700A90083BCFF0A3F021721790083A127481F0A374B9F0A3741EF092
:206FA000A3E4F0A37408F0900836D5E0FBA3E0FAA3E0F91202B7AEEF705A9008305674818F
:206FC000F0A374B9F0A37427F0A37481F0A374B9F0A3742AF0900836D5E0FBA3E0FAA3E0DC
:206FE000F91200A41690081AF0EEF0A3EFF0900836D5E0FBA3E0FAA3E02FF9EA3EFA1202EE
:20700000DBFC90081AF1E02406F090081AF0E0340021724A90083A127481F0A374B9F0A33D
:20702000742EF0A3E4F0A3740AF0900836D5E0FBA3E0FAA3E0F91202B7AEEF60032170E182
:20704000900830567481F0A374B9F0A37427F0A37481F0A374B9F0A37439F0900836D5E034
:20706000FBA3E0FAA3E0F91200A41690081AF0EEF0A3EFF01202DF41900836E0EBF0A3EA04
:20708000F0A3E9F0900836D5E0FBA3E0FAA3E0F990081AF0E0FEA3E0FFE92FF9EA3EFAC018
:2070A00002C001900830567481F0A374B9F0A37427F0900836E0E0F9A3E0FAA3E0900830CD
:2070C00059C9F0A3EAF0A3E9F0D001D0021200A41690081AF1E02FF090081AF0E03E217241
:2070E0004A90083A127481F0A374B9F0A37440F0A3E4F0A3740AF0900836D5E0FBA3E0FAF3
:20710000A3E0F91202B7AEEF60032171AE900830567481F0A374B9F0A37427F0A37481F06F
:20712000A374B9F0A3744BF0900836D5E0FBA3E0FAA3E0F91200A41690081AF0EEF0A3EFE8
:20714000F01202DF5E900836E0EBF0A3EAF0A3E9F0900836D5E0FBA3E0FAA3E0F990081A43
:20716000F0E0FEA3E0FFE92FF9EA3EFAC002C001900830567481F0A374B9F0A37427F09088
:207180000836E0E0F9A3E0FAA3E090083059C9F0A3EAF0A3E9F0D001D0021200A41690081E
:2071A0001AF1E02FF090081AF0E03E21724A90083A127481F0A374B9F0A37452F0A3E4F0CF
:2071C000A37405F0900836D5E0FBA3E0FAA3E0F91202B7AEEF700B90083BD1E07002A3E0D0
:2071E0007035900830567481F0A374B9F0A37427F0A37481F0A374B9F0A37458F090083684
:20720000D5E0FBA3E0FAA3E0F91200A41690081AF0EEF0A3EF8033900830567481F0A3741A
:20722000B9F0A37427F0A37481F0A374B9F0A3745DF0900836D5E0FBA3E0FAA3E0F9120042
:20724000A41690081AF0EEF0A3EFF07F027E001201690422E4FFFEFDFC900835E512008AA9
:2072600069E4FFFEFDFC900835E912008A69E4FFFEFDFC900835ED12008A69E490082D646A
:20728000F0A3F090082D6AF0A3F090082D52F0A3F090082D9AF0A3F090082D50F0A3F09015
:2072A000082D8DF0A3F090082D9CF0A3F0FFFEFDFC90082D5612008A69E4FFFEFDFC90081D
:2072C0002D6C12008A69E4FFFEFDFC90082D5A12008A69E490082D70F0A3F090082D75F04C
:2072E000A3F090082D74F01202E1381202E73E1202E74A7B817AB979EE900830567403F00C
:20730000A374FCF01200A41C1202CB1A120204D11202AA001202C0561202E0A81202602896
:207320001202E3AF1202CA757B817ABA790C1200A41CE490082D64F0A3F01202E2EFEF2445
:2073400014FFE43EFEE43DFDE43CFC900835E512008A691202E2EF900835E5E0F8A3E0F91E
:20736000A3E0FAA3E0FBD31200895650E612015F3A1202BB2C1202E2EFEF241EFFE43EFE3C
:20738000E43DFDE43CFC90082D9312008A691202E2EF90082D93E0F8A3E0F9A3E0FAA3E0C5
:2073A000FBD312008956503990082D77E0640170301202E57ABF010C1202C49CE490082D08
:2073C00077F0801D7B817ABA791CE4FFFEFDFC1201DC27E490082D77F0120212F81202E7CB
:2073E0003B1202E2EF90082D60E0F8A3E0F9A3E0FAA3E0FBD31200895640032174C1900804
:207400002D67E0FF1201089B90082D78EFF090081B23E06006E490082D78F090082D67E0EE
:20742000FF90082D78E0FD1202D2A390082D66E0FEA3E0FF7C007D0C1200871BED4C7004B9
:207440001202C5D390082D67E004F0700790082D66E004F090082D66E0FEA3E0FF7C007D86
:20746000181200871B90082D66ECF0A3EDF01202E2EFEF2402FFE43EFEE43DFDE43CFC90D6
:20748000082D6012008A6990082D66E0FEA3E0FF7C007D181200871BED4C70257B097A2D09
:2074A000799E1202E712C390082D9FE094D690082D9EE0941040061202E74780041202E749
:2074C0004A90080658E0B4022A9008329DE4F0A37402F01202E2EF90080406E0F8A3E0F98D
:2074E000A3E0FAA3E0FBD31200895650101202E0A8800A9008329DE4F0A3740AF07B097AFD
:207500001A79F01202026E90082D97EBF0A3EAF0A3E9F090082D97E0FBA3E0FAA3E04A4B68
:20752000605890082D97A3A3E0F91200864E6401703F1202D5C5900835F1EEF0A3EFF04E04
:20754000701B90082D97E0FBA3E0FAA3E0F990081AF0E0FCA3E0FD1201B1BC800D90083598
:20756000F1E07004A3E0640270071200800B21738E7F011200BA6421764CE490082D70F00B
:20758000A3F090082D75F0A3F01202E2EF900835E9E0F8A3E0F9A3E0FAA3E0FBD312008943
:2075A0005650191202E2EFEF240AFFE43EFEE43DFDE43CFC900835E912008A691202E2EF11
:2075C000900835E5E0F8A3E0F9A3E0FAA3E0FBD312008956507612014F281202CAC81202DC
:2075E000D32A900835E3E4F0A304F0900835E3E0FEA3E0FFC39405EE6480948050357C0020
:207600007D33120086B374EE2FF974193EFA90081AED7409F0A3EAF0A3E9F07F021200BACE
:2076200064900835E4E004F070C1900835E3E004F080B81202E2EFEF240AFFE43EFEE43D32
:20764000FDE43CFC900835E512008A6990082D6AE07004A3E06401700B90082D6AF0A3F0C2
:207660001202D88390082D9AE07004A3E06401700F90082D9AF0A3F01202AFC31202DE6FB8
:2076800090082D52E07004A3E06401600321738E7F01FE1202E5901202DE6FE490082D52AF
:2076A000F0A3F090082D64F0A304F0E4FFFE1202E59021738EE4FFFEFDFC90083433120020
:2076C0008A6990083531E0F9A3E0FAA3E090083425C9F0A3EAF0A3E9F0E490083431F0A3C9
:2076E000F090083431E0FEA3E0FFE4FCFD9008352DE0F8A3E0F9A3E0FAA3E0FBD3120089A9
:20770000565003217AE290083431E0FEA3E0FF7C007D2B120086B390083531E0FBA3E0FA21
:20772000A3E02FF9EA3EFAE92416F9E43AFA1200898DE47B01FAF9F8C3120089566003219D
:207740007AB690083425E0FBA3E0FAA3E0240AF9E43AFA7FFF7EFF7DFF7CFF120089C5ECB0
:207760004D4E4F6003217AB690083425E0FBA3E0FAA3E0F9A3EBF0A3EAF0A3E9F012029685
:20778000029008342BEBF0A3EAF0A3E9F090083425E0FBA3E0FAA3E02421F9E43AFA90006A
:2077A000FFFD12008BA7EBF0A3EAF0A3E9F09008342BE0FBA3E0FAA3E0F99000FFFD12004C
:2077C0008BA7EBF0A3EAF0A3E9F090083425E0FBA3E0FAA3E02421F9E43AFAE92403F9E494
:2077E0003AFA12008AD29000FFFD12008BA7EBF0A3EAF0A3E9F090083425E0FBA3E0FAA357
:20780000E02421F9E43AFA1202842A9008343AE4F0A3F0A3F0F990083437C9F0A3F0A3E99C
:20782000F090083428E0FBA3E0FAA3E02406F9E43AFA1200898DE4FBFAF9F8C312008956A8
:20784000700321793790083428E0FBA3E0FAA3E0F912008AD22179379008342EE0FBA3E085
:20786000FAA3E04A4B70032179469008342EA3A3E0240AF9E43AFA1200898DEC4D4E4F60E6
:20788000032179469008342EE0F9A3E0FAA3E09008343AC9F0A3EAF0A3E9F0E47F01FEFD1B
:2078A000FC9008343312008A699008342EE0FBA3E0FAA3E04A4B703590083428E0FBA3E067
:2078C000FAA3E02406F9E43AFA1200898DE4FBFAF9F8C3120089567002805C90083428E028
:2078E000FBA3E0FAA3E0F912008AD2804A9008342EE0FBA3E0FAA3E0F912008AD2C003C09D
:2079000002C00190083428E0FBA3E0FAA3E0F9D082D083D0E06B7008E965827003EA65838F
:207920007005FBFAF980109008342EE0FBA3E0FAA3E0F912008AD29008342EEBF0A3EAF0C6
:20794000A3E9F021785890083433E0FCA3E0FDA3E0FEA3E0FFEC4D4E4F7003217A49900897
:207960003425E0FBA3E0FAA3E0F9A3EBF0A3EAF0A3E9F0120296029008342BEBF0A3EAF068
:20798000A3E9F090083425E0FBA3E0FAA3E02421F9E43AFA9000FFFD12008BA7EBF0A3EA11
:2079A000F0A3E9F09008342BE0FBA3E0FAA3E0F99000FFFD12008BA7EBF0A3EAF0A3E9F0EC
:2079C00090083425E0FBA3E0FAA3E02421F9E43AFAE92403F9E43AFA12008AD29000FFFD6A
:2079E00012008BA7EBF0A3EAF0A3E9F090083425E0FBA3E0FAA3E02421F9E43AFA120284B5
:207A00002A9008342BE0F9A3E0FAA3E090083437C9F0A3EAF0A3E9F0A3E0FBA3E0FAA3E039
:207A2000F9C003C002C00190083437E0FBA3E0FAA3E0F9D082D083D0E06B7008E9658270B8
:207A400003EA6583600321795E90083428E0FBA3E0FAA3E02406F9E43AFA1200898DE4FBE5
:207A6000FAF9F8C3120089567002801090083428E0FBA3E0FAA3E0F912008AD29008342B38
:207A8000EBF0A3EAF0A3E9F04A4B602A9008342BE0FBA3E0FAA3E0240AF9E43AFA12008947
:207AA0008D90083425E0FBA3E0FAA3E0240AF9E43AFA120089AA90083432E004F070079010
:207AC000083431E004F090083426E475F02B12008753E4FFFEFDFC9008343312008A692114
:207AE00076E1229000FFFD12008BA7EBF0A3EAF0A3E9F09000FFF612008BA7E4FFFEFDFCC6
:207B00009000000612008BCE12008A699000000D12008BCEE0FBA3E0FAA3E0F912008AD215
:207B2000E94A4BC36001D34008E4FFFEFDFC217EF89000001012008BCEE0FBA3E0FAA3E031
:207B40004A4B6003217BCC9000000A12008BCEE0FBA3E0FAA3E0F9C003C002C00190000016
:207B60000D12008BCEE0F9A3E0FAA3E09008397EC9F0A3EAF0A3E9F0D001D002D003120229
:207B80008FB89000000D12008BCEE0FBA3E0FAA3E0F9C003C002C0019000001312008BCE6E
:207BA000E0FBA3E0FAA3E0F5828A838B93D001D002D00312008BA0E47F01FEFDFC900000AA
:207BC0000612008BCE12008A69217EE59000000D12008BCEE0FBA3E0FAA3E0F9900000033C
:207BE00012008BCEEBF0A3EAF0A3E9F09000000D12008BCEE0FBA3E0FAA3E04A4B703F908F
:207C000000000A12008BCEE0FBA3E0FAA3E02406F9E43AFA1200898DE4FBFAF9F8C3120012
:207C200089567003217E379000000A12008BCEE0FBA3E0FAA3E0F912008AD2217E3790006F
:207C4000000D12008BCEE0FBA3E0FAA3E0F912008AD2C003C002C0019000000A12008BCE1F
:207C6000E0FBA3E0FAA3E0F9D082D083D0E06B7008E965827003EA65837005FBFAF98014EC
:207C80009000000D12008BCEE0FBA3E0FAA3E0F912008AD2217E379000001012008BCEE0D9
:207CA000FBA3E0FAA3E0F9C003C002C0019000000312008BCEE0FBA3E0FAA3E0F9D082D096
:207CC00083D0E06B7008E965827003EA65837003217E4B9000000A12008BCEE0FBA3E0FABF
:207CE000A3E0F9C003C002C0019000000312008BCEE0F9A3E0FAA3E09008397EC9F0A3EA56
:207D0000F0A3E9F0D001D002D00312028FB89000000312008BCEE0FBA3E0FAA3E0F9C00391
:207D2000C002C0019000001312008BCEE0FBA3E0FAA3E0F5828A838B93D001D002D00312AD
:207D4000008BA09000000612008BCEE0FCA3E0FDA3E0FEA3E02401FFE43EFEE43DFDE43C15
:207D6000FC9000000612008BCE12008A69855783855882759308E0FBA3E0FAA3E0F99000CF
:207D8000000312008BCEEBF0A3EAF0A3E9F0855783855882759308E0FBA3E0FAA3E04A4B63
:207DA000703D9000000A12008BCEE0FBA3E0FAA3E02406F9E43AFA1200898DE4FBFAF9F809
:207DC000C3120089567002806E9000000A12008BCEE0FBA3E0FAA3E0F912008AD2805885EB
:207DE0005783855882759308E0FBA3E0FAA3E0F912008AD2C003C002C0019000000A120006
:207E00008BCEE0FBA3E0FAA3E0F9D082D083D0E06B7008E965827003EA65837005FBFAF985
:207E20008015855783855882759308E0FBA3E0FAA3E0F912008AD2855783855882759308CF
:207E4000EBF0A3EAF0A3E9F0217C979000000612008BCEE0FCA3E0FDA3E0FEA3E02401FF95
:207E6000E43EFEE43DFDE43CFC9000000612008BCE12008A699000000A12008BCEE0FBA31F
:207E8000E0FAA3E0F9C003C002C0019000000312008BCEE0F9A3E0FAA3E09008397EC9F067
:207EA000A3EAF0A3E9F0D001D002D00312028FB89000000312008BCEE0FBA3E0FAA3E0F926
:207EC000C003C002C0019000001312008BCEE0FBA3E0FAA3E0F5828A838B93D001D002D05E
:207EE0000312008BA09000000612008BCEE0FCA3E0FDA3E0FEA3E0FF9000001602008BA708
:207F00009008331EEEF0A3EFF0A3EBF0A3EAF0A3E9F07E007F047D007B097A337934120033
:207F20008F1378347C337D0990083320E0FBA3E0FAA3E0F97E007F0412008E89EF701190D5
:207F40000820F0E0700A9008332FF0A3F02180319008331FE02409F582E43412F583759348
:207F600008E0FF7E009008332FEEF0A3EFF0F460032180319008332FF0A3F09008332FE0C2
:207F8000FEA3E0FFC3941AEE648094804003218018EF7802C333CE33CED8F92457F9741017
:207FA0003EFA7B0978347C337D097E007F0412008E89EF704D90083338F0A3F090083338C5
:207FC000E0FEA3E0FFC3941AEE64809480502DE02409F582E43412F583759308E0FD9008C2
:207FE000332FE07003A3E06D601290083339E004F070C990083338E004F080C0EF641A4E87
:20800000601690083330E004F06003217F7B9008332FE004F0217F7B90083330E0FF900842
:20802000331FE02409F582E43412F583759308EFF07E017F807D007B097A1F797012008F37
:20804000139008332FE0FEA3E07802C333CE33CED8F92457F974103EA801FC7D0990083376
:2080600020E0FBA3E0FAA3E0F97E007F04120085D090083327E0FE740590083326F0A3CE09
:20808000F0A3E0FE90083328EEF0A3740CF0E49008332DF09008332DE0FFC3941A40032113
:2080A0008150EF75F004A42457F9741035F0FA900833317409F0A3EAF0A3E9F0E4900833CB
:2080C0002EF09008332EE0FFD390082D69E09F7480F890082D68E0648098406A9008332E12
:2080E000E0131313541FFE90083331E0FBA3E0FAA3E02EF9E43AFA1200864EFEEF5407FFB3
:208100007401A807088002C333D8FC5E602E9008332EE075F00CA42470F9741F35F0FA903E
:20812000083A3D7409F0A3EAF0A3E9F090083331E0FBA3E0FAA3E0F9120292309008332EBB
:20814000E004F02180C29008332DE004F0218094E49008332DF09008332DE0FFFDD39008DC
:208160002D69E09D7480F890082D68E06480985003218222EF75F004A424F1F9742035F09C
:20818000FA900833317409F0A3EAF0A3E9F0E49008332EF09008332EE0FFD390082D69E0FD
:2081A0009F7480F890082D68E0648098406A9008332EE0131313541FFE90083331E0FBA304
:2081C000E0FAA3E02EF9E43AFA1200864EFEEF5407FF7401A807088002C333D8FC5E602E72
:2081E0009008332EE075F00CA42470F9741F35F0FA90083A3D7409F0A3EAF0A3E9F0900845
:208200003331E0FBA3E0FAA3E0F9120292309008332EE004F02181949008332DE004F02160
:208220008156E49008332DF09008332DE0FFFDD390082D69E09D7480F890082D68E064806C
:208240009850032182DAEF75F005A42433F582E43426F583759308E05403FD90083326E020
:20826000FAA3E054FCFBEAFCEB4DFD90083326ECF0FCA3EDF0EF75F005A42434F582E434EE
:2082800026F583759308E07E00543F7802C333CE33CED8F9FFED5403FDEC4EFEED4FFF90EC
:2082A000083326EEF0A3EFF09008332DE075F00CA42470F9741F35F0FA9008332A7409F06F
:2082C000A3EAF0A3E9F07B097A337926120192B29008332DE004F02182289008332FE0FE0F
:2082E000A3E0FF7C007D09120086B374DC2FF974103EA801FC7D0990083323E0FBA3E0FA04
:20830000A3E0F912008D55E4900820F0F02290083603EBF0A3EAF0A3E9F0A907AA069008B2
:20832000360CEDF0A3EAF0A3E9F0E4FFFEFDFCA312008A6990083603E0FBA3E0FAA3E0F9FE
:20834000EA494B60119008360CE0FBA3E0FAA3E0F9EA494B70032183E09008360CE0FBA3B3
:20836000E0FAA3E0F990083606EBF0A3EAF0A3E9F0C002C00190083603E0F9A3E0FAA3E0D2
:20838000900837AAC9F0A3EAF0A3E9F0D001D00212027F4CEC4D4E4F705B9008360CE0FBDA
:2083A000A3E0FAA3E02421F9E43AFA90083606EBF0A3EAF0A3E9F0C002C00190083603E08B
:2083C000F9A3E0FAA3E0900837AAC9F0A3EAF0A3E9F0D001D00212027F4CEC4D4E4F7007AA
:2083E00074FFFFFEFDFC22E47F02FEFDFC9008360F12008A69E47F02FEFDFC9008360FE09B
:20840000F8A3E0F9A3E0FAA3E0FBC31200895670032185C090083603E0FBA3E0FAA3E04A6A
:208420004B7032A3E0FBA3E0FAA3E02406F9E43AFA1200898DE4FBFAF9F8C3120089567080
:2084400002805C90083606E0FBA3E0FAA3E0F912008AD2804A90083603E0FBA3E0FAA3E0B2
:20846000F912008AD2C003C002C00190083606E0FBA3E0FAA3E0F9D082D083D0E06B70086F
:20848000E965827003EA65837005FBFAF9801090083603E0FBA3E0FAA3E0F912008AD29031
:2084A000083609EBF0A3EAF0A3E9F090083606E0FBA3E0FAA3E02406F9E43AFA1200898D8F
:2084C000E4FBFAF9F8C3120089567002801090083606E0FBA3E0FAA3E0F912008AD2C00343
:2084E000C002C00190083603E0FBA3E0FAA3E0F9D082D083D0E06B7008E965827003EA658A
:2085000083706A90083609E0FBA3E0FAA3E0F9EA494B6041A3E0FBA3E0FAA3E0240AF9E4AB
:208520003AFAC003C002C0011200898D90083609E0FBA3E0FAA3E0240AF9E43AFA1200890D
:20854000E2EF2BFFEE3AFEED39FDEC38FCD001D002D0038067E4FFFEFDFC9008360CE0FBCB
:20856000A3E0FAA3E0240AF9E43AFA804F90083609E0FBA3E0FAA3E0F9EA494B604290088A
:208580003609A3A3E0240AF9E43AFAC003C002C0011200898D90083603E0FBA3E0FAA3E01D
:2085A000240AF9E43AFA120089E2EF2BFFEE3AFEED39FDEC38FCD001D002D003120089AAC2
:2085C00090083603E0FBA3E0FAA3E0F912008AD2E94A4B700321867890083603E0FBA3E049
:2085E000FAA3E02403F9E43AFA12008AD2E94A4B700321867890083603E0FBA3E0FAA3E09C
:20860000F912008AD2E92403F9E43AFA12008AD2C003C002C00190083603E0FBA3E0FAA352
:20862000E0F9D082D083D0E06B7008E965827003EA6583704390083603E0FBA3E0FAA3E0B5
:208640002403F9E43AFA12008AD212008AD2C003C002C00190083603E0FBA3E0FAA3E0F91B
:20866000D082D083D0E06B7008E965827003EA65837005FE7F0180047E007F00EF4E60712B
:2086800090083603E0FBA3E0FAA3E0F912008AD29000FFFD12008BA7EBF0A3EAF0A3E9F023
:2086A00090083603E0FBA3E0FAA3E0F99000FFFD12008BA7EBF0A3EAF0A3E9F090083603A0
:2086C000E0FBA3E0FAA3E02403F9E43AFA12008AD29000FFFD12008BA7EBF0A3EAF0A3E965
:2086E000F090083606E0FBA3E0FAA3E0F9120287EAE4FFFEFDFC90083603E0FBA3E0FAA3B7
:20870000E0240EF9E43AFA120089AA9008360FE0FCA3E0FDA3E0FEA3E0FF2290083497EB45
:20872000F0A3EAF0A3E9F0C390082D69E09401FE90082D68E09400900834A8F0A3CEF090F6
:20874000080660E0FBA3E0FAA3E0F91200877FFF900834A1E5F0F0A3EFF09008177BE0FB07
:20876000A3E0FAA3E0F990081AF0E0FEA3E0FFE92FF9EA3EFA900830567484F0A3745FF05F
:20878000A37463F01200A41690081AF1E02FF090081AF0E03EF0E49008349FF0A3F09008E7
:2087A000349FE0FEA3E0FFC3940CEE6480948040032188B4900834A2E02FFF900834A1E0D4
:2087C0003EFE900834A3F0A3EFF0C3900834A9E09FEE6480F8900834A8E0648098401E903D
:2087E00008349DE0FEA3E0FFD3900834A4E09FEE6480F8900834A3E06480984057900817A3
:208800007BE0FBA3E0FAA3E0F990081AF0E0FEA3E0FFE92FF9EA3EFA900830567484F0A32B
:20882000745FF0A37478F09008349FE0FEA3E0FFC3740C9F9008305AF0E49E90083059F0A4
:208840001200A41690081AF1E02FF090081AF0E03EF080609008177BE0FBA3E0FAA3E0F91C
:2088600090081AF0E0FEA3E0FFE92FF9EA3EFA900830567484F0A3745FF0A37490F0900828
:2088800034A3E0FFA3E090083059CFF0A3EFF01200A41690081AF1E02FF090081AF0E03E0F
:2088A000F0900834A0E004F070079008349FE004F021879E9008177BE0FBA3E0FAA3E0F98E
:2088C00090081AF0E0FEA3E0FFE92FF9EA3EFA900830567484F0A3745FF0A37463F012007B
:2088E000A41690081AF1E02FF090081AF0E03EF0E49008349FF0A3F09008349FE0FEA3E0CE
:20890000FFC3940CEE648094804003218ABC900834A2E02FFF900834A1E03EFE900834A3F1
:20892000F0A3EFF0C3900834A9E09FEE6480F8900834A8E0648098401E9008349DE0FEA32C
:20894000E0FFD3900834A4E09FEE6480F8900834A3E064809840589008177BE0FBA3E0FAC7
:20896000A3E0F990081AF0E0FEA3E0FFE92FF9EA3EFA900830567484F0A3745FF0A374784B
:20898000F09008349FE0FEA3E0FFC3740C9F9008305AF0E49E90083059F01200A416900831
:2089A0001AF1E02FF090081AF0E03EF0218ABC900834A4E024FFF0900834A3E034FFF0E0E1
:2089C000FEA3E07803CEA2E713CE13D8F8FF90083497E0FBA3E0FAA3E02FF9EA3EFA1200E7
:2089E000864EFD7C00900834A4E05407FF74017E00A807088005C333CE33CED8F9FFEE5C72
:208A0000FEEF5D4E900834A5600D7484F0A3745FF0A3749FF0800B7484F0A3745FF0A374FC
:208A2000A7F09008177BE0FBA3E0FAA3E0F990081AF0E0FEA3E0FFE92FF9EA3EFAC003C0E9
:208A400002C001900830567484F0A3745FF0A374A8F09008349AE0F9A3E0FAA3E090083031
:208A600059C9F0A3EAF0A3E9F0900834A3E0FFA3E09008305CCFF0A3EFF0900834A5E0F96B
:208A8000A3E0FAA3E09008305EC9F0A3EAF0A3E9F0D001D002D0031200A41690081AF1E039
:208AA0002FF090081AF0E03EF0900834A0E004F070079008349FE004F02188F89008066052
:208AC000E0FBA3E0FAA3E0F9E475F00C120087CD90080660E0FBA3E0FAA3E0F91200877F1D
:208AE000FFAEF0C3900834A9E09F900834A8E09E400E9008349EE09F9008349DE09E5005BD
:208B00007E007F0122E4FEFF22900839E7EBF0A3EAF0A3E9F090080403E0FBA3E0FAA3E02C
:208B2000F91200864E147003218C60147003218C6024026003218E61E4900831DBF0A3F08A
:208B4000900837CE7484F0A3743EF0A3740CF0900839E7E0FBA3E0FAA3E0F91202908C90EC
:208B60000839EAEBF0A3EAF0A3E9F0900839EAE0FBA3E0FAA3E04A4B7003FEFF229008376A
:208B8000CE7484F0A3743EF0A37420F0900839EAE0FBA3E0FAA3E0F91202908C900839EA39
:208BA000EBF0A3EAF0A3E9F0900839EAE0FBA3E0FAA3E04A4B7003FEFF227B847A3E7920D4
:208BC0001200BA43900839EBEE8FF0801B900839EAE0FBA3E0FAA3E0F91200864EB42D0E5E
:208BE000900839EBE475F0011200875380DFC3E99401F9EA9400FA900834C37484F0A374E4
:208C00003EF0A3742AF0A37484F0A3743EF0A3742CF0A37409F0A37431F0A374B9F01202D6
:208C20005965900839997484F0A3743EF0A3742FF07B097A3179B91202BD177B097A3179B8
:208C4000B91200BA43900831D9EEF0A3EFF090080403E0FBA3E0FAA3E0F974011200869F2B
:208C600090080403E0FBA3E0FAA3E0F91200864E64016003218D68900837CE7484F0A37421
:208C80003EF0A37434F0900839E7E0FBA3E0FAA3E0F91202908C900839EAEBF0A3EAF0A3F9
:208CA000E9F0900839EAE0FBA3E0FAA3E04A4B7037D3900831DCE09405900831DBE06480B0
:208CC00094804012900839EA7484F0A3743EF0A37445F0218D97900831DCE004F0706090DC
:208CE0000831DBE004F080577B847A3E79341200BA43900839EBEE8FF012008753E49008B1
:208D000031B7F0A3F090080403E0FBA3E0FAA3E0F974021200869F900839E7A3E0FAA3E010
:208D2000AE02FFA3A3E0FAA3E0C39FFFEA9EFE90081AF0E0FCA3E0FDB50708ECB50604E4A9
:208D4000FEFF22C3ED9FFFEC9E90081AF0F0A3EFF0900839EAE0F9A3E0FAA3E0900839E7BC
:208D6000C9F0A3EAF0A3E9F090081AF0E0FEA3E0FF900831B8E02FFF900831B7E03EFED341
:208D8000EF948CEE94084051900839EA7484F0A3743EF0A37457F0900839EAE0F9A3E0FA52
:208DA000A3E09008395AC9F0A3EAF0A3E9F0A37484F0A3743EF0A37478F07B847A3E79696B
:208DC0001202A5C090080403E0FBA3E0FAA3E0F9E41200869FFE7F012290081AF0E0FEA3C9
:208DE000E0FF900831B7E0FCA3E02400F974073CA801FC7D09900839E7E0FBA3E0FAA3E023
:208E0000F9120085D090081AF0E0FEA3E0FF900831B8E02FF0900831B7E03EF0900831D940
:208E2000E0FCA3E0FD900831B7E0FAA3E02400F974073AFA7B09C3E99DF9EA9CFAC3E994A7
:208E40000AF9EA9400FA900837CE7409F0A37431F0A374B9F01202908CE94A4B7003FEFF77
:208E6000221202BFE3900839EDEEF0A3EFF064014E7012900839EA7484F0A3743EF0A374C8
:208E800083F0218D97900839EDE0FEA3E0FF64024E7012900839EA7484F0A3743EF0A374C7
:208EA000A0F0218D97EF64034E7012900839EA7484F0A3743EF0A374B7F0218D9790082D07
:208EC0009AE4F0A304F090080403E0FBA3E0FAA3E0F9E41200869F900819E37410F07E0079
:208EE0007F012290083190EBF0A3EAF0A3E9F0E49008319FF0A3F0900837CE7481F0A3743B
:208F00009FF0A3747FF090083190E0FBA3E0FAA3E0F91202908C90083190EBF0A3EAF0A38B
:208F2000E9F0900834C37481F0A3749FF0A3747FF0A37481F0A3749EF0A3742CF0A3740938
:208F4000F0A37431F0A374ADF012025965E4900831A1F0A3F07B097A3179AD1200BA43C36B
:208F6000900831A2E09FEE6480F8900831A1E0648098502BA3E024ADF582E43431F58375FB
:208F80009308E0FF1202E4A54003219046900831A2E004F070BF900831A1E004F080B67B23
:208FA000097A3179AD1202851FAC06AD07900831A0E025E0FF9008319FE033FE74972FF5C4
:208FC0008274313EF583759308ECF0A3EDF090083191E475F00112008753900831A0E0046B
:208FE000F070079008319FE004F0C3900831A0E094049008319FE0648094805003218EF7F1
:20900000E4FFFEFDFC90083197E0F8A3E0F9A3E0FAA3E0FBC312008956700EFFFEFDFC900F
:2090200008319312008A698046900837627409F0A37431F0A37493F07B097A3179971202D6
:20904000448EEF4E70299008395A7481F0A374A0F0A374B5F0A37481F0A374A0F0A374C5EA
:20906000F07B817AA079A81202A5C0E4FEFF2290083193E0FCA3E0FDA3E0FEA3E0FF12027E
:20908000E6579008319FE4F0A304F09008319FE0FEA3E0FFD39404EE6480948040032192B1
:2090A000A9EE706DEF24FE601B1460451460532403705E900831AA7481F0A3749FF0A37426
:2090C00022F0804D90082DA0E0FEA3E0FF90082D55E02FFF90082D54E03E4F700321929682
:2090E000900831AA7481F0A374A0F0A374CEF08020900831AA7481F0A374A0F0A374D3F023
:20910000800F900831AA7481F0A374A0F0A374D8F0E4FFFEFDFC900831A312008A699008FF
:2091200031AAE0F9A3E0FAA3E0900837CEC9F0A3EAF0A3E9F090083190E0FBA3E0FAA3E0F8
:20914000F91202908C900831A7EBF0A3EAF0A3E9F0900831A7E0FBA3E0FAA3E04A4B70034F
:20916000219229900830567481F0A374A0F0A374DDF0900831AAE0F9A3E0FAA3E090083071
:2091800059C9F0A3EAF0A3E9F07B097A3179AD1200A416900831127409F0A37431F0A3740C
:2091A000ADF0A37409F0A37431F0A374B5F0900831A7E0FBA3E0FAA3E0F91200ADE3900890
:2091C00031A3E0F8A3E0F9A3E0FAA3E0FBC000C001E47F01FEFDFC900831B6E0F9F812002E
:2091E000897AD001D000EB4FFFEA4EFEE94DFDE84CFC900831A312008A69900831AAE0FB3A
:20920000A3E0FAA3E0F91200BA43900831A7E0FBA3E0FAA3E02FF9EA3EFA90083190EBF07D
:20922000A3EAF0A3E9F021911E9008319FE0FEA3E0FFEE7061EF24FE601F146031146043F2
:2092400024037052900831A3E0FCA3E0FDA3E0FEA3E0FF1202E65F803D900831A3E0FCA359
:20926000E0FDA3E0FEA3E0FF1202E6678028900831A3E0FCA3E0FDA3E0FEA3E0FF1202E640
:209280006F8013900831A3E0FCA3E0FDA3E0FEA3E0FF1202E677900831A0E004F07007904C
:2092A00008319FE004F021908B1202D3E87E007F0122900839AFEBF0A3EAF0A3E9F0A3746C
:2092C00002F01200877FFDACF0EC14B40F004003219641900192E275F004A4C58325F0C5B9
:2092E00083730201931E02019651020193530201938C020193C5020196510201948302016D
:20930000946702019651020194BC02019651020194C3020196510201956F020195D59008DB
:2093200039AFE0FBA3E0FAA3E0F9ED5403FFC007EDAE047802CEC313CE13D8F9543FFDE97F
:209340002404F9E43AFA12008AD2D00712013868219651900839AFE0FBA3E0FAA3E0F9126E
:2093600000877FFD5403FFC007EDAEF07802CEC313CE13D8F9543FFDE92404F9E43AFA12AE
:20938000008AD2D0071201D66C219651900839AFE0FBA3E0FAA3E0F91200877FFD5403FF7E
:2093A000C007EDAEF07802CEC313CE13D8F9543FFDE92404F9E43AFA12008AD2D007120181
:2093C0000007219651E4900839B3F0900839B3E0FFD390082D73E09F7480F890082D72E036
:2093E0006480985003219651900839AFE0FBA3E0FAA3E02404F9E43AFA12008AD2900839C3
:20940000B3E075F004A429F9EA35F0FAA3EBF0A3EAF0A3E9F0900839AFE0FBA3E0FAA3E0AF
:20942000F91200877FFD5403FFC007EDAEF07802CEC313CE13D8F9543FFD900839B4E0F9B8
:20944000A3E0FAA3E090083AB4C9F0A3EAF0A3E9F0900839B3E0FBD0071202D49E90083947
:20946000B3E004F02193CB900839AFE0FBA3E0FAA3E02404F9E43AFA12008AD212021DAE05
:20948000219651900839AFE0FBA3E0FAA3E0F91200877FFD5403FFC007EDAEF07802CEC3A8
:2094A00013CE13D8F9543FFDE92404F9E43AFA12008AD2D0071202238F219651900839B29F
:2094C0007401F0E4900839B3F0900839B3E0FFD390082D73E09F7480F890082D72E06480FB
:2094E000985003219651900839AFE0FBA3E0FAA3E02404F9E43AFA12008AD2900839B3E013
:2095000075F004A429F9EA35F0FAA3EBF0A3EAF0A3E9F0900839AFE0FBA3E0FAA3E0F91236
:2095200000877FFD5403FFC007EDAEF07802CEC313CE13D8F9543FFD900839B4E0F9A3E03F
:20954000FAA3E0900836BCC9F0A3EAF0A3E9F0900839B2E0900836BFF0900839B3E0FBD043
:209560000712029A59900839B3E004F02194C9900839AFE0FBA3E0FAA3E0F91200877FFD9E
:209580005403FFC007EDAEF07802CEC313CE13D8F9543FFDE92404F9E43AFA12008AD21221
:2095A00000864EFBC003900839AFE0FBA3E0FAA3E02404F9E43AFA12008AD2E92401F9E42C
:2095C0003AFA1200864E90083A52F0D003D007120270A6807C900839AFE0FBA3E0FAA3E032
:2095E000F91200877FFD5403FFC007EDAEF07802CEC313CE13D8F9543FFDE92404F9E43A2D
:20960000FA12008AD2C003C002C001900839AFE0FBA3E0FAA3E02404F9E43AFA12008AD29A
:20962000E92401F9E43AFA900839E4EBF0A3EAF0A3E9F0D001D002D003D0071202E093802E
:2096400010900839AFE0FBA3E0FAA3E0F91202E45A7F0022900832C7EEF0A3EFF0E4900846
:2096600032E3F0900832E3E0FFD390082D73E09F7480F890082D72E0648098403390083213
:20968000E3E025E024D2F582E43432F583759308E4F0A3F0EF25E024D8F582E43432F58333
:2096A000759308E4F0A3F0900832E3E004F080B3E4900832D1F07F01FEFDFC21981A90082E
:2096C00032D1E0FFFDD390082D69E09D7480F890082D68E06480985003219825EF75F0052E
:2096E000A42434F582E43426F583759308E0900832E2F0C3940A4009E0D394115003E0047C
:20970000F0900832D1E075F005A42433F582E43426F583759308E0900832E3F0900832DE17
:20972000E0FCA3E0FDA3E0FEA3E0FF900832C9E0F8A3E0F9A3E0FAA3E05FFFEA5EFEE95DF9
:20974000FDE85C4D4E4F6045900832E3E025E024D2F582E43432F583C083C082759308E003
:20976000FCA3E0FD900832E2E0FF74017E00A807088005C333CE33CED8F9FFEC4EFEED4FAA
:20978000FF759308D082D083EEF0A3EFF0900832DEE0FCA3E0FDA3E0FEA3E0FF900832CD17
:2097A000E0F8A3E0F9A3E0FAA3E05FFFEA5EFEE95DFDE85C4D4E4F6045900832E3E025E009
:2097C00024D8F582E43432F583C083C082759308E0FCA3E0FD900832E2E0FF74017E00A83D
:2097E00007088005C333CE33CED8F9FFEC4EFEED4FFF759308D082D083EEF0A3EFF0900820
:2098000032D1E004F0900832DEE0FCA3E0FDA3E0FEA3E0FF78011200897A900832DE120022
:209820008A692196BEE4900832E3F0900832E3E0FFFD90082D72E0FAA3E0FBD39D7480F8CB
:20984000EA64809850032199E0D3EB9401EA648094804025EF25E024D2F582E43432F583F8
:20986000C083C082759308E04402FFA3E0759308D082D083CFF0A3EFF090082D90E024015B
:20988000FF90082D8FE03400FE90082D5FE02FFF90082D5EE03EFE90082D55E02FFF900832
:2098A0002D54E03EFE90082DA1E02FFF90082DA0E03ECFC39401CF9400FE9008263375F036
:2098C00005EF12008A86EE75F005A42583F583759308E0FF900832E3E0B50738FF25E024BE
:2098E000D2F582E43432F583C083C082759308E04401FDA3E0759308D082D083CDF0A3ED21
:20990000F0EF25E024D8F582E43432F583759308E054FEF0900832E3E025E024D8F582E413
:209920003432F583759308E0541FFEA3E0FFE4FCFD900832DE12008A69900832DEE0FCA3B5
:20994000E0FDA3E0FEA3E0FF780D1200897A900832DE12008A69900832DEE0F8A3E0F9A341
:20996000E0FAA3E0FB900832E3E025E024D2F582E43432F583759308E0541FFEA3E0FFEB00
:209980004FFFEA4EFEE9FDE8FC900832DE12008A69900832DEE0FCA3E0FDA3E0FEA3E0FFC5
:2099A000EC4404FC900832DE12008A69900832DEE0FCA3E0FDA3E0FEA3E0FF900833901256
:2099C000008A69900832C7E0FCA3E0FD900832E3E0FF12027731900832E3E004F021982BFA
:2099E0007F00229008064FE0FBA3E0FAA3E0F91200877FFFAEF0E5F06003219D67EF24FEE2
:209A0000602E147003219B5C147003219D2924036003219D677F017E00120299A49008060F
:209A20004FE0FBA3E0FAA3E0F9E475F002219D60C390082D69E09401FF90082D68E0940094
:209A4000F990080659E0FBA3E0FAA3E0C98FF0120087F9900830567484F0A37430F0A3740D
:209A6000F2F09008177BE0FBA3E0FAA3E0F91200A41690081AF0EEF0A3EFF0900838CBE4B9
:209A8000F0A304F090080659E0FBA3E0FAA3E0F91200877FFF900838CBE0FCA3E0FDD39FF4
:209AA000EC95F050549008177BE0FBA3E0FAA3E0F990081AF0E0FEA3E0FFE92FF9EA3EFA5E
:209AC000900830567484F0A3742DF0A374B9F0A3ECF0A3EDF01200A41690081AF1E02FF01F
:209AE00090081AF0E03EF0900838CCE004F07094900838CBE004F0808B9008177BE0FBA320
:209B0000E0FAA3E0F990081AF0E0FEA3E0FFE92FF9EA3EFA900830567484F0A3742DF0A3DD
:209B200074C7F01200A41690081AF1E02FF090081AF0E03EF090080660E0FBA3E0FAA3E003
:209B4000F9E475F001120087F99008064FE0FBA3E0FAA3E0F9E475F003219D60900806590E
:209B6000E0FBA3E0FAA3E0F91200877FFFAEF090080660E0FBA3E0FAA3E0F91200877FD39F
:209B80009FE5F09E402B9008064FE0FBA3E0FAA3E0F9E475F004120087F9D390081AF1E052
:209BA000940090081AF0E094005003219D297F00229008177BE0FBA3E0FAA3E0F990081A70
:209BC000F0E0FEA3E0FFE92FF9EA3EFA900830567484F0A3742EF0A3740FF01200A4169055
:209BE000081AF1E02FF090081AF0E03EF0900838CBE4F0A37402F0900838CBE0FEA3E0FF30
:209C0000C3EE648094805003219CFEEF4E701AA37484F0A3742EF0A37417F0A37484F0A3BA
:209C2000742CF0A374CEF0801B900838CD7484F0A3742CF0A374CEF0A37484F0A3742EF0D7
:209C4000A3741FF09008177BE0FBA3E0FAA3E0F990081AF0E0FEA3E0FFE92FF9EA3EFAC0EB
:209C600003C002C001900830567484F0A3742EF0A37424F090080660E0FBA3E0FAA3E0F926
:209C80001200877FC39401FEE5F0940090083059F0A3CEF0900838CBE0FFA3E09008305B5B
:209CA000CFF0A3EFF0900838CDE0F9A3E0FAA3E09008305DC9F0A3EAF0A3E9F0900838D076
:209CC000E0F9A3E0FAA3E090083060C9F0A3EAF0A3E9F0D001D002D0031200A41690081ADD
:209CE000F1E02FF090081AF0E03EF0900838CCE024FFF0900838CBE034FFF0219BF790084C
:209D00000660E0FBA3E0FAA3E0F9E475F001120087CDC390081AF1E0948490081AF0E094E5
:209D2000035003219B5C7F0022900830567484F0A37432F0A3743CF09008177BE0FBA3E00A
:209D4000FAA3E0F91200A41690081AF0EEF0A3EFF09008064FE0FBA3E0FAA3E0F9E4F5F035
:209D6000120087F97F00227F01229008383CE0FBA3E0FAA3E02428F9E43AFA90083C4AEBC1
:209D8000F0A3EAF0A3E9F0E475F001120087F990083C4BE475F002120087531202E6DEEFE1
:209DA0002404FFE43EF990083C4AE0FBA3E0FAA3E0C98FF0120087F990083C4BE475F00224
:209DC000120087531202DF2490083059EBF0A3EAF0A3E9F0900830567481F0A37480F0A35E
:209DE0007404F090083C4AE0FBA3E0FAA3E0F91200A4161202E6DE90083C4BEE8FF01200C7
:209E0000875390083C4AE0FBA3E0FAA3E0F9E475F002120087F990083C4BE475F00212001D
:209E2000875390083C4AE0FBA3E0FAA3E0F9E475F018120087F990083C4BE475F0021200E7
:209E400087531202E6A9C003C00290083C4AE0FBA3E0FAA3E0F8AC02AD03D002D0037E008E
:209E60007F14120085D090083C4BE475F0141200875390083C4AE0FBA3E0FAA3E0F9E47535
:209E8000F003120087F990083C4BE475F0021200875390083C4AE0FBA3E0FAA3E0F9E4759C
:209EA000F018120087F990083C4BE475F002120087531202E6B0C003C00290083C4AE0FB8A
:209EC000A3E0FAA3E0F8AC02AD03D002D0037E007F14120085D090083C4BE475F014120081
:209EE000875390083C4AE0FBA3E0FAA3E0F9E475F004120087F990083C4BE475F00212003B
:209F0000875390083C4AE0FBA3E0FAA3E0F9E475F008120087F990083C4BE475F002120016
:209F200087531202E30F90083C4AE0FBA3E0FAA3E0F9120089AA90083C4BE475F00412008C
:209F4000875390083C4AE0FBA3E0FAA3E0F9E475F005120087F990083C4BE475F0021200D9
:209F6000875390083C4AE0FBA3E0FAA3E0F9E475F008120087F990083C4BE475F0021200B6
:209F800087531202E31F90083C4AE0FBA3E0FAA3E0F9120089AA90083C4BE475F00412001C
:209FA000875390083C4AE0FBA3E0FAA3E0F9E475F006120087F990083C4BE475F002120078
:209FC000875390083C4AE0FBA3E0FAA3E0F9E475F008120087F990083C4BE475F002120056
:209FE00087531202E32F90083C4AE0FBA3E0FAA3E0F9120089AA90083C4BE475F0041200AC
:20A00000875390083C4AE0FBA3E0FAA3E0F9E475F007120087F990083C4BE475F002120016
:20A02000875390083C4AE0FBA3E0FAA3E0F9E475F008120087F990083C4BE475F0021200F5
:20A0400087531202E33F90083C4AE0FBA3E0FAA3E0F9120089AA90083C4BE475F00412003B
:20A06000875390083C4AE0FBA3E0FAA3E0F9E475F015120087F990083C4BE475F0021200A8
:20A08000875390083C4AE0FBA3E0FAA3E0F9E475F006120087F990083C4BE475F002120097
:20A0A00087531202E5CC90083C4AE0FBA3E0FAA3E0F9EE8FF0120087F990083C4BE475F0A8
:20A0C00002120087539008383CA3E0FAA3E0AE02FF90083C4AA3E0FAA3E0C39FFFEA9E9040
:20A0E000081AF0F0A3EFF0221202E33F9008277F12008A691202E35F9008277B12008A69AC
:20A1000090082D90E02401FF90082D8FE03400FE90082D5FE02FFF90082D5EE03ECFC394E7
:20A1200001CF9400900826DDF0A3EFF090082D90E02401FF90082D8FE03400FE90082D5FCB
:20A14000E02FFF90082D5EE03EFE90082D55E02FFF90082D54E03EFE90082DA1E02FFF9051
:20A16000082DA0E03ECFC39401CF9400FEC3900826DEE09FEE6480F8900826DDE0648098C5
:20A18000400321A462A3E0FF7B097A2679E31202A96990082723E0FCA3E0FDA3E0FEA3E0EB
:20A1A000FF9008275BE0F8A3E0F9A3E0FAA3E02FFFEA3EFEE93DFDE83CFC90082743E0F8C1
:20A1C000A3E0F9A3E0FAA3E02FFFEA3EFEE93DFDE83CFCA3E0F8A3E0F9A3E0FAA3E02FFF47
:20A1E000EA3EFEE93DFDE83CFC9008274FE0F8A3E0F9A3E0FAA3E02FFFEA3EFEE93DFDE835
:20A200003CFC9008276FE0F8A3E0F9A3E0FAA3E02FFFEA3EFEE93DFDE83CFCA3E0F8A3E0EF
:20A22000F9A3E0FAA3E02FFFEA3EFEE93DFDE83CFC900826DF12008A69900826DDE0FEA3D0
:20A24000E07802C333CE33CED8F92413F582741C3EF583759308E0F8A3E0F9A3E0FAA3E0B6
:20A26000FB900826DFE0FCA3E0FDA3E0FEA3E0C39BFFEE9AFEED99FDEC98FCE47B32FAF97C
:20A28000F8C3120089565056E4FFFEFDFC9008277FE0F8A3E0F9A3E0FAA3E0FBC3120089A7
:20A2A00056603B9008277BA3A3A3E05404FFEF602D900826DEE02401FF900826DDE0340088
:20A2C000FE3395E0FDFC90083A0112008A69E490083A05F0A3F07FD57E071202786090086C
:20A2E00026DFE0FCA3E0FDA3E0FEA3E0FFC004C005C006C007900826DDE0FEA3E07802C3AB
:20A3000033CE33CED8F92413F582741C3EF583759308D007D006D005D00412008A69900873
:20A32000270BE0FCA3E0FDA3E0FEA3E0FF900826EBE0F8A3E0F9A3E0FAA3E02FFFEA3EFE3B
:20A34000E93DFDE83CFC9008270FE0F8A3E0F9A3E0FAA3E02FFFEA3EFEE93DFDE83CFC9071
:20A360000826DF12008A69900826DDE0FEA3E07802C333CE33CED8F92493F582741C3EF5CE
:20A3800083759308E0F8A3E0F9A3E0FAA3E0FB900826DFE0FCA3E0FDA3E0FEA3E0C39BFF81
:20A3A000EE9AFEED99FDEC98FCE47B32FAF9F8C3120089565056E4FFFEFDFC9008277FE046
:20A3C000F8A3E0F9A3E0FAA3E0FBC312008956603B9008277BA3A3A3E05408FFEF602D9055
:20A3E0000826DEE02401FF900826DDE03400FE3395E0FDFC90083A0112008A69E490083A71
:20A4000005F0A3F07FD67E0712027860900826DFE0FCA3E0FDA3E0FEA3E0FFC004C005C0A9
:20A4200006C007900826DDE0FEA3E07802C333CE33CED8F92493F582741C3EF583759308BF
:20A44000D007D006D005D00412008A69900826DEE004F0600321A12C900826DDE004F02150
:20A46000A12C22900836AAEBF0A3EAF0A3E9F0E4FFFEFDFCA312008A6990083525E0FCA3AE
:20A48000E0FDA3E0FEA3E0FFEC4D4E4F600321A7CA900836AAE0FBA3E0FAA3E0F91200892A
:20A4A0008DE47B2BFAF9F8120088151202677490083531EBF0A3EAF0A3E9F090083531E04C
:20A4C000FBA3E0FAA3E04A4B700321A7CA900836AAE0FBA3E0FAA3E0F91200898D900835A6
:20A4E0002D12008A69E47F2BFEFDFC9008352DE0F8A3E0F9A3E0FAA3E0FB120088157D0030
:20A5000090083531E0FBA3E0FAA3E0F912008F13E4FFFEFD21A74F9008352DE0FCA3E0FD6A
:20A52000A3E0FEA3E0FF900836B1E0F8A3E0F9A3E0FAA3E0FBC312008956400321A75B90A0
:20A540000836B1E0FCA3E0FDA3E0FEA3E0FF7A007B2B1200881590083531E0FBA3E0FAA3E5
:20A56000E02FF9EA3EFAEB3DFBC003C002C00190083531E0FBA3E0FAA3E0F9900836B1E017
:20A58000FCA3E0FDA3E0FEA3E0FFF5828E83742B12008A75E92582F9EA3583FA12008AEF54
:20A5A0007A007B2B1200881590083531E0FBA3E0FAA3E02FF9EA3EFAEB3DFBC003C002C041
:20A5C00001E47F2BFEFDFC900836B1E0F8A3E0F9A3E0FAA3E0FB1200881590083531E0FB9F
:20A5E000A3E0FAA3E02FF9EA3EFAE92403F9E43AFA12008AEFE4FFFEFDFCC004C005C0063C
:20A60000C0077F2B900836B1E0F8A3E0F9A3E0FAA3E0FB1200881590083531E0FBA3E0FAF6
:20A62000A3E02FF9EA3EFAE92406F9E43AFAD007D006D005D004120089AA900836B1E0FC33
:20A64000A3E0FDA3E0FEA3E0FF7A007B2B1200881590083531E0FBA3E0FAA3E02FF9EA3E7F
:20A66000FAEB3DFBE92421F9E43AFAC003C002C00190083531E0FBA3E0FAA3E02FF9EA3E0F
:20A68000FAEB3DFBE92421F9E43AFA12008AEF90083531E0FBA3E0FAA3E02FF9EA3EFAEBC5
:20A6A0003DFBE92421F9E43AFAC003C002C001E47F2BFEFDFC900836B1E0F8A3E0F9A3E002
:20A6C000FAA3E0FB1200881590083531E0FBA3E0FAA3E02FF9EA3EFAE92421F9E43AFAE908
:20A6E0002403F9E43AFA12008AEFE4FFFEFDFCC004C005C006C0077F2B900836B1E0F8A303
:20A70000E0F9A3E0FAA3E0FB1200881590083531E0FBA3E0FAA3E02FF9EA3EFAE92421F96C
:20A72000E43AFAE92406F9E43AFAD007D006D005D004120089AA900836B1E0FCA3E0FDA3C4
:20A74000E0FEA3E02401FFE43EFEE43DFDE43CFC900836B112008A6921A517900836ADE05E
:20A76000FCA3E0FDA3E0FEA3E0FFEC4D4E4F601290083531E0FBA3E0FAA3E0F9120210A379
:20A78000804890083521E0F8A3E0F9A3E0FAA3E0FB90083529E0FCA3E0FDA3E0FEA3E0FF5F
:20A7A000120088A0900836B512008A69E47F01FEFDFC9008352512008A69900836ADE0FC2E
:20A7C000A3E0FDA3E0FEA3E0FF2274FFFFFEFDFC229008385CECF0A3EDF0A3EBF0A3EAF0C6
:20A7E000A3E9F0900838627409F0A37438F0A3745CF0EF14700990083865744AF080079026
:20A800000838657440F03096032095041202CDD61202E496900838651202AEA0A2109296B7
:20A820001202AF32D2951202AF32C295D2341202AF32D2961202AF32D2951202AF32A29684
:20A840009234C2951202AF3230340321A94C90083861E06010A3E0FBA3E0FAA3E02401F94C
